:020000041800E2
:10D0000008A055AA12082220FF21513101803121A8
:10D01000090141808180C1807721C9000181972168
:10D02000C9004181AF21C900818159210901C18114
:10D03000692109010182DF21C900418202498182FF
:10D040000249C18270470000F80B0000F80E000092
:10D0500072B6BFF34F8F04490248C860BFF34F8FC9
:10D06000FEE700000400FA0500ED00E030B5D31C37
:10D070009C0883000A4D5118A40089085B19890097
:10D08000091B400040199C6101849869418099699D
:10D09000044808809969002048609969886030BD1B
:10D0A000509000205AA50000C088884201D101207C
:10D0B000704700207047082807D2EFF3108272B63D
:10D0C0008000024B195082F3108870477490002042
:10D0D0007FB505460E46EFF3108472B602A80DF038
:10D0E00046FB84F310880298039900900191281A56
:10D0F000000101210009C906884205D20098A84212
:10D1000005D10198864202D8012004B070BD0020EC
:10D11000FBE730B5C368826888680125141A2401CA
:10D12000C9682409ED06AC4203D2904203D18B4278
:10D1300001D8012030BD002030BD0A0C838889B29F
:10D14000934204D1C088884201D101207047002059
:10D1500070470000072803D2024A8000801841600F
:10D1600070470000949000200CB5002807D00DA156
:10D1700006C96844203801920091C07F0CBDFF2091
:10D18000F5300CBD0CB5014606A005C80192009013
:10D1900000206A46135C8B4203D3401CC0B20728B0
:10D1A000F8D30CBDFA96644B321E140070B50E46CF
:10D1B0001C46154601210DF063F846608560446108
:10D1C00070BD70B50C460646014615464F480CF03A
:10D1D00099FF4F4A3561F460137820462946002BA9
:10D1E00003D1012313700DF070FB70BDF8B51C4620
:10D1F000069B002A0E46054622460DD00021382007
:10D20000FFF7D4FF434F0446002D0CD010222046D8
:10D2100029461830B8470DE000211820FFF7C6FF57
:10D220003246294610E020463A4B102200211830A1
:10D230005C33984710222046283031460546B847CF
:10D2400021462A4618312046FFF7BBFFF8BDF0B54E
:10D2500089B00E460746002401AD0DF053FAA10037
:10D26000641CE4B26850082CF7D33B46012205A9A0
:10D2700001A80096FFF7BAFF09B0F0BD70B50546EA
:10D280000E4622480CF05BFF04462048002200684E
:10D290001F4900280A7005D001220A700169C06880
:10D2A0000DF013FB002C13D0002D07D16268002A6B
:10D2B00004D0314620469047002809D0A368002BAF
:10D2C00003D0314628466269984720460DF032F86F
:10D2D00070BD30B55B1E5BB2002B04DBCC5CD55C53
:10D2E0006C40C454F6E730BD10B50F228418203CC2
:10D2F000835CE47F5B00E40923438B54521E1206D7
:10D30000120EF3D100784000087010BDB4900020D8
:10D31000DC920020190F0000F0B504468BB000200D
:10D320002646203608900F46F07CB17C884212D207
:10D33000218E0001081AA16910234218394630468F
:10D34000FFF7C7FF32462046E169FFF73AFFF07C5E
:10D35000401CF0746DE0FE2809D2FE20F0744A4BA8
:10D3600010223946304698470022E16930E0FF2814
:10D370005DD2FF20F074208E10210CF0E5FDF87BCB
:10D38000CDB2C009099069463846FFF7ADFF09984C
:10D39000002805D06946087887214840694608700A
:10D3A000002D19D1B07C002816D0374B102204A8CC
:10D3B000A169984704A910236A460846FFF789FF28
:10D3C0003246102304A91046FFF783FFE169324675
:10D3D0002046FFF7F6FE2CE06846C07B6946C70989
:10D3E0000846FFF781FF002F05D06946087887219E
:10D3F0004840694608701021491B8C4600200F21C7
:10D400004F1B04ABA84204D2A1690A5C614609180B
:10D4100007E0A84202D18022DA5503E000220F2162
:10D42000091A5A54401CC0B21028EBD3C2E701209D
:10D43000089008980BB0F0BD70B582610386044671
:10D44000C1610F33180925462035A87401200E4B01
:10D45000E8741022002128465C339847294620466C
:10D46000FFF75AFF70BDF8B51F4614460D46064635
:10D470003A4606493420069BFFF798FE23462A4683
:10D480003146FFF7D9FFF8BD190F000019D3001876
:10D49000F8B5064604462036307E0025002802D026
:10D4A00001252846F8BD2046224618301023283290
:10D4B0000746FFF70EFF012030763A462046E16826
:10D4C000FFF77FFEEDE7FFB581B016460F46054634
:10D4D0000E493C200B9B0A9AFFF768FE0446324631
:10D4E0001830102339460646FFF7F3FE1022204677
:10D4F000074B2830049998470021382001553246BF
:10D5000029462046FFF75DFE05B0F0BD91D4001816
:10D51000190F0000F3B581B00F46486801994968BA
:10D52000421A140101222409D206944203D9081A8E
:10D530000001000944420198BD688668002C02DCA5
:10D5400028D1AE4226D20069FA493018451B281E60
:10D5500004DD681E0CF00EFD201A03E00CF00AFD3D
:10D56000201A401C002801DD0020FEBD3869F14969
:10D57000281A002804DD401E0CF0FCFC201A03E0F1
:10D580000CF0F8FC201A401C002801DD0120FEBD33
:10D590000220FEBD3F69E749E819801B002805DD30
:10D5A000401E0CF0E7FC0019401C02E00CF0E2FC0D
:10D5B0000019002801DC0520FEBD0198DD49006945
:10D5C0003018401BC01B002804DD401E0CF0D2FCAC
:10D5D000201A03E00CF0CEFC201A401C002801DDCC
:10D5E0000320FEBD0420FEBDF1B584B0D2480090FA
:10D5F0000027046857E0A08A22688105890E0292FC
:10D60000820B4ED000294CD0002201921646A27DFA
:10D6100003071B0FD2180901049D1039A275890553
:10D62000890D3F22120190430143A18234E0294633
:10D630002046FFF76FFF002830D005282AD029693F
:10D64000A8684618BB4930460CF07EFC0146686865
:10D65000B84B40185943A268711A8A4200D2401C44
:10D66000060136096660A08A800B022812D3B149F0
:10D6700020690CF069FCE1680346881B0001012267
:10D680000009D206904203D9701A000100094042F5
:10D69000834206DC2E462D68002DC8D10198002853
:10D6A00017D02746029C002CA5D1009800680028BE
:10D6B0000DD0082105200007016282698A430A43D0
:10D6C000826101680122D20691431143016005B0D5
:10D6D000F0BD2246394600980CF056FD9648224689
:10D6E00031460C380CF09CFDDCE7FEB592480C3856
:10D6F0000068002826D0C27D41688768891A0E011B
:10D70000360968460DF033F8019D8A48FF3591359A
:10D71000009C854204D340422D18641C2401240936
:10D72000301B000101210009C906884203D2B4421E
:10D7300003D1AF4201D826462F46394630460DF078
:10D740003AF8FEBD0021481EF9E7F0B505467A48D3
:10D7500087B00C38059000200646019000900746DF
:10D760000290EFF31080069072B603A80CF0FFFF52
:10D77000E97D03987D22401804990001D2006D4B89
:10D78000000989185B4203E0C918401C0001000928
:10D79000684A9142F8D26A68131A1C0101232409CD
:10D7A000DB069C4204D282420DD1AA6891420AD97A
:10D7B000AA8A920B1FD06860AA688A4203D2401CD2
:10D7C000000100096860A88A800B022816D3594915
:10D7D00028690CF0B9FBEA6869680446501A000130
:10D7E00001230009DB06984203D9881A00010009C9
:10D7F0004042844202DD0120029094E04E480C3801
:10D800008468002C67D10598046864E021462846A6
:10D81000FFF780FE002860D0052839D0A97DA27DC1
:10D8200091420FD9444B0C3B9B68A3420AD0002E77
:10D8300000D126467F1CFFB2009401284DD003285A
:10D840004BD025E0AB8A9B0B17D02169A068461806
:10D85000384930460CF078FB01466068354B40187B
:10D860005943AA68711A8A4200D2401C000100097B
:10D8700000266860374600960AE09142BBD92E49DF
:10D880000C398968A142B6D1032826D00428B2D128
:10D89000A88A800B022815D3264928690CF054FB6E
:10D8A0000346E86869688446401A000101220009BD
:10D8B000D206904204D96046081A0001000940428D
:10D8C000834298DC1C480C388068A0429BD0002F13
:10D8D00000D101942468002C98D10298002822D10C
:10D8E000002E0AD01448009A0C3801990CF059FC0B
:10D8F00031461148009A0CF010FC0198002806D01F
:10D9000001460D482A460C380CF08AFC06E00A480D
:10D9100029460C380CF00CFCFFF7E7FE002E02D075
:10D920002846FFF761FE069880F31088029807B03A
:10D93000F0BD000071020000C890002070B50446E0
:10D940000026EFF3108572B600281FD011488268B8
:10D95000A24202D10021816018E0002916D100689E
:10D96000A04205D10B480CF0EAFBFFF7BEFE0DE02C
:10D97000214608480CF0EDFB002807D10548214658
:10D980000C300CF0E6FB002800D1022685F310884D
:10D99000304670BDBC900020FFB5394D0646EC7C8A
:10D9A000A87C81B0201A0007000F8C460E2801D3F6
:10D9B000012000E000200090314AA000803A811848
:10D9C00077680F64111980310B7061461150012086
:10D9D000298AA040014329822A492201B088571888
:10D9E000788070680001000DB88030892721090116
:10D9F000081AF88024493069884208D92349401818
:10DA00000CF0A2FA0121C9030143798105E0C103A9
:10DA10000120C0030818000C78810A981F211F28D4
:10DA200000D308460002B881F8891F210902884303
:10DA30000F2109020843F881039870214843FF3001
:10DA4000513080083881B07D1F211F2800D308463F
:10DA50000099C002890202220843104338809007CF
:10DA60000B4920430860E87C401C0007000FE87465
:10DA70000848018820221143018005B0F0BD000054
:10DA80005091002000800020FF7F00007102000004
:10DA90000001005000900020FFB58FB0064611989D
:10DAA0001F46304363D0012E01D1002F5FD00020EC
:10DAB0000690012E04D011988068002E02D006E056
:10DAC0007868FAE71099002901D01198C068089089
:10DAD000012E0AD01198008A0990012E07D01198C2
:10DAE000C07C002803D0012002E0B889F4E70020C0
:10DAF00000900CF031FE0001C00F0190D0480021D1
:10DB00008160D0488079002815D00198002812D172
:10DB1000CB4804680DE0A5880120294600070CF0D9
:10DB200013FA681AE188401829460CF023FAE180BC
:10DB30002468002CEFD1C34901988871012E14D0BC
:10DB400011984069019008980D90019800280ED016
:10DB50000D9800280BD0012E0CD0009800280BD077
:10DB60000125B7480468059482E03868EAE7012097
:10DB700013B0F0BDBD68F4E70025F2E7002E04D134
:10DB80001098002801D0678900E02789A0880290BA
:10DB900000286CD0002F6AD0A1890998814266D0F4
:10DBA00001990298884200D3084604900D983918CC
:10DBB0000498814201D90320DAE7E08804990CF047
:10DBC000C3F9CF1907917F1E049901980CF0BCF995
:10DBD00000294CD1049902980CF0B6F9002946D1DD
:10DBE000284604990CF0B0F90D980A910818401EC7
:10DBF00003900798814201D3B9421ED9079903982F
:10DC0000884201D3B84218D90A98884202D80398AA
:10DC1000B84212D20498874206D3014638460CF027
:10DC200093F90A98814208D20499039888421ED336
:10DC30000CF08AF90798814219D3012E04D0781C80
:10DC400004990CF081F905E07D48019D84600CE0A9
:10DC500004980918A942FBD900980D46A84303D19E
:10DC600000988143C80700D06D1C059C00E0246823
:10DC7000002C02D00198854280D30198854202D3BE
:10DC8000032006903DE0002E3BD11198856111984C
:10DC900046690898019500901198AD19008A039083
:10DCA0006D1E059C25E0A1890398814220D0A088A3
:10DCB0000290B04201D3374600E00746394630466D
:10DCC0000CF042F9002913D1394602980CF03CF9C6
:10DCD00000290DD1E08839460CF036F900E0C91969
:10DCE00001988142FBD90098081AA84200D2054643
:10DCF0002468002CD7D1314628460CF025F911981C
:10DD0000C161069834E71FB50446808800902089D9
:10DD10000190A08969468881E088002202906B46C4
:10DD200011460120FFF7B8FE032819D14448806846
:10DD3000002815D0E17B002902D1C27B002A0FD038
:10DD4000002901D0224600E00246002905D0C37B0D
:10DD5000002B02D0994200D20246908909F0CFFBF5
:10DD6000214637480CF0CEF91FBD10B501463448A6
:10DD70000CF0EFF910BDFEB50446406800906061FC
:10DD8000216800980291814242D20025ED432E463F
:10DD900000212B4809E08289238A9A4205D0491C38
:10DDA0008288C9B2B24200D2164600680028F2D179
:10DDB000002908D00098B0420FD331460CF0C4F8C7
:10DDC000704305461DE0A67C002E1AD0314600980F
:10DDD0000CF0BAF83546454313E0074600200190A1
:10DDE00009E0394630460CF0AFF8002902D1012095
:10DDF0003D460190BF1E0298B84202D80198002803
:10DE0000EFD00298A84203D80098A84200D36561D9
:10DE10000023224601211846FFF73EFE002809D0C4
:10DE2000E268A168914205D20023224619461846AD
:10DE3000FFF732FEFEBD00220346114601202BE60D
:10DE400064910020D09200201CB541480468002C49
:10DE50001ED068460CF08BFC01980099E02801D395
:10DE6000012000E00020401C08180001000900907B
:10DE700060680099401A000101210009C906884222
:10DE800001D2606801E0009860600CF083FC1CBD6A
:10DE90000020C043F9E7FEB506460025EFF31087E2
:10DEA00072B668460CF063FC019800997C2801D397
:10DEB000012000E00020401C08180001000900902B
:10DEC00070680099401A010101200909C0068142C9
:10DED00001D3009971601E490C6808E0616872689E
:10DEE000891A09010909814203D325462468002CB7
:10DEF000F4D1002D05D03246294615480CF090F992
:10DF000005E0314612480CF013F9FFF79DFF87F347
:10DF10001088FEBD70B50025EFF3108472B60C4E6C
:10DF20003168814208D130460CF009F93068002888
:10DF300009D0FFF789FF06E0014605480CF009F912
:10DF4000002800D1022584F31088284670BD000007
:10DF500070910020F8B53E483C4981800021C943BA
:10DF600001603C48384F46681DE030460CF09BFB92
:10DF70001F210D1A3748A90009188C68002C0FD0F2
:10DF800069000818008B34490BF0DEFF201A84B2B8
:10DF9000022C01D9A41EA4B2A74200D23C46A7B2CB
:10DFA0000120A8408643002EDFD1294A2A499088C3
:10DFB0004F43B84200D33846908026480068411C41
:10DFC0000AD011684B1C06D0091A0901012309095E
:10DFD000DB06994200D31060F8BD022801D11D482C
:10DFE0000160B7E710B5022802D11A49C01E0860C7
:10DFF000FFF7B0FF16480068401C01D10AF0D6FABE
:10E0000010BD30B4032801D004280BD111488C0076
:10E010002418A2604A0012181383012342688B401F
:10E020001A43426030BC95E7032801D0042809D187
:10E0300008488B0000221B189A60012342688B401D
:10E040009A43426086E70000FFFF0000E4570000AB
:10E05000D09200207891002071020000F8B50746A8
:10E06000000214460E460025C01D0CF030FA21783F
:10E0700043233F2818D01F2816D0FA49BA008A58DF
:10E08000B300D158A1420DD00121B140014201D0CD
:10E0900002250EE00125D450C9B22A46384601F0C7
:10E0A000D1FD06E0012504E00C3C2289384601F050
:10E0B000E1FD2846F8BD70B50D46044601F0DEFED0
:10E0C000C0B2294609F02EF900281AD0112809D02B
:10E0D00004DC012806D00C2814D103E0192801D053
:10E0E0001A280FD1DF4BA200995840318D79AD0627
:10E0F00008D5487DFD2420404875985880680CF06C
:10E1000098F970BD9030C2B20221204601F0C3FDE3
:10E1100070BDF7B504020546E61D30460CF0D7F990
:10E120003F2822D01F2820D01F2130460CF0A4F910
:10E13000CC4FAE00B95902988881284601F09EFE66
:10E14000C0B2019907F071FB00280DD09030C3B226
:10E1500001212846029A01F08DFDB859002803D10B
:10E16000E01D00210CF088F9FEBD43230121284663
:10E17000029A01F07FFDFEBDF8B50502ED1D0C46CB
:10E1800028460CF0A4F93F2831D020462030017AEF
:10E190002E0ACA0719D0827A304601F0E5FEB14F47
:10E1A000B5007959206948637959606A886378595C
:10E1B0001022AD4B21461430984778592146102241
:10E1C0001431A94B2430984704E000221146304610
:10E1D00001F0CAFE35020824681D0CF078F9A0434E
:10E1E0000146681D0CF048F9304605F042FBF8BDC9
:10E1F000FFB5150A16460F460A4681B0002128468B
:10E20000FFF72CFF0446012822D13978072922D0B4
:10E2100004DC032907D004291AD10BE0182928D0DF
:10E22000192915D142E0284601F028FEC0B207F0B6
:10E23000C0FB05E0284601F021FEC0B208F0A2F9BB
:10E24000002805D09030C2B20021284601F023FDFD
:10E25000204605B0F0BD01233246844804990CF0F5
:10E26000CFF80646284601F009FEC0B20BF03EFE8C
:10E2700027E0284601F002FEC0B2694609F0ECFC36
:10E2800007000ED1732002233246000104990CF0DE
:10E29000B7F86946497841706946097801700CF011
:10E2A000C8F8002F00D09037FAB2CDE76F480123AD
:10E2B0003246283004990CF0A3F80646284601F0AF
:10E2C00015FE307030460CF0B4F80022BCE770B593
:10E2D00015460C4610460CF0FAF82B0A00253F288C
:10E2E0000BD0E188062908D1000701D5022504E0FA
:10E2F0002278211D184603F015F9284670BD70B527
:10E30000154610460CF0E3F82C0A3F2812D0554869
:10E31000A1004058806800280CD00078092809D155
:10E3200045220221204601F0B6FC2A463B21204628
:10E33000FFF7EFFE002070BDFFB50546000281B07B
:10E34000C01D0CF0C4F83F2883D0464FAE00B8592A
:10E350008468002C15D02078092812D1284601F0B5
:10E360008DFDB959029A4031497DC0B2C943890730
:10E37000C917491C002A0FD0002903D0A11C09F09D
:10E3800039F866E761780022284603F025FDA11CD4
:10E390002846FFF790FE5CE7002903D0002109F032
:10E3A00029F804E061780122284603F015FD48228F
:10E3B0000221284601F06FFC4BE7FFB5160A17460D
:10E3C0000C460A4681B002213046FFF747FE05465B
:10E3D00001285ED12078092802D0172859D149E0B8
:10E3E0002389E2886188A08801F0EAFD002813D023
:10E3F0001C48B100415808464030427D920702D483
:10E40000807980061CD40498C0B2072806D0A11CCD
:10E410003046FFF750FE3CE0402236E01348C98901
:10E4200008233A46801D0BF0EBFF61880180A1882C
:10E430004180E18881802189C1800BF0FAFF28E0CA
:10E440000CF060F90106090E00D101216170A21CD7
:10E45000304603F0D8FC0548054A3946E9300CF04F
:10E460004FF816E0C0910020190F000009070000C6
:10E4700030750000304601F001FDC0B2611C09F0AA
:10E48000FEFB002805D09030C2B20221304601F0D8
:10E4900002FC2846DDE60000F7B5009816460502A6
:10E4A0000F460024681D0CF012F84322102811D0EA
:10E4B0000099BB008A00F8498958CA58B2421CD05A
:10E4C0000122BA40024201D0022408E0C88DC006F1
:10E4D00007D5432233463946009803F02FFA2046E9
:10E4E000FEBDCE500124D6B2681D0BF0F0FF3043C4
:10E4F0000146681D0BF0C0FFF1E70124EFE7FEB510
:10E50000100A0C460A4601210090FFF7C5FF029051
:10E5100001287AD12178204605260C30F602DF4DFD
:10E5200001900B000BF03AFD107109471A713A3A4D
:10E530005365685EA7D9BD71FE716088FF220146F0
:10E540001739EA32D64C914200D8A0830422022126
:10E55000009803F0E6FB0146A08B8AE06078022871
:10E5600015D0102206210832009803F0DAFBA188AA
:10E570004180E1888180C680627821460831074663
:10E58000042A06D038460830A8473946E1E002227E
:10E59000E8E73846083003F04EFEF6E70822114659
:10E5A000009803F0BEFB0146A0884880E088888080
:10E5B000BC4ACA80CDE008221021009803F0B1FBCC
:10E5C0000146A0884880E0888880CE80C1E006228D
:10E5D0000421009803F0A5FB0146A0884880E0884C
:10E5E0008880B6E00098AC49800008588068002810
:10E5F0000CD0E088002835D006220C21009803F0CA
:10E6000090FB0146E088888032E0C1E0A188E08884
:10E61000814201D94022B7E0207A102805D0042891
:10E6200003D0022801D05122AEE0022810D01022DF
:10E630000821921D009803F074FBA1884180E188B5
:10E640008180227A214609310646042A02D005E05B
:10E650000222EDE7B01D03F0EEFD01E0B01D76E013
:10E66000314676E004220A21009803F05AFB014665
:10E67000A08848806DE060780E214200921C0098CE
:10E6800003F04FFB0146002207E090000019530001
:10E690005B188088521C588092B260789042F4D8FF
:10E6A00057E026462489009803F0D5F9C01E84421D
:10E6B00000D2204687B2381D82B25221009803F062
:10E6C00030FB0446B08860803A46201D0199A84777
:10E6D000204608380BF0ADFE5AE06078002809D0DB
:10E6E000009803F0B8F92189C01E884202DBE08857
:10E6F000002820D06189208981422ED2461A0098B4
:10E7000003F0A9F9401F864200D2304687B2B81DF7
:10E7100082B21621009803F004FB0646A0887080A0
:10E72000E08800E036E061893A464018B0806189AF
:10E730000198091892E7091D8AB21221009803F086
:10E74000F0FA0646A08870802289301D0199A847FA
:10E7500086E7009805F0A5F91AE06278002A0ED045
:10E7600002221821009803F0DCFA01466089228910
:10E77000904201D1012000E000204870E9E7814289
:10E7800001D1002200E052220121009803F003F998
:10E790000298FEBD02221821009803F0C2FA014639
:10E7A0006078EAE710B51046140A0BF090FE1028C6
:10E7B00002D0204605F06CF9002010BD70B5150A96
:10E7C0000E460A4600212846FFF766FE0446012849
:10E7D00016D13148A9004058806A002806D04088E8
:10E7E000B188884202D1284604F08CF93146284687
:10E7F00004F01EFA020003D00021284603F0CBF8F3
:10E80000204670BDF8B515460C46002710460BF0A3
:10E810005EFE10286CD0280A1F4E850000907359A8
:10E820008446186A002801D0017D00E0002122788A
:10E83000402A04D0412A0ED0422A59D146E000296C
:10E8400056D0986A002802D00C380BF073FD70592E
:10E850000127846249E0122906D0182910D05229D4
:10E8600007D0D22923D104E062786188604604F0A1
:10E870003CFA705920300BF062FC0BF05BFD13E0AA
:10E880006378002B10D062881821604604F01EFACD
:10E89000009804F0FFF9ECE7E8910020190F000060
:10E8A0009891002003280000009804F0E2FF6078AF
:10E8B00000281DD17059806A002819D040886188CD
:10E8C000884215D1009804F01DF911E016290FD1E6
:10E8D0006378002B0ED06288604604F0F7F9705917
:10E8E00020300BF02CFC0BF025FD009804F0C1FF4C
:10E8F0003846F8BDA1880122D20311434182F4E7D2
:10E90000FFB581B0174610460BF0E1FD3D0A102817
:10E9100021D02A4EAC003059C08DC00606D42848FC
:10E920003A460059C18927480BF094FD305910220E
:10E93000C18D1143C185152101988901401A02D06A
:10E94000012808D102E04522012101E045220021F1
:10E95000284603F020F8002005B0F0BD70B515463C
:10E960000E4610460BF0B3FD0024102822D030785C
:10E970002D0A002804D0342812D03F2810D019E0E6
:10E980003146284604F09BFF0446FF2812D1314649
:10E99000284605F01FFD0446FF280BD1002409E09E
:10E9A000317A4A0606D43F2806D00423002228469E
:10E9B00004F08CF9204670BD0623F7E7E8910020AB
:10E9C000C09100201B050000F8B51F4614460D46F7
:10E9D00010460BF07CFD0026240A3F280DD0504A3B
:10E9E0002946A0000C3910580BF08CFB012631464B
:10E9F000204603F067F83046F8BD462239462046E7
:10EA000003F091F8F7E770B5464D6C8801F023FAF2
:10EA1000FF2808D06988491C698081004048405817
:10EA2000017B491E0173002C02D106200BF0F8FD7A
:10EA300070BDF0B587B014460E4610460BF047FD8A
:10EA40003F2840D0200A0590354980000C5800200E
:10EA50000490708869468881308833494018049052
:10EA60003779012F04D0022F2DD1059803F02FFB09
:10EA7000207C617C884205D203AA04A9059803F092
:10EA80004CFB0227A16800291DD08888274AD04264
:10EA900019D10D466846808904990C3500912346AA
:10EAA00001900E33AA1C0297291D059803F0C8FA9D
:10EAB000002802D1E189002905D10021A160287038
:10EAC00028460BF0B6FC30880BF08CFA002007B01B
:10EAD000F0BD70B514460D4610460BF0F8FC01462B
:10EAE000200A00243F2911D0EA88291D052A0DD1CA
:10EAF0002A78002A0CD0332A08D04979312A0BD041
:10EB0000002903D000231A4603F048F9204670BDBF
:10EB100003F097F90446F9E717230122F4E7000010
:10EB2000F8910020F491002000800020F9FBFFFF05
:10EB300070B505460C4606200BF0C9FC04280BD026
:10EB40000122AA40002C02D00243D1B201E090433E
:10EB5000014606200BF090FC70BD70B5524D064684
:10EB600084002859002807D00C380168491C03D1BB
:10EB70000BF0E0FB0020285100213046FFF7D8FFC2
:10EB800070BD70B5154604460622022310020BF034
:10EB900037FC047045700BF04CFC70BD70B5064638
:10EBA0000D46002406200BF092FC042812D03E4AA9
:10EBB000B1005358AB420CD00123B340034201D003
:10EBC000022407E00124555021463046FFF7B0FFEC
:10EBD00000E00124204670BD70B50A460546324962
:10EBE0008000095800290BD008460C380389DCB294
:10EBF000062C05D0072C03D008781946FFF7C1FF73
:10EC0000012D03D128480421203041712846FFF707
:10EC1000A4FF70BDF8B5244B05461E330C46981C66
:10EC200001792678C907C90F0322002E0BD18079FC
:10EC30001D4A800080188068467C828A002E02D09F
:10EC400003461633012100912946204601F07FF842
:10EC50000446FF2804D002F04DFF204602F04FFE8C
:10EC60002046F8BD10B50446FF280DD001F037F856
:10EC70000021204602F026FF0021204602F091FFED
:10EC80002046012102F0A6FE10BD0020074A0146E1
:10EC90008B00D358002B01D0401CC0B2491CC9B214
:10ECA0000329F5D37047000098910020C0910020FF
:10ECB000F8B50020009008781D460C46012807D0C2
:10ECC00003280BD040221946FFF75BFF0098F8BDE0
:10ECD0000DF028F9002229460120F5E70020FFF772
:10ECE0005DFF00900128F1D16078002507073F0FF4
:10ECF000FFF7CBFF002808D129484068002804D13D
:10ED0000032100F079F9002801D0432543E00020D9
:10ED1000002801D042253EE0608C1B38E12807D254
:10ED2000A08CFF214931884202D31E49884201D973
:10ED3000402530E0E17E1A4EC9073801490F0843EB
:10ED400020363071B8080DD0E08C01221721520214
:10ED5000904200D31046172800D2084610498883F5
:10ED600003F00AFD3079A17E8008800008433071ED
:10ED70000B480622211D0C4B1E309847201D05F024
:10ED8000E4FB20462030017A407A05F09BFBA18C01
:10ED9000608C05F0A8FB29460020FFF71DFF95E7D2
:10EDA0009891002048080000190F000070B50C462B
:10EDB00006200BF08CFB04281BD06148006800285B
:10EDC00017D00178192914D10C380189C3200025E6
:10EDD00010230622C0000BF013FB5A4B06461022EC
:10EDE0002146984730460BF024FB29460020FFF7C8
:10EDF000F3FE70BDF7B5044686B0154606200BF04D
:10EE000066FB04282BD04E4F3968002927D008789C
:10EE1000182824D1002C02D09034E1B21CE02846FE
:10EE2000484D01260C4600281BD00F460C39C12046
:10EE3000098908230622C0000BF0E2FA04460322E7
:10EE4000791CC01CA847032220460799A847A67131
:10EE500020460BF0EEFA00210020FFF7BDFE09B0BE
:10EE6000F0BD0322601C0799A847E078217980064D
:10EE7000800E0843334BE0701022002101A85C3360
:10EE800098470322611C01A8A847B8692E4B0122AC
:10EE900001A90096FEF7AAF9E1E770B50C46062035
:10EEA0000BF015FB04281AD025480068002816D05E
:10EEB00001781A2913D10C3801890025082306226C
:10EEC00022480BF09DFA1F4B064608222146984720
:10EED00030460BF0AEFA29460020FFF77DFE70BDEC
:10EEE00038B50C460020FFF759FE0546012821D110
:10EEF0002078182804D0192813D01A281AD11BE01A
:10EF00002079C02808D0002806D0402804D040210D
:10EF10000020FFF761FE0DE000210B48FEF797F996
:10EF200008E0002100912146094B01221131601CAB
:10EF3000FEF75CF9284638BD00210648EEE70000E0
:10EF400098910020190F0000F5ED00181A06000036
:10EF5000ADED00189BEE001830B504460120F84DC9
:10EF600000218A0052199268002A09D0537B022B93
:10EF700001D0012B04D1527CA24201D0002030BD2F
:10EF8000491CC9B20429ECD330BD10B5FFF77DFE92
:10EF9000EB4C002291000919896800290DD0CB7B28
:10EFA000032B0AD14B7B002B02D0022B03D004E0B1
:10EFB000097C890601D5401CC0B2521C042AE9DB39
:10EFC000032801D3012010BD002010BD70B50E46EE
:10EFD0000546002130460BF053F904000AD0D94B06
:10EFE00032460021984725730020E073D449A800D9
:10EFF00040188460204670BD30B50023D04C0AE034
:10F00000820012199268002A04D0D57B8D4201D16A
:10F01000134602E0401C0428F2DB184630BD0146CE
:10F020000120002904D1C64820300079C007C00F54
:10F03000704770B50D00044607D0007B00F074F9EE
:10F0400029460120FFF7C8FD70BDA18A03230622CF
:10F05000BD480BF0D5F9217B0170617B41700BF04D
:10F06000E8F9B74820300079C007C00F0ED0B44986
:10F0700020461630B34B06221E3106465C3B9847AD
:10F08000607B002805D0304605F03DFA0120E07392
:10F09000D6E7207B314605F082FAF7E770B50446E3
:10F0A0000D460120FFF798FD002D01D0012003E05F
:10F0B000E07B022801D10320E07370BD70B50D46DE
:10F0C0000446818AA04804230622401C0BF098F9CC
:10F0D000217B0170617B417085700BF0AAF9E07BA8
:10F0E000042819D1964900204968002900D00878E1
:10F0F000A52802D0A62805D00EE000210120FFF7A8
:10F100006BFD09E0207B0321401CC0B2FFF774FFB8
:10F110000028F2D0416888470120E07370BD10B527
:10F120008749044649680020002900D00878A728AC
:10F130000CD0A8280ED1207B0121401CC0B2FFF7C3
:10F140005BFF002802D08168884703E0002101208E
:10F15000FFF742FD207B00F0E7F810BDFFB581B05E
:10F160000D460120FFF71AFD009001287BD1297878
:10F1700000260846A43834460427714A03000AF0E2
:10F180000DFF050425313A4A5700687829460428BE
:10F1900061D2800080188768002F04D0F87B012896
:10F1A00003D0032804D0432456E00220F87305E07E
:10F1B000787B0028F7D1B87B0028F4D13A6838462C
:10F1C0009047040048D00120F87345E0687804288F
:10F1D00041D28000801880680028E4D0C17B0329D8
:10F1E000E1D105E003210020FFF706FF00281DD034
:10F1F000C77341680DE0687804282CD2800080181D
:10F200008068002812D0C17B0129CCD10521C173AF
:10F210008168884720E003210020FFF7EDFE0028E9
:10F22000C1D10121FFF7E8FE0028EFD1012613E04C
:10F2300004200024A3009B189B68002B16D0641C9C
:10F24000E4B2042CF6D3042812D0A02912D0A129AC
:10F2500016D0A2291AD040242046304303D021469C
:10F260000120FFF7B9FC009805B0F0BD2046EAE7A1
:10F270004B24F1E769782B1D049A00F0CEF803E0E7
:10F280006978049A00F088FA0446E5E76978049AF8
:10F2900000F0E5FBF8E710B502462B480C460123C9
:10F2A0000621401F0BF0ACF804700BF0C2F810BD43
:10F2B00010B5084600781946002800D09030204B41
:10F2C000C2B2586800281DD0007800281AD018460D
:10F2D000203040798000C0188068448A8C4211D167
:10F2E00000234382437B002B04D0012B05D0022B4B
:10F2F00008D105E000F0EFF804E000F077FA01E053
:10F3000000F015FC002010BD10B514460246FF2089
:10F31000002903D121461046FFF77CFC2178002903
:10F3200001D100F0C7FB10BD810010B504480C18D6
:10F33000A068002801D00AF0FDFF0020A06010BDE9
:10F3400098910020750F0000A40600001CB5027BF8
:10F350006B461A70002906D001225A704A885A80DA
:10F360000979197101E000215970E44C4482184672
:10F3700005F0E4F9014668464078084302D020468B
:10F38000FFF789FF1CBD70B5044601250878002AE7
:10F3900011D0A28B4B889A420DD1A92802D0AA285D
:10F3A00003D006E0207C042101E0207C08210843F2
:10F3B0002074002509E0A92801D0AA2805D12046FB
:10F3C00000F064F9A18B4018A083284670BD10B5E9
:10F3D0000024C477CA4A037B5371FFF7B7FF204666
:10F3E00010BD0021C177C649027B4A71017C4906E4
:10F3F00001D50021AAE7704710B50021C177C049A7
:10F40000BE4C027B4A71E41C4482007B05F0FFF98C
:10F4100001462046FFF73FFF10BDFFB50F46588855
:10F420001021084381B058801C4616460025202133
:10F430000198FFF7CBFD00282FD0002141732278DF
:10F44000827347748682C17761788177AD490160A4
:10F45000AD494160AD498160A94A01995171817BF3
:10F460000029A1781BD0890706D4017C0222114310
:10F470000174A178890703D5017C0122114301742D
:10F48000A178C90703D0017C2022114301742146D1
:10F4900000F0BCF8284605B0F0BD4B25FAE7490757
:10F4A000E3D5E6E770B50C460120FFF777FB05468C
:10F4B00001280ED160789249800020394018806878
:10F4C000002181838E4962784A7100222146FFF72C
:10F4D0005AFF284670BDF8B5C77B894D874C203D43
:10F4E000BF263B000AF05AFD0604101D1037420FDC
:10F4F000824BDB1C994200D0C277418A002902D19D
:10F50000C17FFFF796FDF8BD6968140004D10122A0
:10F51000FFF739FF0028F6D121460120FFF75CFBF9
:10F52000F8BDA14205D1C37F002B02D0017C314040
:10F5300009E0C277002A07D1704A5242D14203D172
:10F54000017C402211430174418A0029E8D1C17F26
:10F55000FFF7A4FDF8BDA14202D1017C3140017446
:10F56000418A0029F6D1FFF7A9FDF8BDFFF7D7FDC5
:10F57000F8BDF7B50E4662490546800020394018AF
:10F580008068002814D0C17B032911D1818AD5203D
:10F5900008230622C0000AF033FF05700446C67136
:10F5A00006225B4B02A9401C984720460AF041FF07
:10F5B000FEBD70B5524B8000203BC018846800250A
:10F5C000002C22D0607B00281FD1E07B03281CD1B7
:10F5D000207CBF2318402074002904D03C290FD080
:10F5E00043290ED10CE0607C00280AD0104600F0C0
:10F5F00032FCFF2805D02146163100F059FC00E00E
:10F60000452529462046FFF759FD70BDF8B50D4642
:10F610000646002120200AF033FE0446307B20708D
:10F62000A8784006400E6080286960606869A06024
:10F63000287E6070687E2077707CFFF7F0FC207376
:10F64000A878400707D5287B60730622A91D2046AD
:10F650002F4B0E3098476879A0762879E076688835
:10F66000C00501D5012000E00020244F6077FF1E77
:10F670007782204604F0BEFF050002D020460AF043
:10F6800059FE29463846FFF706FEF8BD7CB50A4606
:10F6900053880146FB2B01D8032007E0888B002804
:10F6A00006D0181A83B2FB2B04D80220DCB203E088
:10F6B000012000E00020FB240B7B6D462B7068705E
:10F6C000EC708B8B101D181801901078A9280ED0A3
:10F6D00001202A46A870094D6D1E4D82104604F087
:10F6E000CAFF01462846FFF7D6FD20467CBD002014
:10F6F0002A46A870014DAD1EEFE70000392000003A
:10F70000B8910020CFF30018E3F30018F9F30018C4
:10F71000190F00007CB50C46B1496B4649681C7056
:10F720000A795A70827B012300259B02891C012AD9
:10F7300012D0002A10D08A896B465A80C9899980D4
:10F74000A84D4582684605F02EF901460C4302D0CB
:10F750002846FFF7A0FD7CBD69464B808D80EFE712
:10F7600010B58A788273CA780024891C920603D463
:10F77000027C01231A430274994A037B203253719D
:10F78000037BD37100F0EDF8204610BD9449027B55
:10F7900020314A710021BDE770B5044690481646F5
:10F7A000203000790D46C00601D4432418E00846F5
:10F7B000FFF7D2FB002815D01C212046FFF706FCDE
:10F7C000002811D001214173457486828649016069
:10F7D000864941608649002481602146FFF729FC63
:10F7E000204670BD4024FBE74B24F9E770B57C4B05
:10F7F000C57B04242033022D06D0042D03D1DC71F7
:10F800000021FFF75BFC70BD002A04D0DC711146BB
:10F81000FFF744FC70BD734A521E914203D101218F
:10F82000FFF778FF70BD6F4A9142FBD10021EFE7EF
:10F83000F8B505466A482030C07904287AD068496E
:10F84000800040188768B87B042802D3687DC00711
:10F8500070D0687D00214006800F0091002802D002
:10F86000022803D005E00120009002E0387CC007A8
:10F8700060D06E7FB98A3346163306225D480AF09F
:10F88000BFFD0446002E0BD0A682298CAA7F2046FD
:10F890008918594B163089B2C918584B32469847C7
:10F8A000687D010747D5C00601D5032000E002208E
:10F8B0006070687DC00703D06078102108436070D5
:10F8C000687D800703D56078202108436070687DDB
:10F8D000400703D5607840210843607000980028F5
:10F8E00003D06078082108436070387B2070287F3F
:10F8F0006074E87E2074687E401CA074E87DFF2858
:10F900001CD0C007C00F20720622291D3B4BA01C33
:10F910009847687D40070AD5287E2946C007C00F52
:10F92000E07306220A312046344B093098472046BE
:10F930000AF07FFDF8BDC006C00FB9E7FF202072B6
:10F94000E7E7274910B52031C879042808D0244AB0
:10F950008000801880680422CA714521FFF7AEFB41
:10F9600010BDF8B50D460646002144200AF088FC7B
:10F97000044600274030C7708770707CFFF74FFB4C
:10F9800020706770B07B0121032801D0052800D1C9
:10F990006170707C012806D16878C00603D5607854
:10F9A000022210436070A7706878C00708D0A17069
:10F9B000A888E080E888208168784007C00F20711F
:10F9C000084F20467F1E778204F0B2FF050002D068
:10F9D00020460AF0AFFC29463846FFF75CFCF8BD2C
:10F9E000989100204220000061F700188DF7001860
:10F9F0001FF10018A706000000800020190F00006A
:10FA000070B504468878A0730026542006558A886D
:10FA10008D1C002A05D00A204243062176480AF0B0
:10FA20006FFD7648217B4171217B817129462046FB
:10FA300000F0A3F8304670BD70B5044606216E484C
:10FA40000AF0B1FD6D48217B41716D4D658205F075
:10FA5000EFF9010002D02846FFF71DFC70BDF8B594
:10FA6000074666480D460079002401090520164620
:10FA7000884301D0432417E02846FFF76DFA002899
:10FA800014D058213846FFF7A1FA002810D00221DF
:10FA90004173457486825B4901605B4941605B4903
:10FAA00081600021FFF7C5FA2046F8BD4024FBE73E
:10FAB0004B24F9E770B5514E0025B17932468900E3
:10FAC000203A89188C68FF280DD0617C002903D06A
:10FAD0002146163100F0ECF9A07B00280AD106215E
:10FAE00045480AF060FD0422012520460021B2713C
:10FAF000FFF7E4FA284670BD70B540488479042CBD
:10FB000013D03E49A00020394018856806223520D0
:10FB10000223114640010AF073FCA52101704470D4
:10FB20000AF087FC452040352875002070BDF8B5E7
:10FB30000746C17B04263048304C022907D00329F0
:10FB400010D004290DD154213846C95D11E01500AB
:10FB500003D006210AF027FDA67129463846FFF793
:10FB60009DFAF8BD1500FCD006210AF01CFD3846B0
:10FB70002946A671FFF7A2FAF8BDF8B50D4606466C
:10FB800000211E200AF07CFB0446707CFFF747FA38
:10FB90006070002020703620405D2946A07006224B
:10FBA00030311B4BE01C98476878C007C00F60726B
:10FBB0006878C0070FD0A8886081E888A081A889EC
:10FBC000E081E8892082A88AE082E88A2083288A66
:10FBD0006082688AA0820A4F20463537778205F016
:10FBE000A5F8050002D020460AF0A4FB29463846B5
:10FBF000FFF751FBF8BD0000F2060000B8910020AD
:10FC00000E20000001FA001839FA00181FF1001840
:10FC1000190F000070B50C460546012901D101F00D
:10FC2000A6FCF24EAD007059A4000059002808D07F
:10FC30000C380168491C01D10AF07CFB7159002085
:10FC4000085170BD70B50502ED1D16460C462846DC
:10FC50000AF03DFC1F280CD028460AF038FC002E84
:10FC600002D00146214301E0A043014628460AF0A4
:10FC700003FC70BD70B5164602021C460D460720F7
:10FC8000022331460002D21D0AF0BAFB057044700F
:10FC90000AF0CFFB70BD70B50D460646D349800013
:10FCA00008581346A9004258002A0CD010460C38B8
:10FCB0000489E0B2052806D0062804D0117822462F
:10FCC0003046FFF7D7FF29463046FFF7A3FF012054
:10FCD000A840C1B200223046FFF7B4FF70BDF1B5B5
:10FCE00000988600C148815900980502002920D05B
:10FCF000E81D0AF0ECFB074600241F2F04D0214624
:10FD00000098FFF787FF0AE0B848A10080594058E3
:10FD1000002804D0462221460098FFF7BCFF641C4F
:10FD2000E4B2032CE9D3B14CA0590AF003FB002044
:10FD3000A051E81D3F210AF09FFBE91DAC480AF0E5
:10FD400032FCAB48E91D801C0AF02DFCF8BDFFB564
:10FD500081B0054600242002C01D0AF0B8FB3F28F0
:10FD600003D0641CE4B2032CF5D3032C71D0002122
:10FD700058200AF085FAA6009C4F58229D4BB85196
:10FD800000219847B859C8218187B9590F204031BF
:10FD90004875200200900021C01D0AF06DFBB95982
:10FDA000029840318880B859E97B40308175B85954
:10FDB000DF21403082790A402978002900D00121D2
:10FDC00049010A4382718B4BB8590622A91C5C3B3E
:10FDD0004E309847B859697840300175854BB8590D
:10FDE00006225C3B473004999847B9590A9840313C
:10FDF0004873B959FF208881B9590398C88103987D
:10FE0000062822D001467A48009A1223F138D21DE2
:10FE10000AF0F6FA0646029830806878754BC007FB
:10FE2000C00F707230460622A91C0A305C3B98470E
:10FE3000288970806889B080A889F080A87B30729A
:10FE40002878307430460AF0F4FA204605B0F0BD48
:10FE5000FFE7FF24F9E70346644A00208100515878
:10FE6000002903D040318988994203D0401CC0B298
:10FE70000328F3D3032800D1FF20704701465E48D2
:10FE8000032906D28A0059498958002901D04031F6
:10FE90008888704701460020FF2908D08A0053490E
:10FEA0008958002903D0403188798006C00F7047F7
:10FEB00070B54E4D84004F4B285906225C3B4730AD
:10FEC0009847285901214030417370BD02460020F7
:10FED000FF2A0AD0022908D29300444AD258002AA5
:10FEE00003D0C800401A47301018704701468A00F6
:10FEF0003E4900208958002901D04031887D704753
:10FF0000024600209200394B002909D001290CD06B
:10FF1000022904D1985840308079C006C00F70473C
:10FF20009858403080794007F8E7985840308079F9
:10FF30000007F3E701460020032908D28A002B4975
:10FF40008958002903D0403188798007800F704795
:10FF500001460020FF2906D08A002449895800293B
:10FF600001D02031887F7047F0B5032827D21F4F7A
:10FF70008300FC58002C22D04034A579FB26354064
:10FF8000CE07760F3543A571FC58EF263540120198
:10FF9000154340340020A5710A0701D5032008E06D
:10FFA0004A0701D5022004E0C90701D1290700D57D
:10FFB0000120AA08F9589200024340318A7146E7AD
:10FFC00010B51924E401401EA0420AD2491EA142E4
:10FFD00007D20A480A3B834203D2FF20F430824210
:10FFE00001D9002010BD012010BD0000C0910020EB
:10FFF000F2070000750F0000FFFF0000770C000003
:020000041801E1
:10000000F7B582B016460546FFF725FF04020090BB
:10001000E01D0AF05CFA3F2823D000988700C24810
:10002000C0598189FF2900D1C189E21D0423BF483D
:100030000AF0E6F9058086700AF0FBF9BA48C05963
:100040008289FF2A08D00398002800D09030C3B2DC
:1000500001210098FFF70EFE324629460098FEF770
:1000600001FE05B0F0BDF8B516460D46FFF7F3FEEC
:1000700007460402E01D0AF02AFA3F2812D0B80011
:10008000A949009008580068002806D00278032A81
:1000900003D1002D07D09035EDB22A460021384615
:1000A000FFF7F9FDF8BD0C380189A048E21D0623D1
:1000B000001D0AF0A5F9044630782071B0886080F0
:1000C0007088208020460AF0B4F920790628E4D808
:1000D00095490098FD2208584030417D11404175F6
:1000E000DBE7F7B50C46FFF7B6FE06460502E81D4E
:1000F0000AF0EDF93F283DD08B4AB700D159086886
:10010000002832D00378042B2FD1002C0DD090344E
:1001100040318879E4B2800627D5A12C21D01CDC9F
:10012000912C1ED09C2C20D11BE00C380189E120A1
:10013000EA1D0823C0000AF063F9054602987C4BCB
:1001400001787948C0594030417508222846029903
:10015000984728460AF06DF907E0A92C01D0AA2C8F
:1001600003D1487DFD2210404875224600213046CB
:10017000FFF791FDFEBDF8B50C460546FFF76BFE97
:1001800006460702F81D0AF0A2F93F280DD066497D
:10019000B0000858FA1DC18964480423401E0AF0C3
:1001A0002FF9058084700AF044F9F8BDFFB581B0DD
:1001B0000F46FFF750FE05460602F01D0AF087F9CC
:1001C0003F281FD03C469034574A3946112F0BD058
:1001D00006DC00291DD0012906D00C2F2AD103E00E
:1001E000192901D01A2F25D1A90050584030837900
:1001F0009B061FD5437DFD242340437550588068DE
:100200000AF017F92DE7E2B202212846FFF743FD75
:1002100027E7A8001058F21DC189444806230E3074
:100220000AF0EEF803990180049941800A998180CF
:100230000AF0FFF8002FE6D10024E4E7FFB581B013
:1002400015460E46FFF707FE04460702F81D0AF0A2
:100250003EF93F2818D03548FA1DF91D0E230B3002
:100260000AF0CEF83049A2008958022340314A7D75
:100270001A434A7509210170858046800499C1801E
:100280000A9901810AF0D5F8EBE6FFB581B01C466A
:100290001546FFF7E0FD06460702F81D0AF017F9BC
:1002A0003F2811D02049B0000858FA1DC1891F48C5
:1002B000082329300AF0A4F80A998180C4800580B7
:1002C000029941800AF0B5F8CBE6FFB581B00D4642
:1002D000FFF7C1FD04460702F81D0AF0F8F83F28B1
:1002E00021D0114E002D0ED1A0003058FA1DC18929
:1002F0007320022300010AF083F8049941700399E6
:1003000001700AF096F8A0003058806800280AD0E2
:100310000078172807D1002D00D09035EAB20221CD
:100320002046FFF7B8FC9CE6C091002003070000C0
:10033000190F0000F8B51E460546F84B1746800019
:1003400018580024069A012903D11A214030144676
:100350000170012208212846FFF774FC2846FFF7A8
:100360008DFDC0B223463246394605F070FF0028A5
:1003700005D09030C2B201212846FFF78CFCF8BDB1
:1003800070B516460C460546FFF778FDC0B2002C46
:1003900008D0314605F0B0FF012208212846FFF7BA
:1003A00051FC70BD002105F0A7FF962201212846CF
:1003B000FFF771FCD94AA8001058002140300170A5
:1003C00070BDF3B581B001980F468100D348212359
:1003D00046580198F18902023569D148D21D0AF0C8
:1003E0000FF80446077002213B0009F0D7FD08050D
:1003F0003737371437100C37A87CC006C00E607032
:10040000403631702AE00198FFF7A2FD16E0132074
:100410004036307022E0687C012802D1287E012815
:100420000BD04036B079012280060028E87D0BDB36
:10043000022805D0042803D00FE0002060700DE0F2
:10044000287C02280ED108E000280BD0012809D012
:10045000042802D1287C022804D06170204609F0CB
:10046000E8FFFEBD6270F9E7F7B50F46064681006A
:10047000AA4832024558AA48E9891E23801CD21D89
:1004800009F0BEFF04460770B81EA64F030009F02E
:1004900085FD0608042E1E231C2E02980078A070ED
:1004A0000DE028694030C17BA170427CD207D20F99
:1004B000E270407CC207D20F3046FFF755FD403551
:1004C000A879BF210840A87111E01C2200E0172282
:1004D000A01C0299B8470AE01022A01C0299B84754
:1004E0001022284624300299B8470020A8632046ED
:1004F00009F09FFFFEBDF8B5884A81005558884F26
:100500002E462036F17F04028907E137002903DAFD
:10051000E11D38460AF047F8AA8F0A204243E11D40
:10052000384609F0EDFFF07F02210843F077F8BD6F
:1005300070B50546794B800019583F22525C002463
:1005400092071CD58A8F784CA24214D05204120C08
:100550008A87A2420DD38C8718582A02C189704815
:100560001E23801CD21D09F04BFF0821017009F0E9
:1005700060FF032400E001242846FFF7BCFF20466B
:1005800070BDF0B50446654BA2009A58012012696F
:10059000137DD57E2B409E46537D157F2B409C4678
:1005A000937CA500DE075D4B5B591B69DF7E1D7DDB
:1005B0003D401F7F5B7D3B401D43002E05D0537E99
:1005C000DB0702D0002D00D10020544BA4001B59A2
:1005D000ED071B6940335C7C002D07D001252C43BF
:1005E0005C74012905D0022903D007E06408640087
:1005F000F6E74032527CD20700D10020032901D017
:10060000042906D17146490703D46146490700D43D
:100610000020F0BD7FB50646404980000C58684672
:10062000007A1D4600281BD002AA03213046FFF79E
:100630001BFF002D02D03046FFF75DFF0022012195
:100640003046FFF728FB20690025002802D009F07A
:1006500071FE2561304601F0E9F8403425707FBD18
:10066000002202213046FFF7FFFEE7E770B52B4B73
:1006700082009A581469403215782E46143E330091
:1006800009F08CFC060C04090609090C162000E090
:100690001820107070BD1423137001E0142DF9D1CF
:1006A0004034237CDD0705D015201070207C4008E5
:1006B000400006E09D0706D517201070207CFD2124
:1006C00007E0207470BD5B0705D519201070207CF1
:1006D000FB210840F5E7002904D000231A46FFF764
:1006E00099FF70BD002100F0B7F870BD30B40B4B1E
:1006F00082009C5885005B5922691B6940330029A0
:1007000008D0157DD27E154014221D74403422700D
:1007100030BCABE7557D127FF5E70000C0910020AB
:1007200013070000190F0000B80B0000F8B50E46C3
:10073000FE4A8100545805022034E17FFC4FC9076E
:10074000002907D0E91D384609F02DFFE07F400859
:100750004000E0773046083809F06BFE30780B280F
:100760000AD0052808D0E91DF24A384609F0C8FE2B
:10077000E07F01210843E077F8BDF3B50646EB4979
:1007800080000D5881B02C6940352878102807D09A
:10079000112803D0122801D013280FD1102028705F
:1007A0004034207CC1070AD0C0B240084000207409
:1007B00007213046FFF705FE11202870FEBD810796
:1007C0002CD5FD2108402074DB48112287690821BF
:1007D000304601F094FA0090002F04D01022D74B3D
:1007E0003946401C984730460099FFF79FFF082282
:1007F0000921304601F083FA0746CF48CE49203020
:1008000000791E31C007C00F78700622CB4BB81C90
:10081000984739463046FFF789FF0AE041070CD573
:10082000FB21084020741320287006213046FFF772
:10083000C8FD28781028B4D0FEBD0298002804D046
:1008400001463046FFF752FFFEBD002301461A461F
:100850003046FFF7DFFEFEBD30B4B44B82009C583B
:1008600085005B5922691B694033002908D0557DFA
:10087000127F154010221D744034227030BC7CE77A
:10088000157DD27EF5E710B58100A84AA74B5158D7
:1008900080001858096900694A7C00244030012A08
:1008A00002D10A7E012A07D08A7C520706D44A7EEA
:1008B000520703D484730FE002220CE0CB7D0A7C44
:1008C000032B05D0032A03D0012B03D8012A01D81A
:1008D000002200E00122827308464030827B002A19
:1008E00006D0012A01D0022A03D10422C27300E0FB
:1008F000C4738A7CD20706D0497EC90703D0C17B66
:1009000001221143C17310BD00B5884A8000105800
:100910000029006907D0417F0B0009F03FFB060664
:10092000060806080C11817DF6E7012000BD403065
:10093000C07B400702E04030C07B0007C00F00BD15
:10094000002000BDF7B500981646850077480024C2
:100950004759224608210098FFF774F9062E0AD05D
:10096000112E0AD0222E0AD0002E0AD0903634063C
:10097000240E06D00BE0222409E0232407E02424DF
:1009800005E03846403081790822114381713E46A6
:100990004036009930780A020E2830D00F282ED029
:1009A0001A282BD1002C22D1604F01237859D21D57
:1009B000C1895F48DA3809F023FD009A0021032A33
:1009C00012D27A59002A0FD040329279530700D5BB
:1009D00001219207920F022A02D0032A04D101E0DA
:1009E000042200E00C221143017009F022FD0020D6
:1009F0003070224601210098FFF74DF9FEBD002C12
:100A000006D00023224601990098FFF703FEFEBDA1
:100A10000F2823D13869817CC9071FD0407EC007C9
:100A20001CD042481E234059D21DC1894048DE389F
:100A300009F0E6FC0446072020701C223F4BA01C56
:100A40003969984720463D4B0822002114305C3319
:100A5000984700206082204609F0EBFC01980028AE
:100A600004D001210098FFF7F7FEFEBD0021009899
:100A7000FFF73CFEFEBDF0B505462C4A800010583D
:100A800085B02E4F046903AE002918D008222146F4
:100A900001A82E31B847082221461E313046B847FA
:100AA000FF20000285430320000228180090244BF9
:100AB000012201A92046FCF799FB05B0F0BD0822F0
:100AC000214601A81E31B847082221462E31E5E70C
:100AD000F7B505468100154816464058174F8AB0AD
:100AE00010220021046902A85C37B84710220021B7
:100AF00006A8B8470B98114F002844D0012128467A
:100B0000FFF7E4F980796946087200212846FFF76B
:100B1000DDF980796946487200212846FFF7D6F949
:100B20000146062206A8B84701210BE0C09100202B
:100B3000F30700003075000098910020190F0000A5
:100B4000DF0B01182846FFF7C1F90146062207A866
:100B50000230B847012269468A7202A80330062291
:100B600021461031B84702206946487404A8023073
:100B7000062221461731B847FF2000028543002E88
:100B800019D0012018E000212846FFF79FF980794D
:100B90006946087201212846FFF798F9807969466D
:100BA000487201212846FFF791F90146062206A85E
:100BB000B8470021B9E7022000020543FE4801952D
:100BC0000090002E02D021461E3101E021462E3138
:100BD00006AB02AA2046FCF776FC0DB0F0BDF7B5D7
:100BE0000346D7B2F548B900405886B0002833D044
:100BF0004168002930D009780A292DD104464034B3
:100C0000A1798D06ED0F002B03D09033DAB20023CB
:100C10005CE00669100A0006000E1FD001282CD0E7
:100C2000022844D0032817D13846FFF791F904462B
:100C30000246E34B01A8079998471020021B01A820
:100C4000DF4B001900215C339847002D55D001AAD5
:100C500001213846FFF794FB09B0F0BD1022304661
:100C6000D74B1E3007999847A0794006F4D401224B
:100C700029463846FFF72CFFEEE74806ECD40798E4
:100C8000009011220321384601F039F8064610225F
:100C9000CB4B401C0099984731463846FFF746FD3C
:100CA000002D02D008202070D6E70720FBE7304651
:100CB000C34B10223E308A330799984700280AD048
:100CC0000421384600F0C5FD012364222946384638
:100CD000FFF7A0FCC0E7A0794006BDD40E2020702D
:100CE000002D05D031461E31384600F0BFFDB3E778
:100CF00000213846FFF7BFFEAEE70020034601465D
:100D0000009001AA3846FFF715FBA5E7F8B50D4698
:100D10000746AA4980000E584620805D00248006C0
:100D20004FD5687804280FD8E878410707D04007E6
:100D3000400F012803D0042801D0052804D1A87849
:100D4000002803D0012801D00A243AE02879C01FE6
:100D50000A2801D3062434E03846FFF7E9FB0028CF
:100D600002D003282DD12BE03069002829D19548E5
:100D700000790107890F0ED0E97809070DD44007E3
:100D80000BD463206946087003246A46214638461E
:100D9000FFF76AFB15E0052413E03902CA1D08239A
:100DA0008948C91D09F02CFB06460A20307006222E
:100DB000691C834B701C9847304609F03AFB00E0F1
:100DC00009242046F8BDF3B581B00F4601987B4950
:100DD00080000E5878780024042859D8F878410704
:100DE00007D04007400F012803D0042801D0052870
:100DF0004ED1B878002801D0012849D13879C01FD8
:100E00000A2847D235464035A879800650D428783C
:100E100001284DD1781C00F0E5FC002838D030695D
:100E20000622791C664B173098473069417E0907C6
:100E300006D5807C000703D5A87940210843A87116
:100E4000A879400603D45F480079400726D5019869
:100E500000F0DBFC00281DD03069817D0198FFF790
:100E600090FB002818D00198FFF70DFD0021019894
:100E7000FFF74AFD002811D0052028703069403066
:100E8000817B00290CD004210198FFF79AFA0FE02A
:100E90000A240DE006240BE0082409E0032407E0FF
:100EA000417C0422114341740021019800F0F1FCBF
:100EB0002046FEBDF8B50746404A80001458206918
:100EC000002819D025464035AA793D4B9206D60F09
:100ED00010223E30491C9847287807280CD1002E54
:100EE0000CD00520287020694030407C400703D595
:100EF0000021384600F0CDFC0020F8BD21693846BD
:100F00001E3100F0B3FC08202870F5E770B50646E6
:100F10002A4A800014582069002815D04034A2794C
:100F2000274B9206D50F10222E30491C9847207867
:100F3000082809D106202070A079400604D4002298
:100F400029463046FFF7C4FD002070BD08B54A7839
:100F5000511E0E2900D3082270210A4369460A70E7
:100F600016498300C9580B69002B07D04031897995
:100F700000238906C90FFFF74DFB03E06A460321F2
:100F8000FFF772FA002008BD70B504460B4A8000D6
:100F900012581346403318781D4615280AD1106997
:100FA0001022074B491C9847A8798006C10F20469C
:100FB000FFF75CFB002070BDDF0B0118C091002023
:100FC000190F0000B891002012070000F0B5054687
:100FD000FF4A8000145887B02646403630781628DD
:100FE0001ED188784A78000210436A46108204A80D
:100FF0000822F84F0230C91CB84710226846216900
:10100000B8472846FEF7A4FF6A469076072128468F
:10101000FFF72AFAB0798006C10F2846FFF726FBB2
:10102000002007B0F0BD70B50446E94A80001258B0
:101030001346403318781D4617280AD1106910222C
:10104000E44B491C9847A8798006C10F2046FFF75A
:101050000DFB0020AFE7F0B50D460646DC498000E9
:101060000C5887B0274640373878182817D1062201
:10107000D84BA91C04A89847687869468875D54B51
:1010800010226846216998476A4605213046FFF7D5
:10109000EBF9B8798006C10F3046FFF7E7FA002078
:1010A000BFE770B50546CA4A80001458403420781E
:1010B00019280AD14A1C06212846FFF7D5F9A0793C
:1010C0008006C10F2846FFF7D1FA002073E7F8B574
:1010D00006468700BE480D46C05900904878002457
:1010E000410709D04007400F012805D0042803D04C
:1010F000052801D00A242DE03046FEF7CBFE00285B
:1011000028D13046FFF714FA002823D16878000769
:101110000DD4B1480079400709D4632069460870AE
:1011200003246A4621463046FFF79EF912E00098F4
:10113000006900280ED1A6483202C0590123C18996
:10114000A648D21D09F05CF96978C906C90E01707C
:1011500009F06FF92046F8BDF3B581B00F4601984C
:101160009B4980000E583F20805D0025410701D536
:10117000452549E0800701D5692545E0384600F05E
:1011800031FB002803D0F878C01F0A2801D36A2554
:101190003AE0B878010790480029007901DA0007A1
:1011A00000E04007002801DB63252DE001215220EB
:1011B00009F066F8874B5222002104465C33306107
:1011C000984707222046834B394610309847A07C29
:1011D000C00701D12075607507220121019800F038
:1011E0008EFD0146207C4870607C8870A07CC870B1
:1011F000E07C0871207D4871607D88710198FFF75F
:1012000095FA0120403630702846FEBDF7B5944669
:101210000A4600986E4980000C580025002C35D0F5
:1012200026464036B0798006C70F206900281DD0B9
:101230004030417C4B0729D4042319434174206971
:10124000002A0DD0634B102261469847002F02D030
:10125000307805281AD10021009800F01AFB15E01B
:101260004030807B012811D1012500E0082530782D
:1012700000280BD02946009800F0EBFA2A4660209F
:101280000243012339460098FFF7C4F92846FEBD02
:10129000F3B581B00C4601984D49800008580026EE
:1012A000002838D040300178112934D18079800667
:1012B000C00F00900198FEF74BFE002102E0215480
:1012C000401CC0B21028FAD311220621019800F068
:1012D00016FD054610223F4F2146401CB8472946BF
:1012E0000198FFF723FA0B220721019800F007FD70
:1012F0000546401C218A0170090A417021460822D6
:101300001231E81CB84729460198FFF70FFA0099F7
:101310000198FFF732FA3046FEBDF3B506462C4978
:1013200080000C58002581B0002C22D0204640308F
:10133000017813291DD1807910228006C70F20461D
:10134000244B1430029998470020606311220A212F
:10135000304600F0D4FC044610221E4B401C02997B
:10136000984721463046FFF7E1F939463046FFF706
:1013700004FA2846FEBDF3B583B0039814498000F3
:1013800008580025009000286AD006464036B079FB
:101390008006C00F01900098046901982746173411
:1013A000103700285CD03078022859D104980028E2
:1013B00027D00146074B0722204698470648017967
:1013C000090703D4A178F7221140A170A17807E0A2
:1013D000C0910020190F0000B89100201B070000E9
:1013E000090706D5B978090703D5B1794022114319
:1013F000B171B1794A0606D40079400703D40325B8
:101400001FE0082520E004984078002806D178786D
:10141000012803D1480601D4022512E0039800F008
:10142000F4F9002807D0049881790398FFF7A9F808
:10143000002802D017E0062503E0B079400612D458
:101440000825307800280BD02946039800F001FACF
:101450002A4660200243012301990398FFF7DAF836
:10146000284605B0F0BD0398FFF70DFA0121039857
:10147000FFF74AFA0028C2D0A07841072DD04007D4
:10148000400F042829D020793979084020716079EB
:1014900079790840607107220221039800F02FFC3F
:1014A00001462078487060788870A078C870E0782D
:1014B000087120794871607988710398FFF736F9CF
:1014C00007203070009800694030817B002907D0E8
:1014D00004210398FEF775FFC2E700202071D9E7C9
:1014E000417C042211434174BAE770B50E46EE4BBD
:1014F00081005C580025002C12D0214640318B79A8
:101500009B060DD5002A07D01A230B700121FEF788
:1015100037FF2034A67703E000221146FEF730FFA4
:10152000284648E570B50D460646002A1ED12879A2
:10153000DE49800040188038C26F291D3046904730
:10154000040013D00146304600F083F928790128C1
:101550000CD00B280AD03046FEF79CFC01466020D8
:101560002246024301233046FFF754F823E570B5C5
:101570000646CD4980000C5800252069002802D07D
:1015800008F0D8FE2561304600F050F9403425704F
:1015900011E5FEB5140A16460D460A461F460121FE
:1015A0002046FCF75BFD019001282AD1A000BE492E
:1015B000029008584621095C2A788906C90F0A2A30
:1015C00004D00B2A26D00C2A7CD150E0002919D057
:1015D000BE421DD126460446012152206D1C08F052
:1015E0004FFE5222B24B002120619847B04B206938
:1015F00006225C3B29461030984700213046FEF712
:10160000E0FE5FE0691C2046FFF7A6FD024653E0BE
:10161000422253E02A461435002918D0BE42F7D1A1
:101620002146941CC0890A0201460A23A148D21D02
:1016300008F0E6FE0646208A30809D4B0822B01C4A
:1016400029465C3B9847304608F0F3FE3AE0518A61
:10165000961C009120462B4632460121FEF76AFE79
:1016600091490298B27E0858203082772AE00029FA
:10167000CED020306E78C07F0025410701D54525AA
:1016800019E0800701D5692515E08B4831070079FD
:10169000002901DA000700E04007002801DB63258C
:1016A00009E002220B21204600F029FB014646708A
:1016B0002046FFF73BF82A46002A03D001212046A6
:1016C000FEF7E9FA0198FEBD70B5054616460C46D0
:1016D000084608F0FCFE3F281DD0240A002E1AD030
:1016E0007148A10040584068002814D000780A28AA
:1016F00011D12E2D10D008210D46204600F0A9F85A
:101700002046FEF7C7FB60212A460A430146012313
:101710002046FEF77FFF4EE40B21EDE770B505464E
:101720001446104608F0D3FE3F281FD0240A5E4915
:10173000A00008585F49DC318D4210D14621095C78
:101740002030C27F0423520852001A43C277890610
:10175000C90F002345222046FEF75CFF06E0C821A2
:1017600081872030C17FFD221140C177002022E413
:1017700070B516460D46FEF76EFBFF281ED04A498F
:10178000820089584968002902D009780A2916D0B0
:1017900001024848CA1D1E23401FC91D08F030FE23
:1017A00004460B2020702046414B082214306582ED
:1017B00031465C3B9847204608F03BFE4AE4012155
:1017C000FFF759F946E470B50D46FEF744FB0446B1
:1017D000FF2806D0FEF75EFB01462A462046FFF7AB
:1017E000B1F837E401460A780120042A01D9002023
:1017F00070474A78002A01D0012AF8D10A79102AC4
:10180000F5D849791029F2D870470146264A89004F
:10181000525800201369D97C9B7E994200D3194607
:10182000072902D3012020329177704710B51E4A54
:10183000810054582034E17FC90709D001021D48B6
:10184000C91DDC3008F0AFFEE07F40084000E077C3
:1018500010BD70B50C4605460222052100F04FFA76
:10186000014644702846FEF761FF2FE470B50E462E
:1018700005461122042100F042FA04460C4B1022C6
:10188000401C31465C3B984721462846FEF74EFFF8
:101890001CE4FF2212029043090210B501430748DD
:1018A000FBF7D5FC10BD0000C091002014C5011845
:1018B000750F000017070000B8910020DF0B01181A
:1018C00070B584007B4E0D46012909D130598168DD
:1018D0000830002904D008F032FC08F02BFDF5E7B1
:1018E0003059AD004059002808D00C380168491C17
:1018F00001D108F01FFD31590020485170BD70B56D
:1019000004460021302008F0BBFC30226A4B05461B
:10191000002198471720A885A000664924020D5091
:10192000601D002108F0A8FD0825601D08F0CFFD0E
:1019300001462943601D08F09FFD70BDF8B51C46A7
:101940001546074600290BD1A08801F08BF8060048
:1019500006D06570A288234603213846B047F8BDFB
:101960000A2D06D16088010403D500254004400CEF
:10197000608020460C3801893A02052004230002C9
:10198000521D08F03DFD457021780170618841804D
:1019900008F04FFDF8BD70B50D460446454980007E
:1019A0000858A9004358002B03D029462046FFF7CA
:1019B000C5FF29462046FFF783FF0120A840C5B296
:1019C0002402601D08F083FDA8430146601D08F055
:1019D00053FD70BDF8B50646850036480F464059A0
:1019E000002829D00024002F05D046222146304669
:1019F000FFF7D1FF03E021463046FFF761FF641C8B
:101A0000E4B2022CEFD3304601F044F9294C60597E
:101A1000016A2030002904D008F091FB08F08AFC0C
:101A2000F5E7304601F044F9304601F06BF86059B3
:101A300008F080FC0020605134021520611D8001F7
:101A400008F0B1FD611D1D4808F0ADFD601D1021BD
:101A500008F012FDF8BD174980000858808D7047C6
:101A600070B5012217235202914200D31146172963
:101A700000D219460F4D84002A590423918510493C
:101A8000020209590D48C9893F38521D08F0B8FCB7
:101A90002959898D018029594968002902D00A787D
:101AA000012A04D00021418008F0C3FC70BD4988A0
:101AB000F9E70000E8910020750F000041050000E3
:101AC000C091002070B50124094D84402888002968
:101AD0000BD0204205D16888002802D0062008F0EB
:101AE0009FFD28882043288070BDA043FBE70000AD
:101AF000F491002010B5044600020021001D08F0FA
:101B0000BBFC0021242008F0BBFB002807D00021EB
:101B10000160416081600173017404214174994A3C
:101B2000A100505010BDF8B50646C8B2B400174623
:101B3000052814D0072811D1084608F0C8FC3F2812
:101B40000CD0914800594068002807D000780C2834
:101B500004D1002201213046FEF79DF8F8BD084669
:101B600008F0B5FC1028F9D0884D285900680028E5
:101B700007D00078122804D13A4600213046FFF7FA
:101B80000AFF295900204968002900D008780D284B
:101B900001D00E28E2D13A4601213046FFF7FBFE84
:101BA000F8BDF3B507468600764881B08459002C0D
:101BB00027D0A068002801D008F0BCFB7449207B26
:101BC0004A88101848800BE0A9887248814204D1E5
:101BD000298946223846FFF7A6FF284608F0AAFBC7
:101BE0002068002807D0204608F0A9FA0546029888
:101BF0000028F2D1E8E7634CA05908F09BFB0020D5
:101C0000A05138023F21001D08F036FCFEBDF3B59F
:101C100085B005985B4980000E58002E5FD034686F
:101C2000002C04D00698002801D0012000E00020FC
:101C3000039049E0002069468880012708F0E3F915
:101C400005468088544943185249A0884942C842F1
:101C500025D121460C31081D0290E089002800D0D2
:101C600000E0002701AA0097891C029800F09CF967
:101C70000090002803D10298008800280FD1218904
:101C8000009A0598FFF74FFF304608F058FA2046B3
:101C900008F050FB00200390009800280DD1694601
:101CA000898838030843E8800598FEF7E7F8C0B252
:101CB000294607F078FF002813D0A88808F0B8F963
:101CC0000698002802D003980028B3D13068002875
:101CD00013D00021012041400598FFF7F3FE07B023
:101CE000F0BD2B494888401E4880307B401C307333
:101CF0000698401EC0B20690E3E70121EAE770B5FE
:101D00000D46114608318BB201021446CA1D214806
:101D1000091D08F075FB0621C1808480057208301A
:101D200070BD70B50D46114609318BB201021446E3
:101D30004A1D1848091D08F063FB0421C1808480F6
:101D40000572083070BDF8B5069D1E4614460F4654
:101D5000042A13D0062C13D004212A460A3200028A
:101D600093B2021D01430B48401C08F049FB077069
:101D700000214180C48085800672F8BD0521ECE712
:101D80000721EAE7F8910020C0910020E8910020A7
:101D9000F49100200604000000800020F8B50F46F2
:101DA000540021461E460E318BB2010215460A1D13
:101DB0007A48091DA41C08F023FB0521C180211DC0
:101DC000818001210172477244818581002D00D0FC
:101DD000C68108F02EFBF8BD70B50D460102144611
:101DE000CA1D0E236D48091D08F00AFB0521C1809C
:101DF0000621818013210172457202214181848173
:101E000008F017FB70BD70B50D4601021446CA1DDF
:101E100014236248091D08F0F3FA0521C1800C2142
:101E200081801221017245720821418121888181BE
:101E30006188C181A1880182E188418208F0F9FAB4
:101E400070BD10B50A790024012A0AD0122A0CD0DC
:101E5000132A0FD0002349791A46FFF79FFF204627
:101E600010BD091D00F00AF802E0091D00F02BF872
:101E70000446F4E7091D00F062F8F9E770B58B88B5
:101E800000244C220546002B04D0012B04D0022B49
:101E900005D103E03C2202E0312200E03322404839
:101EA000AE00805900230068002800D00378092B79
:101EB00007D140784978814203D100212846FDF7B7
:101EC000EAFE204670BD70B50C4605460026FDF7BB
:101ED000E1FF012825D063892289A188E088FEF7E7
:101EE0006FF8002824D02902CA1D0E232D48C91DD1
:101EF00008F086FA0921017061784170A18841805B
:101F0000E18881802189C1806189018108F091FA8D
:101F10002348A9004058FD224030417D11404175C1
:101F20000BE0002361781A462846FFF737FF04E0EC
:101F3000617801222846FFF74FFF304670BD70B52B
:101F40000C4605460026FDF7A5FF002809D01448D9
:101F5000A90040588268002A1ED01078092807D0AE
:101F60001AE0002361781A462846FFF717FF13E0AE
:101F70006078517888420FD1A088002801D048228B
:101F800000E0002202212846FDF785FE05482902CF
:101F9000E430C91D08F007FB304670BD06040000A0
:101FA000C09100200E070000FFB583B00D46044627
:101FB00000210C980193271D8E4B0091002814D00E
:101FC00026887C207C2E00D9064628883246C119F6
:101FD00001989847059806802888801928802088CD
:101FE000801B2080009807B0F0BD6188207904290B
:101FF0000AD18149C140C90706D1012129807870E1
:102000002088401E20807F1C7C482188808B88424D
:1020100002D231200090E6E7764B04222146019857
:102020009847019826887821001D782E00D90E4601
:10203000704B3246394698470599301D0880CBE7EA
:10204000FEB51D46002301936D4B800014461B58BE
:102050000A9A081D099E0090022A21D108790122BE
:1020600022804A88042A08D1634AC240D00704D19A
:10207000022020800888401C0880587C1946401F98
:10208000C7B222880098173110185A4B3A46984721
:10209000781C2988C0B2081A28802088C01920809E
:1020A000002E12D02888B0420DD321880098514BC1
:1020B0000818324608999847208880192080288877
:1020C000801B288001E0342001900198FEBDF8B506
:1020D00006464B4980000C580025A068002806D011
:1020E000342101730C3008F0A4F9A56011E0207CC4
:1020F000617C88420DD204280BD3A28A101F0228CB
:1021000007D80095A37D34213046FFF71CFE08F068
:1021100090F9257404206074F8BDF7B582B00020F2
:1021200001900F4602983649800016460C5821E06F
:10213000904214D2121A8A4200D2114622468DB21F
:10214000123280182B4B2A4639689847207C401958
:1021500020743088401B3080386840193860207CFB
:10216000042807D1608A0C210C2800D30846617C22
:1021700040186074207C627C904202D23188002931
:10218000D6D1C0B2D1B2884230D1A68A658AA77DA5
:10219000301F02281FD81948808BA84206D3042E6E
:1021A00006D10298FFF757FCA84201D2312006E081
:1021B000002D03D0019800281AD001E034200190AE
:1021C000002000903B46324601990298FFF7BBFD84
:1021D0000C38A060E581A068002807D0019900298B
:1021E00004D00C3008F025F90020A06005B0F0BD47
:1021F0002846E6E7190F000022AA0A43989100201A
:10220000F89100203EB50546B8A107C96B4607C343
:102210001024B94B0C22694628469847002806D15D
:10222000A87B002802D1E87B002802D004242046A5
:102230003EBD0224FBE7FEB50E460546ABA207CA2B
:102240006B4607C3AC4C0C22694628468A3CA04723
:102250000422284631460C30A047FEBDF8B51E4684
:1022600015460C46B14202D10A46294612E00746FD
:10227000102C03D1FFF7C6FF04460C37102E04D1F3
:102280002846FFF7BFFF06460C35B44206D122466A
:1022900029463846984B9847002801D00020F8BDC1
:1022A0000120F8BD70B515460446102903D1FFF78B
:1022B000A9FF01460C34022907D160782178000279
:1022C0000843A84201D1012070BD002070BD10B5A7
:1022D000491EC9B200F018F910BDF7B50E46002529
:1022E00014462946009800F05FFA020069D0108970
:1022F0000099824F884206D110463946083027603F
:1023000000F0BAFA55E0081A062148438018C1893E
:102310000A308C464904890F20D101880523DB024D
:10232000CB1A032B03D929231B02994216D1744BD4
:10233000994220D100995289491C8A4219D32760B9
:102340000289801D120A3A7022685170090A917040
:102350002168C91C00F0AAFAC01C2AE06146C90B1A
:102360002DD061460905090D0818011D216040881E
:102370001FE0802526E062461205120D1018604A03
:10238000521E914217D18088002100F00DFA0028DA
:10239000EFD0276001893970090A79702168428974
:1023A0008A70120ACA7021680830091D00F064FAA8
:1023B000001D308006E0001D20600220F9E70625A0
:1023C00000E001252846FEBDFFB50F4681B0154649
:1023D00006460124002100F0E7F9002830D00189E9
:1023E0000624B1422CD0711A062251430818C28922
:1023F0000A305104890F0FD101880523DB02CB1A63
:10240000032B1DD929231B02994219D09B1C9942E9
:1024100016D05B1C994213D0D10B11D01105090DB8
:102420000C1820887E19864209D8334B60198A3BE4
:102430003A46001D049998476680002400E00D2468
:10244000204605B0F0BDF8B50E46154607460124F6
:10245000002100F0A9F900281FD00189B9421CD041
:10246000791A062251430B18D8890A334004800F89
:1024700009D118880521C902411A03290DD929213A
:102480000902884209D05E80E9041E48998801D576
:10249000014300E08143998000242046F8BDF8B54F
:1024A0000E46154607460124002100F07DF900285C
:1024B0001AD00189B94217D0791A062251430B1854
:1024C000D8890A334004800F09D118880521C90230
:1024D000411A032908D929210902884204D05888C1
:1024E000B0432843588000242046F8BDFB349B5F4E
:1024F0008000008000100000A30F0000D491002095
:10250000032800000010000070B50446F94A238833
:1025100000201268002B0AD10CE054899C4205D39C
:1025200012895918914200D3012070BD1268002A07
:10253000F3D170BD012307E016895D18B54205D3BC
:10254000538912685B1C9BB2002AF5D1238070BDB1
:10255000F8B50546CE88888868807004800F1446D8
:10256000022806D00F4601282AD00222022A29D0AA
:102570000EE00F683846FFF745FE0246102807D0E8
:102580000320400386430C37042AEFD1D0020643D0
:10259000A41AD94B394620469847601B2880F00B77
:1025A00035D03005000D411D49084900641A2080CE
:1025B00000206080601B310B09030843A88027E0DE
:1025C0000422D3E77878397800020843CB49288081
:1025D000884201D10020F1E7C849FF31884202D08A
:1025E000491C884203D1F004C00F801CE6E7C349B0
:1025F000491E884203D0292109028842CFD10220F6
:10260000A41F208060800021A180601BD6E7AE80DF
:102610002046F8BDFFB583B0002000901020019047
:10262000507A15464006800F0F46029003D00228CC
:1026300009D001280CD00226022E02D030461030DC
:102640000190002421E02868FFF7DCFD0646F3E74F
:102650000426F1E7002F07D0601CC108795C400711
:10266000400FC140C8070ED06868E100401800F074
:10267000B0F900283AD00199081880B2019000986A
:10268000401CC0B20090641CE4B2287AA042E1D899
:1026900000990398FFF738FF002828D100210198FE
:1026A00007F0EEFD044601986A7A2018019002981E
:1026B00002281ED029460698606003980088208171
:1026C000009BC0186081002022736073022E1BD013
:1026D0000198894B801B3246019098470198001B56
:1026E0000838E0810020064600902EE0402007B028
:1026F000F0BD2968102EDED09F2002400C31042E40
:10270000D9D120200243D6E748780978000208434F
:10271000E7E7002F07D0701CC108795C4007400F25
:10272000C140C8070FD06868F10041180098062220
:10273000504300191030019AFFF70AFF01900098EA
:10274000401CC0B20090761CF6B2287AB042E0D8A5
:10275000684A0021106805E023890589AB4203D34C
:10276000014600680028F7D12060002901D00C60E4
:1027700000E014600020BAE770B55E4E3468002CAB
:102780000ED0207BC00705D0002365681A460421BF
:102790001846A8472046256807F0CCFD2C00F0D14C
:1027A00000203060706070BD30B5524C024609CCDC
:1027B000083C002B13D01D89954210D858899042AF
:1027C00001D3184630BD186809E0038993420AD83E
:1027D0004389934202D3437BDB0707D0006800287C
:1027E000F3D1002030BD0029F5D1FAE7606030BD9B
:1027F00010B5404B1A6813E0548984420FD3507BC4
:10280000C407E40F8C4203D04008400008435073D3
:102810005868904201D100205860002010BD126815
:10282000002A02D014898442E6D9012010BD30B5B7
:1028300083885C04A40F0BD104880525ED02651B79
:10284000032D03D929252D02AC4201D1062030BD2C
:10285000DC0B04D01B051B0D1818008801E01805BF
:10286000000D824201D3072030BD5118814201D9A9
:102870000D2030BD002030BD10B50B46014600795B
:102880004006820FC88808D04118012A0AD018468D
:10289000194B10229847102010BD1870000A58706C
:1028A000022010BD1846FFF7C6FCF4E710B50B4632
:1028B000014680884004820F088808D04118012A08
:1028C0000AD018460C4B10229847102010BD1870E3
:1028D000000A5870022010BD1846FFF7ACFCF4E760
:1028E0001389834213D1107BC00909D00348801E8D
:1028F00008E00000CC910020190F00000328000020
:102900000520C0020870000A487002207047C01AF3
:102910000623584380180A30C8E7F0B50E46002554
:102920009C46144607462946FFF73EFF01004DD05E
:102930000889B8423FD0381A0622504340180A305E
:102940006246002A00D01060828853049B0F09D190
:1029500003880527FF02DF1B032F2CD929273F02FD
:10296000BB4228D04088002C23D00346E340DB073D
:102970001ED0097BCB0601D508251AE08B0701D4B0
:10298000D20400D50C250907890F092C09D00C2C7D
:102990000AD00D2C0AD00007800F814209D90846C1
:1029A00007E08007800FF8E70006F5E78006F3E709
:1029B000062530800BE0002C03D0092C04D006251E
:1029C00005E001204002F4E70020F2E70125284657
:1029D000F0BD70B505460188C08806244004800F0C
:1029E0001CD0012802D0022802D02CE0042009E0EB
:1029F0002868FFF707FC29684A7B0B7B1102194303
:102A000002280BD0841DE888C10B05D00005000DFD
:102A1000401D400840000419204670BD1048814206
:102A2000FAD0C01E81420ED0401C81420BD00C480F
:102A3000FF30814202D0401C814206D1A988052086
:102A400040028843E8D00024E6E70548401E814262
:102A500003D0292000028142D5D10C24DCE70000FC
:102A60000328000010B50021FFF79EFE406810BD4E
:102A7000F8B514460D4607460A4600266946204624
:102A8000FFF74BFF040006D00C2C02D0062C1CD004
:102A900036E00024012668460088002830D03846F9
:102AA000FDF748FA002822D00E2D22D00121384609
:102AB000FDF726FA002812D0002E1AD03846FDF76E
:102AC00047FA102815D20C241AE00C2D18D00D2D21
:102AD00016D0092D01D0032412E0022410E00221B7
:102AE0003846FDF70DFA002801D00F2408E0052430
:102AF00006E03846FDF71EFA694609888842F6D393
:102B00002046F8BD70B5FF4D84002859806A002822
:102B100005D00C3807F00EFC29590020886270BDE2
:102B2000FFB581B0174601980D46F64A810050580E
:102B30001E46806A002817D04388AB4211D14478E2
:102B4000062C02D0002C05D000E080240198FFF76D
:102B5000D9FF0FE0808838805058806A801D30602F
:102B600013E00198FFF7CEFF324639462846FFF7BB
:102B7000B4FB0446062C08D12846FFF773FF06462F
:102B800000232A4619460198B047204605B0F0BDFB
:102B9000FFB585B0088816460C46002704902088AB
:102BA0000121FFF701FE050015D021882889814207
:102BB00000D2208020883188884214D82A4669466D
:102BC000FFF78EFE03466A4608990E98FFF746FB0C
:102BD00000280AD104E030882080002F1AD004E0B9
:102BE0002088401C2080002F0ED02288002309213D
:102BF0000598FFF73DFF07462088294600F0A3FE11
:102C00003080002F0AD010E0318880B2884201D88D
:102C10000028C4D104980A27208006E02188109B50
:102C20000F9A0598FFF77CFF0746384609B0F0BDBC
:102C3000F8B507460020009008780C46122827D0E7
:102C40001D26E5883846FEF706FFC01E854200D2E5
:102C5000284685B2281D82B231463846FFF761F812
:102C60000646A088214670800831A74B2A46301DB1
:102C700098473046083807F0DCFB2078122805D04A
:102C80003902A24AA248491D07F03AFC0098F8BD53
:102C90001B26D6E770B59B4D84002859016910307A
:102CA000002904D007F04BFA07F044FBF5E770BDAC
:102CB00070B5944D8400285981691830002904D0DA
:102CC00007F03DFA07F036FBF5E770BD70B5154625
:102CD0000E461C4605220121FFF723F84670458069
:102CE0000471083807F0A5FB70BD10B5002A05D0A7
:102CF00013460A461221FFF7E9FF10BD01221321F6
:102D0000FFF70FF8083807F094FB10BDF3B5814FBB
:102D100081B00E46BD8B042203210198FFF701F814
:102D2000BA8B718804468A4200D211460198FEF798
:102D300097FE20466580083807F07BFB0020FEBD2B
:102D4000F3B585B0002002900F460598FEF783FE8C
:102D5000801E86B2049605987C88B988800000257C
:102D600003908C4201D8002C01D101201FE00121E9
:102D70002046FFF719FD0090002817D000898442F3
:102D800000D20446B888A04226D30121182007F0BB
:102D900077FA0190848001992046C91D009AFFF7B7
:102DA0009FFD0199002D887103D003E00A20029055
:102DB0001AE00546A84203D0019807F0BBFA13E0D9
:102DC0005049039808580199183007F09BF9701B77
:102DD000801E641C86B2A4B2B888A04204D3002C22
:102DE00002D0A81C8642C2D2464C03982058806963
:102DF000002812D004980027801B801C82B2052175
:102E00000598FEF78EFF0646022D0AD0022070704C
:102E100003983D4D2058846913E00298002817D08C
:102E200018E00120F3E7F019A1884180BF1CBFB270
:102E3000F019E11DA279801CA847A0792468C01967
:102E400087B2002CEFD13046083807F0F2FA07E0DD
:102E50000A20029003467A8839780598FFF736FFF2
:102E6000002007B0F0BDF3B58BB00C46488869462A
:102E70008881204640380990C68F0B9880000790C3
:102E8000002E0AD10B98FEF7E6FD401E86B2608840
:102E9000A18888421ED800281CD0A01D0A90801C42
:102EA000059009986946808F04AA083887B2A088DF
:102EB00008830A9808A96D4607C5022306AA03A934
:102EC0000B98FFF765FE050006D00A2D50D0062DA1
:102ED0004ED03FE001254BE0E0880521C902884241
:102EE00002D0491C884209D16846008CF9B2C3B2AD
:102EF000049A0598FFF7B2F9002815D16846008CAE
:102F0000B84209E0E8910020190F00003075000078
:102F100041050000989100201CD1FD4B3A460499D0
:102F200005989847002815D10121082007F0A8F935
:102F300001466846808988806846008BC880F54ACB
:102F40000798361F1058B6B2183007F0DBF80B9808
:102F5000FFF7D8FD6946088B401C8881A0888989C5
:102F6000884205D36946098B884201D0042E98D245
:102F70000998062DC68734D0E64E07983058183089
:102F800007F0B6F8002822D08000801C82B200240E
:102F900007210B98FEF7C5FE014607983058806957
:102FA0000CE0630082885B185A80641CA2B2540053
:102FB0006418C3886380521C006894B20028F0D162
:102FC0000846083807F035FA062D0DD006E06846A9
:102FD000828921782B460B98FFF778FE00200DB0F0
:102FE000F0BD6846808960800120F8E7F3B58DB0B8
:102FF000002006900D4648886946088228464038D9
:103000000A90C48F0027002C0CD10D98FEF723FDE9
:10301000801E84B26888A988884201D8002801D11E
:10302000012006900D98BB498000079008588069E0
:10303000002800D087790698002856D1A81D0B904B
:103040000A98A988808F6A4691840B9908AB03AAD5
:103050006E460EC6801FC3B209AA04A90D98FFF7D9
:1030600097FD0690002840D1684681898F4201D0A3
:10307000002F3AD1A01EFD22FD2800D31046814228
:1030800000D2084686B230460121083007F0F8F831
:10309000059068468789018A05989D4B818005982F
:1030A0008A3B867105983246C01D08999847A01B37
:1030B000801E84B29749079808580599183007F080
:1030C00021F868468089864202D10D98FFF71AFDE3
:1030D0006A46908C411C89B21182AA888A4204D324
:1030E000824202D0B81C8442AAD20A98C4870698A9
:1030F00006283FD0874C07982058183006F0F8FF74
:1031000000282DD00799002661588C69A179891C67
:103110004143891C8AB209210D98FEF702FE05463B
:10312000A079801C687011E0A819A1888170090A33
:10313000C170B61C764BB6B2A819E11D8A3BA279C4
:10314000801C9847A0792468801986B2002CEBD1A6
:103150002846083807F06DF9069806280DD006E0D5
:103160006846028A2978069B0D98FFF7AFFD00207C
:103170000FB0F0BD6846008A68800120F8E7F3B51B
:103180008BB0002002900D46488869468881284609
:1031900040380890C48F00200490002C0CD10B986C
:1031A000FEF759FC801E84B26888A988884201D83D
:1031B000002801D1012002900B9856498000079009
:1031C00008588069002801D080790490029800286E
:1031D0005BD1A81D0A900898A988808F6A46118340
:1031E0000A9909AB05AA6E460EC6801FC3B206AA8D
:1031F00003A90B98FFF7CCFC0290002845D1694643
:10320000898A0498884201D000283ED1201FFB22E1
:10321000FB2800D31046814200D2084686B23046D1
:1032200001210C3007F02CF807466846808A04908C
:1032300068468089B8806846008BF8803846344BF1
:103240003E72093032468A3B09999847A01B001FFD
:1032500084B23049079808583946183006F052FFB2
:103260006846808A864202D10B98FFF74BFC6A467B
:10327000108B411C89B29181AA888A4205D382426F
:1032800003D00498001D8442A5D20898C4870298F0
:1032900006284AD01F4C07982058183006F028FFFF
:1032A000002839D00799002661588C69217A091DB8
:1032B0004143891C8AB211210B98FEF732FD054665
:1032C000207A001D687019E0A819A1888170090A88
:1032D000C170B61CB2B2A818E1888170090AC17029
:1032E000921C96B20A4B2146A81909318A3B227AD0
:1032F000801C9847207A2468801986B2002CE3D17C
:103300002846083807F095F80298062810D00AE0F9
:10331000A30F0000E8910020684682892978029B6B
:103320000B98FFF7D3FC002059E668468089688037
:10333000012054E67CB50C464A8805460023092145
:10334000FFF796FB030007D1618801AB6A46284668
:10335000FFF7E6FB030007D0062B2ED0628821780A
:103360002846FFF7B3FC26E0684604882846FEF7A7
:1033700072FB401E844200D2204684B2601C82B29E
:103380000B212846FEF7CDFC0646FF4B2246401C8B
:10339000019998473046083807F04BF8684600888E
:1033A000844208D12846FEF756FB401EA04202D0B8
:1033B0002846FFF7A7FB00207CBD01207CBDFEB5A1
:1033C0000D464A88064600230921FFF751FB0400F9
:1033D00007D1698801AB6A463046FFF7A1FB0400BC
:1033E0000AD0062C3BD06A88297823463046FFF75E
:1033F0006DFC062C33D030E06946A88809888842E5
:1034000001D90724EFE70C1A3046FEF724FB401ED3
:10341000844200D2204684B2601C82B20D21304624
:10342000FEF77FFC0746A8880199D74B4118224632
:10343000781C98473846083806F0FBFFA88869468C
:1034400009880019884208D13046FEF704FB401E67
:10345000A04202D03046FFF755FB0020FEBD012000
:10346000FEBDF3B587B00898C84940380390808FF7
:103470000025C0034018000C05900798C44980003F
:1034800002900858183006F033FE06460398C48FA1
:10349000002C39D10798FEF7DEFA401E84B233E0E3
:1034A000089871000F187A88002309210798FFF700
:1034B000DFFA05002FD179886B4604AA0798FFF739
:1034C0002FFB050020D16846008AA04200D3204689
:1034D00087B238460121083006F0D2FE019087807D
:1034E0000198A94B3A46801D00999847A84902982F
:1034F00008580199183006F005FE0798FFF702FBFF
:10350000E01B761C84B2B6B20598B04203D9002CF9
:1035100001D0002DC4D00398002DC48722D1079874
:10352000FEF799FA001B82B200270F210798FEF7D9
:10353000F8FB009096490298085884690AE00098C0
:10354000A11DC019904BA288401C9847A0882468F0
:10355000C01987B2002CF2D10098083806F069FF34
:10356000002D0BD0062D0CD0089871000818428849
:1035700008982B4601780798FFF7A8FB002009B0B0
:10358000F0BD0120FBE7F0B506460A78002085B0C3
:10359000122A10D0522A11D10C464039888F0027A8
:1035A000001F85B2628802AB0A213046FFF760FA3D
:1035B000002805D01FE0304600F02DFA05B0F0BD20
:1035C000002229460298FFF732F9002813D1522031
:1035D00003906788241D3846FFF744FA84466946FD
:1035E000039808804D8001946B463A46012130468D
:1035F0006446A04701273846E0E7F3B5084685B0A2
:10360000403800900025C68F0C462F46002E07D16B
:10361000628800230B210598FFF72AFA050037D1AD
:103620000598638800218000594A049010589C46F0
:103630008646006905E0C28A9A4201D1012100E074
:103640000068002802D00029F5D003E0002901D14C
:10365000002E26D00098808F801F80B20290704686
:10366000203006F06CFD039060883105090D019152
:103670000090A388029A0399059800F093F9050039
:103680001CD04349049808580399203006F050FD97
:10369000628821782B460598FFF718FB384607B05B
:1036A000F0BD6046FFF7DEF906460023628802217E
:1036B0000598B0470127002DEAD1EFE702981721BE
:1036C000801D82B20598FEF72CFB05466088688055
:1036D000A11D2D4BA81D029A9847A088A8802846B6
:1036E000083806F0A6FE0227D8E7F3B587B0089899
:1036F000002140380290C08F0491009108994978C8
:1037000001297DD107998900039100285AD12048C9
:1037100040580469002C55D0002006460546059007
:103720002746E08A00211437FFF73EF800280DD025
:1037300001897A88914209D0511A0622514308180A
:10374000228961890A30FFF772F800E001200090B9
:1037500001200190009800280DD1788805998842B1
:1037600004D00590E68800202546A0802089B0423C
:1037700013D90720009008987A880178009B079851
:10378000FFF7A4FA079805E0190F00000000FFFFFB
:10379000E8910020FFF77EFA11E0B04206D2A54280
:1037A00004D0E68060892546A08005E06189401844
:1037B00086B2A8884018A8802468002CB0D102994D
:1037C0000198C887AE4E039830580469002C40D049
:1037D000E08A0490A0880690254614350498FFF7E7
:1037E00041F90746A08869464881208969460881D1
:1037F00060894880A81D019016200880002000E004
:1038000027E005902668002E0ED0069800280BD0E1
:10381000F18A354604981435814205D1012005907E
:10382000FF201730694608806B460121049A0798EB
:10383000B847934903980858103006F080FC20469A
:1038400006F078FD059834460028CED1012004907A
:103850000DE00798FFF71EFA0098002807D1012213
:1038600019210798FEF75DFA083806F0E2FD049882
:1038700085E6F8B507468500814E1BE0207D214690
:10388000C0061431000F401E00067E4A800D1258FB
:1038900038469047002804D001280FD002280BD1C9
:1038A00008E03846FFF704FA7059203006F047FC6C
:1038B00006F040FD7059046A002CDFD1F8BDF8B560
:1038C00006460A7A0402FF2580006D4B1E2A02D0AC
:1038D000D70715D033E01858002100680D4600289E
:1038E00000D00178132901D0142928D1611D664820
:1038F00006F059FE002211463046FEF74CF81EE055
:10390000002A1CD0D706FF0E182F18D8142A16D05C
:103910001A58126A002A14D000270022CA801858A8
:103920000C39203006F0EEFB0125601D06F0CFFDBE
:10393000000704D4002F02D03046FFF79AFF284634
:10394000F8BD0127E9E7F0B50C89844201D1488927
:10395000F0BD021B06235A435218D3890A325B0476
:103960009B0FF5D11388494EB342F1D1401C00257D
:1039700083B2771E488910E05189921D4904890F4E
:1039800004D11188B14205D0B94203D05B1C9BB26F
:10399000002D02D05B1E98B2F0BD9842FCD39C4231
:1039A000EAD3F0BDF8B58600002535480095855965
:1039B00014462D69069A2746002D09D0AD880127A7
:1039C0002D197F02BD4202D911200090F8BDAFB27F
:1039D0004C810B81079B2A48CB8080590D46046996
:1039E00010300AE0E18A914206D92A46214606F0C3
:1039F00002FC002C03D008E02468002CF2D12048FF
:103A000029468059103006F07DFB1D488059006919
:103A100087800098F8BDFEB5074608464038808F7D
:103A20000C46001F85B24A8800266B460B2138469B
:103A3000FFF71EF8030006D1002229460098FEF782
:103A4000F6FE030006D0628821783846FFF73EF97B
:103A50003046FEBD122002906688241D3046FFF7D6
:103A600001F884466946029808804D8001946B46AF
:103A70003246012138466446A0470126E8E70000A7
:103A8000E891002040C5011841050000032800000E
:103A900010B501221E21FEF744F9083806F0C9FCD2
:103AA00010BD10B50C4601021520F74A8001491DD2
:103AB00006F026FD2046083806F0BBFC10BDFEB51A
:103AC00001468000F14B02901A589468002C64D093
:103AD00050680190E2890092921D0C3893B20089DF
:103AE0000A02264601460C360027E948521D06F018
:103AF00087FC009A05468280019881882980019878
:103B0000C1886980307A092819D137460837727A16
:103B1000A81D391DDF4B921E98477878811E8FB201
:103B20002168002903D06988081A801C6880304603
:103B300024680C3806F0FEFB26460C3622E00836D8
:103B40000196403EB08F401E86B2009887420AD24E
:103B5000C01B3246864200D30246E8190199CD4B7C
:103B6000801D491C9847B81987B22068002802D0E8
:103B70006888801B68802468019826460C361438B3
:103B800006F0D8FB002CDAD1C04902980858002171
:103B90008160C160284606F04CFCFEBD10B50446AD
:103BA000BD484988828B8A4200D211462046FDF7E3
:103BB00057FFB648A10040584068002802D000785E
:103BC000012801D0412200E0002201212046FDF71A
:103BD000E2FE002010BDF3B583B00398AB4A80002D
:103BE000019010584068002802D00178072901D0C0
:103BF00040223AE0009004984078012809D010272C
:103C0000049800254038808F2E46801E80B2029096
:103C100024E00227F4E79D4901983B1D08584068BD
:103C20000C380189039802029948521D801E06F043
:103C3000E7FB04460498974B401946882680A770F6
:103C4000AD1C0498ADB24119E01C3A46891C984756
:103C5000E81985B2204606F0ECFB02988542DAD3DB
:103C60000098C088B04205D8002201210398FDF7D2
:103C700092FE0FE00098761C868000980121408813
:103C8000C903084300994880804901980858406852
:103C900006F0CFFB002005B0F0BDF3B583B003986C
:103CA0007A498000009008584468002C02D020789F
:103CB000032801D040223AE0049878494038808FA8
:103CC0000026C0034018000C3746019029E06F49D8
:103CD0000098637808589B1D40680C380189039848
:103CE00002026B48521D401F06F08AFB0546710018
:103CF0000498761C0818B1B24A00408828800498BD
:103D0000491C101847886F808EB260782871214650
:103D10000831604B6278681D9847284606F089FB99
:103D200001988642D3D3E088B84205D80022012109
:103D30000398FDF730FE0CE07F1CA780608801210E
:103D4000C90308436080514900980858406806F04C
:103D500070FB00209FE7F3B589B000250846019568
:103D600040380595808F0C46801E80B204900999DA
:103D7000464E8F00F15928464968002900D008783E
:103D8000099A1202039204286ED0052805D006284D
:103D900003D00A2872D04022D6E00091607807282C
:103DA00001D9102000E0022002900520079048E091
:103DB0006019C1788278080210430690019000983B
:103DC000007805280CD00098009A437807980832AC
:103DD00028180019801C0299FEF740FA00282DD0FF
:103DE0002A48039AC059029B4068521D0C38018929
:103DF00027489B1DC01E06F003FB06460698308030
:103E0000AD1CA8B221188978401C317180B22118EC
:103E1000CA788B7811021943801C718085B2029890
:103E200070716119B01D1B4B891C029A984702984A
:103E3000281885B2304606F0FCFA02E06078401996
:103E400085B204988542B3D30098C1880198814215
:103E500079D90099401C8880009801214088C903C5
:103E600008430099488077E00020064602900498B5
:103E70000691400703D01020009040E073E001203D
:103E800002900220F8E7000030750000E891002061
:103E900009050000190F0000989100200000FFFFA5
:103EA000F748039AC059009B4068521D0C3801899D
:103EB000F448083306F0A4FA0646601941883180B8
:103EC000AD1CA9B260184288891C89B26018728042
:103ED0004288B280891C02988DB2002816D00098C2
:103EE000B0716119F01DE84B891C009A9847009841
:103EF000281885B230880190304606F09AFA049866
:103F00008542CDD30298002807D017E0DC4831461F
:103F1000C0590C39083006F0F5F8002E0ED00422F6
:103F20000A210998FDF7FDFE01467088488009982E
:103F3000FFF7B7FD00200BB0F0BD04E00698C18884
:103F40000198814205D8002201210998FDF723FD3F
:103F500007E00699401C8880C948C059406806F0AF
:103F600068FA0598E7E70998FDF775FD6378801E04
:103F700098421BDDF059039A4068521D0C380189A4
:103F8000C0481B1D001D06F03BFA054660882880CE
:103F90006078211D801E82B2AA8000206880BA4B02
:103FA000A81D9847284606F044FACCE7F0596288E5
:103FB00040682146828062780839921EC2800022C1
:103FC00002816078801E4880F0590C39083006F074
:103FD00099F801200590F059C0E7F3B5084640383C
:103FE000808F85B0801E80B204904C780F462146A9
:103FF00005F0AAFF0599A24A8900039151584D681E
:10400000002D69D02978022966D1002864D00026C5
:104010000196142C01D0022000E010200090002016
:10402000029032E096490398009B08589B1D406817
:104030000C380189059802029248521D401E06F074
:10404000DFF90446B8194088B61C2080B1B2781850
:104050004288628001920098891C20718EB2B91941
:10406000601D894B891C009A984700992A46701850
:1040700086B26B780832601DFEF7F0F8002801D098
:1040800001200290204606F0D4F904988642029856
:1040900006D200280AD17D4901988842C2D101E0A8
:1040A000002803D1E9880198814205D80022012126
:1040B0000598FDF770FC0CE0401CA8806888012181
:1040C000C903084368806E4903980858406806F0A1
:1040D000B0F9002007B02FE74122E8E7F3B581B03F
:1040E000002000900198664A860090590F46456866
:1040F0000021002D00D02978042907D008291FD0DD
:1041000009291DD00A291BD041223AE0083006F0C7
:1041100016F804460C341022791C5B4B1330984778
:104120001020A071204606F084F92088E988814299
:1041300001D8002225E0401CA880514880593CE06D
:104140003946403FBA8F4E48521E94B20839002279
:104150004A8080590C39083005F0D4FF288900289E
:1041600002D0844200D30446454FB8598068C189C3
:10417000091989B2C181012000904002814205D90C
:10418000112201210198FDF706FC19E00198FDF7C5
:1041900062FC401EA04204DC2889A04205D8002809
:1041A00003D00198FFF78BFCC3E7E9880919E98080
:1041B000002801D0001B2881B859406806F039F961
:1041C0000098FEBDF3B585B005982D4A8000039098
:1041D00010584068002802D001780B2901D04122F4
:1041E00047E006994039898F0190491E002589B220
:1041F0002E460095029132E021490398B2000858FA
:1042000040680C38018901981718F888801D83B21E
:10421000059802021B48521D001D06F0F1F8B988EE
:10422000044601800298F988401B814200D208466A
:1042300082B2A280002060800698134B4119A01D15
:10424000491C9847A08841198DB2F988884201D04D
:1042500050200090204606F0ECF8761CF6B201984B
:104260004078B042C8D80298854201D050200090D2
:10427000009A01210598FDF78EFB00202AE7000037
:10428000E891002005050000190F0000FFFF000065
:1042900010B56149820089584968002902D009781F
:1042A0000C2901D0412200E000220121FDF773FB1F
:1042B000002010BDF8B5584F0B468600B9594C6820
:1042C000002C02D021780C2905D041220121FDF7D4
:1042D00062FB0020F8BD18464038808FE188801FBF
:1042E00085B298882A46401A80B221460C316081F6
:1042F0004118981D494B9847002804D160892189AD
:104300004019884201D90020C0436081B8594068F3
:1043100006F08FF8DDE710B53F498300C958002249
:104320004968002900D00A780C2A03D00F2A0BD044
:10433000412204E04A8909898A4205D0522201219A
:10434000FDF729FB002010BD0022F8E770B50D46EF
:104350004039898F324A091F8EB281005158B21DEF
:1043600093B202022878C989521D1B2816D02D4805
:1043700006F046F8044628781B2812D01320207037
:1043800066806888A080254B291DA01D32468A3B87
:104390009847204606F04DF8002070BD2148401E89
:1043A000E6E71220EBE770B5044608790D461228BF
:1043B00009D11B49A00008582202C1891948521D81
:1043C000163006F047F82A7901212046FDF7E3FA76
:1043D000002070BD70B506460A7A0D46FF20002405
:1043E000D10707D0002A05D01D2A03D851080E4B4B
:1043F00089005C58002C0DD01D2A07D01B2A05D03F
:10440000310215208001491D06F0CDF829460831FA
:104410003046A04770BD0000E8910020A30F0000C7
:10442000C09100200D05000070C50118F3B50024EF
:10443000224FCE0781B0F60F1C206043C519A87B20
:1044400009280BD129461431019806F04EF90028AD
:1044500004D0A87EC007C00F864204D0641CE4B21A
:10446000042CE9D303E0042C01D20120FEBD00207E
:10447000FEBD1C214843114910B54018002181732D
:10448000F9F773FC10BD70B50C49054600241C20DB
:1044900060434018807B002805D0641CE4B2042CE3
:1044A000F5D3072070BD1C2060434018082200216E
:1044B000034B143098472C70002070BD04920020EC
:1044C000750F0000032283079B0F02D083079B0F09
:1044D00000E01346244843708B079B0F01D08A07E6
:1044E000920F0270704702461B3AE02A0AD8FF2258
:1044F0004932904206D31D4A904203D81A4A403AA4
:104500009087D187704770B50146174D0C24002065
:10451000803D1C2242435219937B072B03D116691D
:104520003678F6070FD1052B03D112695278D207DE
:1045300009D1401CC0B20428EBD30B4806220C4B17
:104540000A3898470024204670BD70B505460146DC
:1045500005480622064C0A38A04703480622294689
:104560001038A04770BD00008492002090420000E7
:10457000190F000010B50346E94C00201C214143EF
:1045800009198A7B521E022A03D8096909789942BF
:1045900004D0401CC0B20428F0D3FF2010BDF3B5F6
:1045A00081B04227FFF7E6FF0446042820D21C20F2
:1045B000DB4960434618356900270622D94B284657
:1045C000143002999847B07B022811D1EFF310867E
:1045D00072B6287BC00709D070204443D248FF340C
:1045E00006225934CF4B20180299984786F3108839
:1045F0003846FEBDF8B504460C260078FFF7BAFF32
:104600006946C74D0870FF2806D01C214843401951
:10461000807B01282DD104E00846FFF734FF060017
:1046200027D1684600781C214843401900690028BA
:1046300001D005F07FFE684600781C2148434119EF
:10464000FF200C610876217B002903D0012908D0C6
:10465000022906D1B249062270312046B14B1430EE
:104660009847684600781C22504301214019817305
:1046700000263046F8BDFEB5054642200090287859
:10468000FFF778FF0746FF2850D0072000901C2036
:10469000A349784340180190A9780026490044189E
:1046A000607D143400280DD005F009FD06464088D1
:1046B000E9784018402805D9607805F005FD00200C
:1046C000607033E06878032801D001280CD160784D
:1046D000002801D005F0F8FC05F0D9FC6070002836
:1046E00024D005F0ECFC0646308872888E4B80188A
:1046F00080B2C0188B4BEA78696898477088E9786F
:10470000401870806878032801D002280CD10198E5
:10471000807B02280CD02078002801D005F0D4FC42
:104720006078207000206070002000900098FEBD2E
:104730006278A978384603F00CFEF1E7F8B5054633
:1047400012260078FFF716FF0746FF2808D01C2026
:104750003946414372480C18617D002955D101E06A
:10476000422652E0E17D00294FD16978002944D0EA
:10477000064620694188CA0717D00907890F07D064
:10478000417B0E30FFF752FE002801D00B263CE0A3
:1047900000201C2141438919897B002903D0401C3A
:1047A000C0B20428F5D304280BD0A07B02280AD07D
:1047B0002A7969883846266903F022FC002808D047
:1047C00022E0072621E02A796988384603F0F7FBC2
:1047D0001AE00220A073B078514DC00714D068468B
:1047E000FFF751FE00280FD16846007820761C2282
:1047F000042150434019817306E0384603F07CFDE4
:10480000002801D10320A07300263046F8BD10B562
:10481000FFF7B0FEFF2808D01C21414A4143891808
:10482000897B012903D00C2010BD422010BD00F06F
:104830005BF8002010BDF8B50C4609781C225143E6
:10484000374AE0788E18211D37690091B17B357E9B
:10485000032918D000281BD02846009900F0A8FB97
:1048600028461C2148432E4940180021C180009948
:104870000989490081800521018141810121C1739C
:104880008581B17317E000212848FAF704FD04E0A0
:1048900060783C2801D0432801D10120B073B8785A
:1048A000C00705D01C211E4A00206943891888735F
:1048B00060783C2809D1E078002801D0002100E090
:1048C0003C212846009AFAF71FFDE078002802D123
:1048D0006078002804D0617838782A46FAF769FEB3
:1048E000FF2030760020F8BDF8B500240C491C22CA
:1048F0005043274645182E19307D002802D005F078
:10490000E3FB3775641CE4B2042CF4D32869002857
:1049100002D005F00FFD2F610020A873F8BD000044
:1049200004920020190F00000080002039200000B0
:1049300038B505460C2300206946F94C0870097803
:104940001C2048430019827B062A01D3082A05D976
:10495000491CC8B2694608700428F0D3684600783C
:10496000042806D21C2148430019807B062818D150
:1049700004E06846FFF787FD030012D1684600781F
:104980001C21484300190069002801D005F0D2FC21
:10499000684600781C21484300190621056181738F
:1049A0000023184638BD70B503460C25DC4A0020AC
:1049B0001C2141438918897B062901D3082903D981
:1049C000401CC0B20428F3D31978002904D001296F
:1049D00017D01225284670BD0428FBD21C2148435D
:1049E0008418A07B0728F5D103F07DFF050006D0D1
:1049F0000620A0730021032005F0D5FDEAE708207A
:104A000023E00428E6D21C2141438C18A27B082A0B
:104A1000E0D0217E5E78490800254900002E00D0B4
:104A2000012631432176FD2631405E78022E0ED0DC
:104A300000267600314321765988A1829988E18247
:104A4000072A06D003F0DAFD0720A073C2E701268B
:104A5000EFE720690078800702D5B14A763200E09E
:104A600000229988588803F04DFFB3E710B5AC4A8F
:104A700000201C2141438918897B072904D0401C50
:104A8000C0B20428F5D303E0042801D203F0B6FD38
:104A9000002010BDF0B5487E8FB0401CC0B2099018
:104AA0000C46087D1C2148439D4906224018076991
:104AB0009C4D002105A8A847062200216846A8476A
:104AC0000025E07D2E460290FF282BD0954B062234
:104AD000211D05A85C3B9847607D40072FD5607875
:104AE000002810D03878C507E07BED0F8009012839
:104AF00001D1022005438A498A4B0622703168465B
:104B00005C3B98470EE02146864B06220A316846F8
:104B10005C3B9847257E002D04D0E07B800903286C
:104B200000D0FE25607D400709D5684640798009A0
:104B3000012804D1FE2D02D1787802287ED3207D71
:104B40001C21484376494018007EC10777D0099957
:104B5000012905D08006800F06D0022803D101E08C
:104B60000007F8E701267DE0A27CFF210020002A53
:104B700003D0208A010B0005000D05AA0B920A370D
:104B8000029A03970C92627D079108920290608CC2
:104B9000049000200D90054620370A9036E00E2044
:104BA00003996843461831460B9805F09EFD00288E
:104BB0002BD0F17A0C98814227D1B17A08988142A2
:104BC00023D1317B079881421FD107990020FF290B
:104BD00009D00E21039A69438918CA8802998A422A
:104BE00001D0F18001200499062909D30E214D43FB
:104BF000039969180A8904998A4201D0318130E009
:104C000000282ED101200A902BE06D1C787EA8424E
:104C1000C5DC0D98002824D1387E0E214843039925
:104C2000404B4518062228465C3B0B99984708984C
:104C3000A8720C98E8720798287301E039E035E013
:104C40000298E88004982881387E401CC0B23876EB
:104C5000042801D100203876787E042801D2401C37
:104C600078760A9EA07D012801D0002004E0002E65
:104C700001D0022000E001200999227D01290CD0F9
:104C80001C214A432649CF2351180A7E1A400001AD
:104C900002430A76002E09D00BE01C214A4320492A
:104CA000F32351180A7E1A408000F1E72046FAF7F4
:104CB000BFFD607F002802D0208C05F093F9002012
:104CC0000FB0F0BD10B548781C2148431449441872
:104CD000A07B08280ED0E08A002810D00521090208
:104CE0004843A18A0A225143421A0021032005F0B9
:104CF00007FC08E000210C48FAF7CDFA01E0FAF7CA
:104D000020FE0620A073A07B062802D0207E80070C
:104D100004D5206900214030C1708170002010BD91
:104D200004920020750F000042200000F0B500261C
:104D300089B0054668460C240670704B2022314627
:104D400001A8984768460670684600781C216C4A9E
:104D500041438918897B052905D0401CC0B26946AA
:104D600008700428F0D36846007804285DD3687A78
:104D700005F072FC06466846FFF785FB040054D137
:104D80002EE0142060434119CA89C88A520090421B
:104D900000D3104682B20220022A00D802460B8AB3
:104DA000088B5F00B84200D3384683B2934200D8E4
:104DB00013469C46630101A818184760C98901AFD2
:104DC0004900F9506346C360002182608174C17458
:104DD000694609780182F8F7CEFF002802D1641CE9
:104DE000B442CEDBB44201DA3B241EE068460178CF
:104DF0001C204143424801AB08180521056181731D
:104E000000200BE04101C9184A69D203140C142296
:104E1000424352195483098B9183401CB042F1DB09
:104E20006846007803F08FFE0446204609B0F0BDC6
:104E300070B50024324D0C261C2060434019807B45
:104E4000052804D0641CE4B2042CF5D30BE0042C38
:104E500009D204F035F81C2044436419206905F098
:104E600069FA00202061304670BDF8B50E781C222A
:104E7000234B487872430090D418A27BC878052A47
:104E80003AD1091D27690D46002F27D0002822D0CE
:104E9000304600F08DF8698CE180298914224900A0
:104EA000A180009902235143CA19D18A20460229C0
:104EB00000D819460181128B8A4200D911464181DE
:104EC00086810421C173F8F71EFF2A46002130466F
:104ED000FAF71AFA08E00020A07308E00021094858
:104EE000FAF7D9F90020A0732069002804D02069BE
:104EF00005F020FA002020610020F8BD750F0000A9
:104F0000049200200E20000010B50C460102491C3E
:104F10000346002C11D0FF200230002A14D0FA4A98
:104F20009B00D258002A0BD040239B5CDB439B079D
:104F300006D0F64A05F0E4FA10BDFF200130ECE798
:104F400092890A235A43F5E705F02DFB10BDF8B509
:104F500006468700EC48C559002D28D02C6A03E08E
:104F60002046246805F0E6F9002CF9D10124A000C0
:104F70002858002802D00C3805F0DCF9641E64B211
:104F8000002CF4DA002211463046FFF7BDFF002264
:104F900001213046FFF7B8FF3002FF21401C05F029
:104FA0006BFA284605F0C6F9D7480021C151F8BD73
:104FB000F8B5D54C06468700E0590D46002802D0CA
:104FC000FF242046F8BD0021442005F059F9E051A6
:104FD000002862D0044630020021401C05F04CFA43
:104FE0004422CB4B00212046984729892181698999
:104FF0006181A989A18129462046C54F0522143126
:1050000018305C3FB84720462830EB210170D12191
:105010004170012181700821C1700021017141712D
:105020008171C1711B23FF21E38149316182238298
:10503000A182B84926228B8FE386C98F2187515DD3
:105040000838491CA175E17502216177B1494031E9
:105050000A7882764978C176E08F4108287849003D
:10506000002818D000200143E1872946304604F08B
:10507000D5FB04461C204643A64806224038361875
:1050800030461430A91CB8476878B0762878F07696
:105090000920B07395E70120E5E7072491E770B593
:1050A000994C8300E358002B1AD040331C78E54319
:1050B000AD0715D0A508ED43AD0711D0002910D0DC
:1050C000012905D002290BD1A108890011431970CB
:1050D0001978F324214092001143197000F0D0F99F
:1050E00070BDA00880001043187070BDF8B50402B0
:1050F0000646641C17460D46204605F0E8F9824A2C
:10510000B1005158AA008F500121A9400143C9B2F2
:10511000204605F0B1F9F8BD30B47B4B84001B5933
:10512000002B10D08C001B59002B0CD09C78002C2D
:105130000BD0012C0ED0022C14D0032C03D1002A4A
:1051400001D00220987030BC7047002AFBD00122A9
:105150009A7001E0002A02D0012230BCD4E600227D
:105160009A70FAE7002AEED10320EBE7F8B505467E
:105170000002401C0F46009005F0A9F9064662495E
:10518000A8000C58002239462846FFF7C5FFBD008D
:1051900060590C3805F0CEF800206051FF2E06D083
:1051A0000120B84031468143009805F065F9F8BD0B
:1051B00070B51C461546544B82009A58002A11D0EF
:1051C0008B00D258002A0DD01278130004F0E6FEAE
:1051D000090A060B101A1F2933380A0022462946ED
:1051E00000F0A2FB70BD2246294601F031F970BDE6
:1051F00000292246294602D001F01AFF70BD01F0B5
:1052000042FE70BD2246294601F007FB70BD002911
:105210002246294602D002F057FC70BD02F086FB00
:1052200070BD00292246294602D000F0E5FE70BD7F
:1052300000F0C1FE70BD2246294600F087FA70BD1D
:105240002246294602F0E3F970BD70B513461C0AE8
:105250002D4B0A46A5005B590020FF211578002B35
:105260000BD04026F65CF643B60706D01968002935
:1052700007D0072D04D0022070BD072DFCD200E01E
:1052800009782B0004F08AFE0805060A0E12161A89
:105290001E05F1E7204600F04CFB70BD204601F0F2
:1052A000ADF970BD204602F0D4F870BD204601F083
:1052B000B4FB70BD204602F02AFD70BD204601F00F
:1052C00054F870BD204600F091FA70BD100A10B578
:1052D000D9B20D4A8300D258002A3DD040239B5CAE
:1052E000DB439B0738D01368002B1AD01B788B4206
:1052F00017D1032902D005292ED10DE00022042167
:1053000001F0DBFC28E0000088920020409C0000B7
:10531000750F0000449200200022042102F0D2F90F
:105320001AE05268002A17D012788A4214D1032951
:1053300004D0052907D008290ED109E000220A214E
:1053400001F0D5FD08E00022072102F019FB03E07F
:105350000022042102F032F9002010BD10B5100A1D
:105360000122222100F09EF9002010BD10B51E4B35
:1053700084001B59002B10D08C001B59002B0CD023
:105380009C78002C0AD0012C0CD0022C10D0032CBD
:1053900003D1002A01D10020987010BD002AFCD052
:1053A0000320F9E7002AF8D002229A70002203E0D5
:1053B000002AF2D101229A70FFF7A6FD10BD024625
:1053C000094B92009A5800201268002A03D01278E4
:1053D0008A4201D123207047032A03D0052A01D035
:1053E000082AF8D12A2070478892002070B5154607
:1053F000100A0C46214A81005158002911D0227907
:10540000032A10D0403109788907890F032905D074
:1054100000290CD001223D2100F044F9208804F03D
:10542000E1FD002070BD214600F0E1F8F9E7FAF750
:1054300012FD01022A462046091D05F012F801203E
:1054400070BD70B5150AD8B2032804D02846F9F704
:10545000DAFA002070BD0949A8000C58002C09D0C8
:105460002046203004F06BFE04F064FFE08F022140
:105470008843E087284600F003F8EAE78892002096
:10548000F8B50746834980000D58E88F800728D477
:1054900001262A464032804B2C6A32E01078617A2D
:1054A0000007800F4900C9184978C140C807C00FDC
:1054B00025D004F0C7FD2146784B09310090C01873
:1054C000774B227A9847E88F02210843E887217AB0
:1054D0003846009A04F04BFB002803D0009804F0F3
:1054E000C8FDF8BD002EFCD12846203021460546D7
:1054F00004F02FFE2146284604F01AFEF8BD246869
:105500000026002CCAD1F8BDF7B50F4600986149B6
:1055100080000E58002F1ED0002E1CD0387819287D
:1055200019D25D4940000D5C012128460C3004F081
:10553000A7FE0446029860602046594B2A46394629
:1055400009309847304625722146203004F0DAFDB4
:105550000098FFF795FFFEBD70B50C460B4605465B
:1055600002220021FFF724FE2346022201212846C1
:10557000FFF71EFE002070BD70B50C460B460546B9
:1055800003220021FFF714FE2346032201212846AF
:10559000FFF70EFE002070BD10B50B460122002162
:1055A000FFF706FE002010BD38B504280CD2394D97
:1055B00084002C59002C07D02034247A04252C4058
:1055C00000D00124002C01D10D2907D911246D46EA
:1055D0002C70AA7069701A46694605E00D216C4668
:1055E000217062701A466946FFF78EFF38BDF0B52C
:1055F0000C460546274980000E582188274B182263
:10560000C9188BB0264B01A89847403630786946B8
:1056100080070979800F192928D21F4B4A00668814
:105620009F5CBE422CD1D2185278C240D2071FD004
:105630008800194664390B58E28801A92846984722
:1056400001000BD03D2916D0282914D068460079D6
:105650000A46014600232846FFF7A6FF208804F0EB
:10566000C1FC0BB0F0BD022804D0F7E7002807D03A
:105670000128F8D13D210122284600F013F8EDE77A
:1056800007226B461A705970284600226946FFF7B8
:105690003BFFE3E78892002010C60118008000203D
:1056A000190F000010B50446814B80001B58403391
:1056B0009878002809D199701146204604F021FA03
:1056C000032202212046FFF7EAFC10BD70B5054613
:1056D000774A800010580029046825D16178002994
:1056E00002D0012920D11AE0032202212846FFF727
:1056F000D6FC002201212846FFF70EFD217928461D
:1057000000F019F801206070002211462846FFF7CA
:105710002DFE012200212846FFF7FEFC70BD6179B5
:1057200001222846FFF7BEFF00212846FFF71EFD95
:1057300070BD0021CAE708B502226B461A70597085
:10574000C0B25C4A6946FFF7DFFE08BD002901D1FF
:105750001178BBE7704770B50E4604465449800087
:105760000D58002211462046FFF7D6FC00220121E9
:105770002046FFF7D1FCE88F7178C007C21720469A
:10578000521CFFF78FFF002070BDF8B5150A48497D
:10579000A8000C58D8B21646162801D04221085548
:1057A0002346423300221F4611462846FFF700FDDC
:1057B0003B46002201212846FFF7FAFC0322022182
:1057C0002846FFF76CFCFF21304604F055FE4034BC
:1057D000A27800212846FAF713FC00212846FFF79B
:1057E000B6FB2846FEF745FE0020F8BD70B514460E
:1057F00006462F4A80001058C08F800512D4002919
:1058000005D00022631D11463046FFF7D1FC01256B
:10581000224600213046FFF769FC00213046FFF7A1
:1058200055FF00E00225284670BD70B50E462049A0
:1058300082008C580025002C09D040342178C943BF
:10584000890704D06178C90703D03A2517E00C25F1
:1058500015E00102491CFF2006230A46073004F028
:10586000CFFD07210170002141700671132E08D071
:10587000467104F0DEFD607801210843607028461F
:1058800070BD16214171F4E710B50C460102491CA8
:10589000FF2006230A46073004F0B2FD07210170FD
:1058A000002141700471447104F0C3FD10BD00007B
:1058B0008892002033570118F8B50F46064681003C
:1058C0005748445825686878002815D0012825D005
:1058D0001F27E87800280AD0224630323946304661
:1058E000FAF7C1FB40346078FD2108406070002168
:1058F0003046FFF73BFCF8BDE08F4007E9D4304667
:1059000000F07FF8E08F08210843E08701206870ED
:10591000024600213046FFF7FFFBF8BD002211468A
:105920003046FFF7F9FBD4E7002901D11178C3E72E
:10593000704770B500250446FF2909D001250021D4
:10594000FFF7D4FB00212046FFF7B6FF284670BDC5
:10595000D0780028FAD03249A0000A584220815C51
:1059600020463032FAF77FFBF0E770B52C4D82000D
:10597000AC584E7830231E554B8863868988A186A3
:10598000E38F04210B43E387A9580968002902D05B
:105990000978012909D0190705D400F032F8E08F01
:1059A00008218843E087002070BD0021FFF784FFB5
:1059B000F9E770B51A4982008C580025002C09D0EF
:1059C00040342178C943890704D06178890703D519
:1059D0003A2514E00C2512E00102491CFF200423A3
:1059E0000A46073004F00CFD0121017000224270CC
:1059F000C17004F01EFD60780221084360702846E3
:105A000070BD1CB50C216A4611700B2151700549FF
:105A100051800521918000226946FFF775FD1CBD6C
:105A200088920020C509000010B5FF4982008958FE
:105A30004968002906D00978062903D100221121DE
:105A400000F010F810BD10B5F74982008958496878
:105A5000002906D00978062903D10022122100F07E
:105A600001F810BDF0B51746064685B08000EE4A35
:105A70000090155804206C6862788A420BD0132974
:105A800001D03D2701E03D2F04D1012239463046A7
:105A9000FFF708FEC0E00A390B0004F07FFA0906A0
:105AA0003F46577389A8BDBC55000021304604F01D
:105AB000B4F8012200213046FFF758FC2746E98F51
:105AC0002037B87D8906C90F884207D0D74B2422DA
:105AD00003213046FFF768FD12206070B87D002872
:105AE00012D00021304604F0B3F9012202213046E1
:105AF000FFF7D5FA0B256946304600220D70FFF7F7
:105B000003FD657001221BE0022211463046FFF7BB
:105B1000C6FA304600F049FA0D203CE0002130463C
:105B200004F07EF90C206070ECE70222114630464A
:105B3000FFF7B5FA304600F038FA0D206070002209
:105B400001213046FFF7E8FA05B0F0BD6A46107053
:105B5000254600A820350822B54F013021462C31BA
:105B6000B847042202A829460130B84700226946F6
:105B70003046FFF7C9FCA18E221D3046FBF7F8FD29
:105B80000E2008E0002F08D0A84B06220321304643
:105B9000FFF70AFD12206070D6E720462146A54B8C
:105BA00001220C3024310096F7F720FB0F20F2E79A
:105BB0002146224630460C311C3204F061F90121A5
:105BC000304604F045F905216A461170304600223E
:105BD0006946FFF799FC102060700122114630469B
:105BE000FFF79AFAE88F01214902084347E00022B3
:105BF00001213046FFF790FA0121304604F010F9F8
:105C00001120607006216B46197030468A4A694639
:105C1000FFF77AFC98E70627834800994058002848
:105C200025D040300078C043800720D00121304685
:105C300003F0F3FF002202213046FFF730FA002F75
:105C400003D02034A07D002803D039463046FBF72E
:105C5000BAFDE98F20208143002F12D0002040019F
:105C60000143E987002211463046FFF77FFB0121FF
:105C70003046FFF77BFAE88F012149028843E88725
:105C800062E70120EBE710B567498200895809688F
:105C9000002906D00978062903D10022022100F04C
:105CA00001F810BDF0B51746064687B080005E4A81
:105CB000009015582C68607888421CD0092901D0C2
:105CC0003D2712E0132F0ED004DC062F07D0082F3B
:105CD000F6D108E01A2F04D0222FF1D103E00528D5
:105CE00001D00428ECD13D2F04D1012239463046A1
:105CF000FFF7D8FCCCE0030004F050F909061F1AA6
:105D0000427785A240C540000021304603F085FF60
:105D10003620005D00280BD00A216A4611703046FB
:105D200000226946FFF7F0FB01206070024657E051
:105D3000304600F03AF903201FE0012200213046EE
:105D4000FFF7ADF9012211463046FFF70FFB0022A5
:105D500011463046FFF7E0F90021304604F078F8AC
:105D60000021304604F05CF80B216B461970304678
:105D7000324A6946FFF7C8FB0220607007B0F0BDE9
:105D80002246A08E2432069203236A461370507274
:105D9000000A9072274600A81C370822244D0130C3
:105DA000211DA847082202A803300699A84704220B
:105DB00004A839460330A847002269463046FFF759
:105DC000A3FB04206070012200213046FFF7A4F9F4
:105DD0002034A07D002802D00222114601E00222D8
:105DE00001213046FFF75BF9C8E702220021304667
:105DF000FFF755F9012211463046FFF7B7FA0520A3
:105E0000607001220BE0204621460A4B01220C3033
:105E100024310096F7F7EAF906206070002200218D
:105E20003046FFF779F9A9E788920020475A011810
:105E3000190F0000FF5E0118295A0118875C01182C
:105E40002146224630460C311C3204F019F801215B
:105E5000304603F0FDFF0121304603F0E1FF06214B
:105E60006B461970304600226946FFF74DFB08204B
:105E70006070012200213046FFF74EF9E88F0121C2
:105E80004902084337E0002211463046FFF744F943
:105E9000FE4800994058002821D040300078C04387
:105EA00080071CD0284640304178F72211404170CD
:105EB0000121304603F0B1FE002202213046FFF7F7
:105EC000EEF8002201213046FFF750FAE98F20203A
:105ED0008143002F11D0002040010143E98739465A
:105EE0003046FBF770FC00213046FFF73FF9E88FA2
:105EF000012149028843E88740E70120ECE7F8B533
:105F00000F461006E149800D0858154600282AD092
:105F10004022125CD243920725D0AA008958DC4E59
:105F2000C98FC90720D00468002C1CD0207806280F
:105F300019D16078032802D006280FD109E0042285
:105F4000204639461C30B0470822391D20462430EF
:105F500003E01022204639460C30B0476178E8B2A1
:105F60000022FFF79FFEF8BD4468002CFBD020788C
:105F70000628F8D160780D2802D00F280FD109E04B
:105F80000422204639462030B0470822391D2046D9
:105F90002C3003E01022204639460C30B04761789F
:105FA000E8B20022FFF75EFDF8BD10B50146B94822
:105FB000F7F74DF910BD30B4B44C8300E358002915
:105FC00010D0012910D0022912D0032912D1517802
:105FD00003290BD04033197889070BD03D2230BC00
:105FE00009215FE61278FAE71A22F8E79278F6E7D5
:105FF0005278F4E730BC704710B5A44C8300E358E6
:1060000000290ED0012903D0022901D0032907D18C
:1060100040331978890703D03D221321FFF722FD71
:1060200010BD1278F9E770B5054698498000085808
:106030000024C18FC90702D14068002802D024245F
:10604000204670BD0122FF2038231146073004F09E
:10605000D7F90246062010700A2050700121362020
:1060600081542846FFF742F800220A212846FFF70C
:10607000F9FCE5E710B58549820089580024CA8FEC
:10608000D2070AD0096800290DD0097806290AD15B
:1060900000220121FFF706FE06E04968002902D030
:1060A0000978062902D02424204610BD00220B21A5
:1060B000FFF7D8FCF8E7F7B500980D468100734864
:1060C00000264458E08FC0070BD02068002825D058
:1060D0000078062822D13D2209210098FFF7E2FD31
:1060E0001DE060680C27002814D10122FF2038230E
:1060F0001146073004F084F9074606203870002066
:106100003621C8553A4601210098FEF7EFFF0A20D4
:106110007870074660680178062902D02426304648
:10612000FEBD0446A97A687A09020143A186294680
:10613000042213312046564B1C309847294608222A
:106140000B312046524B243098470822691C504B93
:10615000201D9847002239460098FFF783FCDEE7B0
:10616000F8B50E4605468100484800244058C18FC6
:10617000C90706D00068002809D0017806290FD089
:1061800005E04068002802D00078062802D02424C8
:106190002046F8BD3D2213212846FFF763FCF7E7B0
:1061A0003146074604220931394B203098470822EE
:1061B000711C3846364B2C30984700220421284663
:1061C000FFF770FDE4E710B53049820089580024DC
:1061D000CA8FD20706D00968002909D00978062994
:1061E0000ED005E04968002902D00978062902D0BE
:1061F0002424204610BD3D221321FFF733FCF8E78D
:1062000000220521FFF74EFDF3E710B51F4982007C
:1062100089580024CA8FD20706D00968002909D0FE
:10622000097806290ED005E04968002902D00978CE
:10623000062902D02424204610BD00221021FFF799
:1062400011FCF8E700220821FFF72CFDF3E7FFB56A
:106250000E4982008E58002581B0002E1ED0374690
:1062600040373978C943890718D0F18FC90715D04D
:10627000042815D22821895DC907C90F00D0012142
:1062800000290DD0797809070CD505E08892002007
:10629000190F0000FF5E01183A252BE00C2529E0BC
:1062A0001A2527E00102491CFF2038230A4607303F
:1062B00004F0A6F8044606202070002060700498C0
:1062C000002805D0A0860822344B201D039998474A
:1062D00010222046314B0C3002999847F08F8006EF
:1062E000C10F36200155204604F0A3F87878082124
:1062F00008437870284627E4F8B5294F06468500FC
:1063000078590C2400282ED04022125CD2439207E8
:1063100029D04068002826D00278062A23D1427866
:106320000E2A20D10024002905D010221B4B0C304E
:106330009847002213E02030807D00280ED00121F4
:106340003046FEF713FF78590122C18F5202914364
:10635000C18706213046FFF797FA04E006220E2196
:106360003046FFF77FFB2046F8BD70B50025044698
:10637000FF290AD001250021FEF7B8FE00221146B0
:106380002046FFF78FFC284670BD0549A00008583D
:10639000403081782046FBF716FAF4E7190F000029
:1063A000889200203EB56C462170EB236370D122A9
:1063B000A2700122E27000226271A271E271227267
:1063C0002271092906D19B4A810051582031097A4E
:1063D0000B40637000222146FFF796F83EBDF8B5EA
:1063E0000F4606468100934844582568687800287F
:1063F00015D0012826D01F27E87800280AD0224689
:10640000283239463046F9F76CFE40346078FB217B
:106410000840607000213046FEF7A8FEF8BDE08F0E
:106420000106E9D4C00701D0082100E00E21304662
:10643000FFF7B8FF01206870024600213046FEF7E2
:106440006BFEF8BD002211463046FEF765FED3E72D
:1064500030B400290ED001290ED002291ED0032904
:106460001ED151780E291BD19178002918D01A29F4
:1064700006D011E01178F8E751780E2910D11A21D1
:10648000042809D26B4B82009A58002A04D020328B
:10649000137A0824A343137230BCA0E75178E4E7D1
:1064A00030BC704770B5634A8300D2580024D38F44
:1064B000DB0701D0242418E013464D7820321572F2
:1064C0008D785572CD7895720D79D5724D79157399
:1064D0008D795573CD799573097AD173D98F8022CF
:1064E0001143D9870921FFF75DFF204670BD70B5C4
:1064F000504A8300D2580024D38FDB071AD01346AA
:106500004D78203215728D785572CD7895720D794F
:10651000D5724D7915738D795573CD799573097A47
:10652000D173D98F80221143D9870921FFF73AFF10
:10653000204670BD2424FBE770B53E4D84002B59E6
:106540004E781A46203216728E785672CE7896722F
:106550000E79D6724E7916738E795673CE799673FC
:10656000097AD173D98F80221143D98729590968B3
:10657000002905D00978022902D10021FFF72FFF59
:10658000002070BDF8B5014682002A4800248058DA
:10659000021E0AD0054640352B78DB439B0704D00A
:1065A0006B785B0703D53A2426E00C2424E0002610
:1065B0000127042907D22030007A0823184000D090
:1065C0000120002806D1D08FC20703D1000601D4D4
:1065D0001A2411E00902491CFF2004230A4607304F
:1065E00003F00EFF022101704670C77003F021FF17
:1065F00068780421084368702046F8BD70B500250E
:106600000446FF2909D001250021FEF76FFD002176
:106610002046FFF7E4FE284670BDD0780028FAD067
:106620000449A0000A584220815C20462832F9F72C
:1066300058FDF0E788920020F3B50646FE4A800038
:10664000155800272C6883B06178002902D00129F1
:1066500070D13BE001216170E98F09060CD5042E51
:106660000AD21058002807D02130007A08210840AB
:1066700000D0012000280AD1E088F049884200D3E8
:106680000846E0806089884200D308466081E3883C
:10669000A1886289248914276D462F706C70240AA2
:1066A000AC70EA70120A2A716971090AA971EB715A
:1066B000190A2972304600226946FEF725FF012299
:1066C00000213046FEF728FD05B0F0BD002211463E
:1066D0003046FEF721FD0498002819D1298A208927
:1066E00081420BD1E989A288914207D1A98A6289A6
:1066F000914203D1698AE288914209D0009063896E
:10670000A288E188304603F0ECFA00281FD0002769
:10671000002F0FD020892882A088E8816089A88274
:10672000E0886882208900906389A288E1883046E9
:10673000F9F7ABFDE078002804D040356878DF2118
:106740000840687000213046FEF710FDBCE70127C5
:10675000DEE7FFB583B003980C9C8500B64840592E
:10676000C58EA54200D22C46058FA7B29D4200D30C
:106770001D467C237C2A00D91A464524240116464E
:10678000A14200D80C46C18F09060CD503990429F3
:1067900009D2010007D02921095C0822114000D04C
:1067A0000121002906D1A5498D4200D30D468C4216
:1067B00000D30C46018AB14208D1C189B94205D142
:1067C000818AA14202D1418AA94211D00682C781A1
:1067D0008482458223463A4629460096039803F070
:1067E00080FA23463A46294600960398F9F74DFD6C
:1067F0001522694603980A704E70320A8A70CC706E
:10680000220A0A714F713A0A8A71CD712A0A0A72F4
:106810000022FEF779FE07B0F0BD30B4002910D099
:10682000012910D0022920D0032920D15178142920
:106830001DD1917800291AD0192908D01A2906D01B
:1068400011E01178F6E75178142910D119210428A4
:1068500009D2794B82009A58002A04D02032137A48
:106860002024A343137230BCE6E65178E2E730BC43
:106870007047F8B5704B82009A5800255268002A7C
:1068800001D0242529E08B784E781C024A1C344321
:106890001B2C1DD3537916791A0232431B2A17D3A6
:1068A0000B79CE781B023343FF264936C91CB3420D
:1068B0000ED34F7909793F023943B14208D3FB2CFB
:1068C00006D8FB2A04D85E4EB34201D8B14201D9A2
:1068D000202502E00094FFF73CFF2846F8BDF8B5FC
:1068E0000A460546810054480024405801680029A2
:1068F00002D00878042801D0242443E09078567808
:106900000002531C30431B2816D35E791F793602D0
:106910003E431B2E10D31679D77836023E43FF270D
:106920004937D21CBE4207D35679177936023E4307
:10693000FF274937BE4201D220241FE08E888642BD
:1069400000D23046888050781778CE8800023843CD
:10695000864200D23046C88058791B790E890002E1
:106960001843864200D230460881507912794B890B
:1069700000021043834200D218464881214628462F
:10698000FFF75AFE2046F8BDF7B517462A498200A0
:106990008C580025002C0AD0264640363178C94351
:1069A000890704D07178890603D53A2531E00C2592
:1069B0002FE004282FD22821095D2022114000D089
:1069C0000121002927D0E28901998A4202D1618AF6
:1069D000B9421BD00102491CFF200C230A46073094
:1069E00003F00EFD04210170002141700121C170EE
:1069F00001998180C7807C21018145210901418164
:106A000003F017FD70782021084370700198E0862C
:106A100027872846FEBD1A25FBE738B50024054622
:106A2000FF290FD001240021FEF760FB002128463A
:106A3000FFF702FE204638BD88920020480800007B
:106A400090420000D0780028F4D00020034602468F
:106A5000014600902846F9F718FCEBE730B5F74CF3
:106A60000398E47AA40701D5012400E006248A42B1
:106A700016D8FF25F435AB4212D81925ED01A942ED
:106A80000ED8A2420CD3A8420AD80A2808D30A2258
:106A900050438A00891849085B1C5943884201DA2F
:106AA000002030BD012030BDF0B50C460746E4495A
:106AB00080000E588DB0384603F027FAA1880222D4
:106AC00049000091E18849000191A189022900D87B
:106AD00011460291E1890222022900D81146254679
:106AE00020350391E9786A46490091741782F18F45
:106AF000C9070BD10199401E081803F025FA084672
:106B00000299C91C02910399C91C0391C107C90FBD
:106B10006A46D174E17800291DD1697A00291AD119
:106B2000618AC84A914216D0002914D0A1886A46C9
:106B30004900089102990991118A9185618A490059
:106B40000818A188490003F0FFF908A80A91F7F78F
:106B500072F900280BD06846F7F70DF900280AD023
:106B60000020E084E088A084E8700DB0F0BD608A69
:106B7000E084089815E0F18F0698C90704D1401CFD
:106B8000059903F0E1F9084683B20598218AC0030C
:106B9000020C384603F011F9AB4903F0EBF9E0843D
:106BA0000598C003000CDEE770B586B014466A464F
:106BB000117005460822211DA44E00A80130B047DF
:106BC0002320005D6A46507221460E22103102A831
:106BD0000230B047002269462846FEF795FC06B011
:106BE00070BDF7B5164686B0954A8100019054589D
:106BF0002922F178925D114301D0012700E000279E
:106C00000799002945D1B18C2289914207D1328957
:106C100063899A4203D17289A3899A4205D021815E
:106C2000318961817189A18101271C21884A4143F1
:106C30008D18B1890222022900D811460491F189E8
:106C40000222022900D81146039103F05EF9009058
:106C50002089400002902846F7F787F80298A8801C
:106C60000098E8800498288103996981E08FC00723
:106C70000CD10098A988401E081803F065F9E98036
:106C80002889C01C28816889C01C68812846F7F7BC
:106C90003AF8002F07D0A0890090638922890799CC
:106CA0000198F9F783FAF078002804D0403460782E
:106CB000EF210840607009B0F0BDF0B516460746F8
:106CC00085B0BA005E4B00929D5800202C680629C2
:106CD0000BD062788A427DD161780B0003F05EF9B7
:106CE000072B280896BCBABCBA0006216170F3E7EE
:106CF000002211463846FEF70FFA002E18D0042F56
:106D000016D24F4900980858002811D02030007A38
:106D100000210222104000D00120002808D0E88F76
:106D2000C00704D11C204A4A78438018C17393E0FD
:106D3000012028210855E88F10210843E8872046C4
:106D400020300390007A0028384626D003F026F839
:106D500001463B4A009810584089C2008018081824
:106D600009302084039A01219170208221463846FF
:106D7000FFF79AFEE28CE2832089238C61896E46BC
:106D80000BC60398A38C8178384602F069FF06464B
:106D900004206070002E5FD121E002F0FFFF20820E
:106DA00021463846FFF780FEE08C60822548A082AD
:106DB000E08220836083A08322460F213846FFF7BC
:106DC000F3FE012200213846FEF7A6F9E88FC0073E
:106DD00003D000E018E002202EE003202CE0002188
:106DE0006A4611700399384689785170E18B518059
:106DF000A18C91802189D18061891181218C51815F
:106E000000226946FEF780FB05B0F0BD0022114666
:106E10003846FEF781F9002E1ED12089228C618927
:106E20006B4607C32220015DA38CE28B384602F03B
:106E300017FF060010D104206070E5E7989200204B
:106E400088920020FFFF0000E2040000190F0000FC
:106E5000049200200028D7D0E078002805D12846E9
:106E6000403041784906490E417022463146384645
:106E7000FFF7B7FE00213846FEF778F9E88F1021BA
:106E80008843E887C0E730B4F84B84001B59DC8F97
:106E9000E40701D0022400E00324002910D00129D6
:106EA00011D002291FD003291FD151780F291CD1DD
:106EB0009278002A19D0192A09D01A2A07D00FE08F
:106EC00006241278F5E751780F290ED11A220428EA
:106ED00006D2002B04D02033197A0225A943197257
:106EE000214630BCE9E65278E3E730BC7047F7B59D
:106EF00084B0049B16469C00DC4B00221D591046B2
:106F00006C680B290BD063788B422DD16178C91F37
:106F10000B0003F043F805113D077F7F7B000B2139
:106F20006170F3E7002E75D1002201210498FEF76D
:106F3000F3F8012028210855E88F1021084327463F
:106F4000E8872037387A002810D02089228C618980
:106F50006B4607C3A38CE28BB978049802F080FEDD
:106F6000060057D10A20607007B0F0BDA1882889BB
:106F7000814216D8E288824213D322896B899A42D1
:106F80000FD16289AB899A420BD1A0802889E08019
:106F9000002E12D0002332460F210498FEF704FB86
:106FA00041E0608900902389E2880498F9F746F966
:106FB0000820607001207872D6E7E88FC00713D0F0
:106FC00004982A230102491CFF200A46073003F0D7
:106FD00017FAA74B05462A222146984701206870D8
:106FE000284603F026FA1EE021460498FFF75CFDD0
:106FF000224610210498FFF7D7FD09206070012276
:1070000011460498FEF788F8AEE703E0002AABD0FB
:10701000002808D1224631460498FFF7E2FDE98FA7
:1070200010208143E98701210498FEF79FF89BE730
:10703000092300290AD0022906D003290CD151784E
:10704000102909D1927803E0527801E012780B23DD
:10705000002A01D019464AE77047F7B582B00C46BE
:107060000298824980000E5820890090A188174616
:107070000025E3880A460298FFF7F0FC002803D0B9
:10708000F08FC00741D101E020253FE060897949B8
:10709000381A80B2884201D2282537E030680028AB
:1070A00002D00178032904D070680921002813D088
:1070B00027E0A1888184E18801812189418161895A
:1070C00001846188C1836178203081702A46032160
:1070D0000298FFF7F2FD19E00122FF202A23114652
:1070E000073003F08DF90246032010700021D170A3
:1070F00029208154481E508201210298FDF7F6FF95
:10710000072170680278032A02D0242528467BE6EE
:107110004170A2888284E288028122894281628948
:1071200002846288C28362782030827001220272F7
:1071300000220298FFF7DBFEE8E7F7B582B00C46C5
:1071400002984A49800008580190406800270028AA
:1071500001D0242779E0207AE179000208430090E9
:10716000A079617903020B43A078617802020A4397
:107170002179E07809020143E61C651C0298FFF7BB
:107180006DFC00280AD00198C08FC00708D00321E9
:107190000298FEF714F9070002D056E01E2754E0CB
:1071A00002982A230102491CFF200A46073003F0F7
:1071B00027F9024603201070072050700023D37077
:1071C0006978287809020143918071783078090242
:1071D0000143D180687929790002084310817079D0
:1071E00031790002084350811146657A2031CD7013
:1071F000E07AA57A000228431082607B257B00029A
:1072000028435082E07BA57B000228439082607C6B
:10721000257C00022843D082E07CA57C0002284324
:107220001083607D257D000228435083E07DA47D8E
:107230000002204390834B7201210298FDF756FF14
:10724000002207210298FFF752FE3846DCE5F7B529
:1072500082B0029800278200044880580468002CFD
:1072600002D02078032807D0242759E088920020F4
:10727000190F0000FF7F0000087ACA79000210434E
:1072800000908879CD1C4E1C497903020B4370781D
:10729000317802020A43697828780902014302988A
:1072A000FFF7DCFB002833D0707831780002084308
:1072B000A18888422ED3E288944690422AD86A78E0
:1072C0002B7812021A43624524D88A4222D372795B
:1072D000337912021A4323899A421BD1814200D981
:1072E0000846A08068782A7800021043844500D9B7
:1072F0006046A08068792A79618900021043814242
:1073000000D9084660810020E0832034A07002E0AC
:107310001E2700E020273A4602210298FFF7CDFC05
:10732000384671E5F8B50C4605468000A149009045
:1073300008580026002810D0074640373978C9433E
:1073400089070AD0042D0AD22821095C02221140A3
:1073500000D00121002902D004E00C2648E0C08FB3
:10736000C00704D07878C00603D53A2640E01A2634
:107370003EE02902491CFF202A230A46073003F079
:107380003FF803210170002141700123C37061881F
:10739000628949008A4200D21146C181218822892E
:1073A00049008A4200D2114681816188C1802188CA
:1073B0008180A1880181E18800224181042D0CD2C5
:1073C0007C4C00996158002907D02031097A0222AB
:1073D000114201D0012200E0002201465A40203132
:1073E0000A724B7203F025F8787810210843787000
:1073F0003046F8BD10B503466E4A9C0012590C2069
:10740000002A25D04024A45CE443A40720D052687D
:10741000002915D0002A1BD0D4884888844200D97E
:107420002046D08090880C88A04200D820469080CA
:107430005489C888844200D920465081002202E045
:10744000002A05D03B2208211846FFF750FD0020F6
:1074500010BD70B514460646564A800000251258E5
:10746000FF2912D0D08FC00602D5607800281CD02A
:107470000125224600213046FDF738FE61780022C2
:107480003046FFF71AFC284670BDE078002806D089
:107490004032917822463046FFF7A3FBF3E74032B3
:1074A00050784006400E5070EDE70225EBE7F8B546
:1074B0000D46100A1C21404A414300278C18FF2B1F
:1074C00006D0DEB23146F8F756FE012E0BD014E09E
:1074D000E088A188401C02F037FD288888420CD043
:1074E0002046F6F742FC2888A1884018401E02F08A
:1074F0002BFDE1802046F6F706FC3846F8BD70B556
:10750000C5B22C4EAC003059002850D04030017824
:10751000C94389074BD04078C10648D4C00946D139
:107520002902491CFF202A230A46073002F068FF7F
:107530001C21214A6943335989180A89DB8F4989FB
:10754000DB0701D1C91ED21E032303700023437041
:10755000C3708281C18131590989C180315909893A
:107560008180315949890181315989894181315954
:10757000CA8FD2070BD0042D1AD2002918D020317F
:10758000097A0222114000D00121002910D00022E6
:10759000014620310A724B720021C943418202F038
:1075A00048FF30598022403041781143417070BD0E
:1075B0000122EDE78892002004920020F7B50098A0
:1075C000042682003C481027845865686878884201
:1075D00009D103280FD004280CD1204605221830E9
:1075E000364B291D9847E08F0121B843E08700986A
:1075F000FDF7BCFDFEBDE08F291D3843E0876A8999
:10760000009802F053FB0028EDD16E70FEBD0029FA
:107610000BD129498300C95812784968002904D040
:107620000978082901D10521C8E77047F8B50E4649
:1076300007462149800008580025C18FC90702D19B
:107640004068002801D0242525E0F0881C49101A44
:1076500080B2884201D228251DE03902491CFF2052
:107660000C230A46073002F0CBFE044608202070A7
:10767000032060700522711C104B201D9847F08874
:107680006081224601213846FDF730FD00220321AA
:107690003846FFF793FF2846F8BD8100064840585A
:1076A000002806D04021095CC943890701D0183061
:1076B000704700207047000088920020190F0000DA
:1076C000FF7F0000F7B582B0029817468200FD48A0
:1076D00000268558002F2C6805D0002211460298FC
:1076E000FDF71AFDE8E06078884278D1030002F0E7
:1076F00055FC0504403BC2EBBB00E88F102108435A
:10770000E8872846E1792030C176A1798176E17A4F
:107710000177E179EA7D4800D040C00705D0A07923
:10772000AA7D4000D040C0077ED1A27916266B46C4
:1077300002981E7099705A7000226946FDF7E4FEA7
:10774000012200210298FDF7E7FCE88FC00701D075
:107750000220B7E0A0790121C00700D000210298E3
:1077600002F0FFFA0320ADE0002211460298FDF777
:10777000D3FCA079012100280CD0AB7D4200DA4077
:10778000D20701D0002002E0800702D5022020723B
:1077900000E02172E07900280CD0EB7D4200DA4055
:1077A000D20701D0002002E0800702D502206072DB
:1077B00000E06172A07A002812D0207AA97D00280A
:1077C00001D04108491C607AEA7D002801D04208B6
:1077D000521C914204D000206072207246E043E0C7
:1077E000207A002802D1617A00293FD0A97D0028A3
:1077F00001D04108491C491EC8B20090607AE97D59
:10780000002801D04108491C491ECFB2029802F05D
:10781000C5FA6989CA0089184018093083B2A38063
:107820003A460099029800E045E002F076FA070037
:107830001ED001260020A08020726072627A217A18
:107840009446A2886B469646182202981A70597080
:1078500062469A707246DA70110A197100226946FE
:10786000FDF752FE002E41D105B0F0BD0126E5E73F
:1078700004206070E2E7002211460298FDF74CFCFC
:10788000207A002802D1617A002915D0617AAA7D78
:10789000002901D04A08521C521ED1B2EA7D0028AC
:1078A00001D04208521C521ED2B2A388029802F0A4
:1078B00034FA070005D019E00421029802F051FAC9
:1078C00014E004206070CFE7E88FC00702D0617A2F
:1078D000207A01E0217A607A002902D04908491C07
:1078E000E975002802D04008401CA875E98F1020D7
:1078F0008143E987E078002805D1207A002802D169
:10790000607A00280DD0EB7DAA7D39460298F8F701
:10791000DCFCE078002804D040356878BF210840BE
:10792000687000210298FDF721FC9DE7002910D026
:10793000012910D0022920D0032920D151781629FD
:107940001DD19278002A1AD0192A08D01A2A06D0F6
:1079500011E01278F6E75178162910D1192204287F
:1079600009D2584B81005958002904D021310B7A93
:107970005B085B000B720021A4E65278E2E77047D7
:10798000F8B51746064682004E48002F85586C68A9
:1079900004D00421304602F0E4F914E06078884213
:1079A00058D1052813D0062855D0072852D1207A5F
:1079B000002802D04008401CE875607A002802D0F8
:1079C0004008401CA875E88FC10767D075E0E88FB4
:1079D00010210843E887C0071ED03102491CFF2050
:1079E0000C230A46073002F00BFD0521017001212E
:1079F00041700021C170294620318A7EA3791A4046
:107A00008271CA7EE3791A40C271097FC172A17A7C
:107A1000817202F00EFDD6E72035A87EA279012101
:107A20001040C00700D00021304602F09AF906202D
:107A30006070A97EEA7E17236C462370A270617085
:107A4000304600226946FDF75FFD012211463046AF
:107A5000FDF762FBF8BD002201213046FDF75CFB1B
:107A6000207A002802D1617A002992D0617AAA7D19
:107A7000002901D04A08521C521ED1B2EA7D0028CA
:107A800001D04208521C521ED2B2A388304602F0E6
:107A900044F9070097D107206070F8BD1021884392
:107AA000E887207A002802D1607A002805D0EB7D93
:107AB000AA7D39463046F8F708FC01213046FDF72B
:107AC00055FBF8BD88920020002901D1127857E7B4
:107AD000704770B50C460646A1498000085800253D
:107AE0004168002901D0242537E0A17800290CD075
:107AF0006178002909D0C08FC00708D00521304621
:107B0000FDF75DFC050002D027E01E2525E03102CF
:107B1000491CFF200C230A46073002F071FC0521A6
:107B2000017041706178C171A17881710246A078BD
:107B30006178884206D1002804D0411E084201D154
:107B4000012000E00020907201213046FDF7CEFABE
:107B5000002205213046FFF713FF284670BD70B59F
:107B60007F4A83008C78D2580025002C02D04B78B5
:107B7000002B00D11E25D38FDB0705D01368002B07
:107B800002D01A78052A01D0242517E09A792240DC
:107B90009A71DA794C782240DA718C7849788C4283
:107BA00006D1002C04D0611E0C4201D1012100E05D
:107BB000002199722A460221FFF784FD284670BDF4
:107BC000F8B513464A78054696080024B600C81C46
:107BD000002E03D18E78B708BF0001D020240DE01D
:107BE000002A01D1002E09D04678077836023E439C
:107BF0009B1B5C4E9BB2B34200D22824584BAE0074
:107C00009E593368002B02D01F78052F08D0736867
:107C1000002B02D01E78052E10D02424204650E7D9
:107C20001A72897859724178027808021043988054
:107C3000224603212846FFF745FDEFE71A728978AF
:107C40005972417802780802104398802246062132
:107C50002846FFF795FEE1E702469300404A0C20D4
:107C6000D258002A0AD040239B5CDB439B0705D0F7
:107C7000D07D4870907D0870002088707047F8B5FE
:107C80000C468200364900268F583146042807D218
:107C9000002F05D02921C95DC907C90F00D00121D6
:107CA0004D0001210D43002F09D040373978C943D9
:107CB000890704D07978490603D53A2625E00C26B1
:107CC00023E06178294202D02178294201D11A2685
:107CD0001BE00102491CFF200C230A46073002F07A
:107CE0008FFB05210170002141700121C170617875
:107CF0002940C171217829408171A178C17202F0B7
:107D000098FB78784021084378703046D9E6F8B57A
:107D100015460746124A800000261458FF2912D043
:107D2000E08FC00602D56878002817D001262A46C1
:107D300000213846FDF7DAF9697800223846FFF766
:107D4000C1FC3046BDE6E8780028FAD0E37DA27D8C
:107D50004034A1783846F8F7B8FAF2E70226F0E79F
:107D600088920020FF7F000070B5304D1C21A87A5A
:107D700048432F494418A08C002802D102F01CF976
:107D8000A084208A4004400C2082A87A0621401C4E
:107D900002F0DAF8A97270BD24491C22897A514395
:107DA000234A89180A8AD20B05D0898BC90A8142D5
:107DB00001D10120704700207047F8B50E460546F6
:107DC00002F0A0FC194CC022A17B1346CB40217BC2
:107DD000C0B20907090F0B438707BF0F0121B94044
:107DE0000B432B70A37B1746DF40237B1B091F43EC
:107DF0006F70A37BDA4033071B0F1A43AA70627BB4
:107E000000095201203202430A43EA70607B0321D9
:107E1000401C02F099F86173A07B0221401C02F023
:107E200093F8A173207B401C2073F8BD989200202A
:107E300000830020F7B5164607468500FE494859DD
:107E4000002828D004460021F5F778FDA08E000711
:107E500002D50220F6F7C6F80198002815D00423B1
:107E6000FF220021F54802F0CBFA0770002146708E
:107E7000C170002E05D0218F002902D02034A17EB0
:107E800000E00021817002F0D4FAEB4C605902F05E
:107E900051FA00206051FEBDF8B51F4600230D4683
:107EA00006461C46002A04D0104602F008F98378E2
:107EB0000488B10048190006020DE1481218908F9D
:107EC000568F9B1DF6B21B021E4356879487012DC9
:107ED00010D10B06548F0421240924010C4354872C
:107EE000190D7723DB00C918138F89089B0B9B039F
:107EF0000B431387002F03D0002801D002F0E4F8D1
:107F0000F8BD38B5002817D0014620310C46CA7E8E
:107F1000416A4B1C08D04368CA4DC91AC903702373
:107F2000090C53435B1919800C2100911346C64973
:107F3000F5F732FD0120207738BD70B504003DD043
:107F4000A08E254600072035002803DAA07D401CBE
:107F5000A07523E0A16A6068411A0A01E16A12096A
:107F600049008A421AD3A17D491CA175A06202F082
:107F7000C9FB112101F0E8FF4804E97F000C00294A
:107F800007D0002802D0202802D002E0012000E023
:107F90001F20616808180101090961602046F5F792
:107FA000D4FB00280AD0E87F002807D1606A401C73
:107FB00004D0E87E3C220121FFF73CFF70BD30B5C4
:107FC000EFF3108372B684009B48002500593A24D1
:107FD00025540287828E120704D5012241681203BC
:107FE000891804E0002905D04268490151180901A7
:107FF000090901E00021C94383F31088416230BDC3
:10800000F7B586B006988C4D8600A8590C24002838
:108010007ED10021402002F033F9A851002877D00A
:10802000054606981C214843884940180190046978
:1080300002F092FB069A039202904022844B0021A8
:10804000284698478348E8618348A8610220E8757C
:108050000520A8750020A8608048A8822846203006
:10806000069A00900146C276A068E8626088A886F9
:10807000607F4877207F401E887708982887F0B275
:10808000761CF7B204900026607802F0E5FA01460B
:10809000A88E13280AD004DC10280DD012280FD186
:1080A00008E0152804D01D280AD101E06C4805E03D
:1080B0000126FBE70626F9E76A48022641432961C3
:1080C0000498012E04D1617BC90701D0012200E090
:1080D0000022217BD201CB070321490211435A0E12
:1080E000114320221143020155483143161871876C
:1080F000217B0422C907490E11433A011018059249
:1081000004904187A88E400718D50098C07E00E0F3
:10811000EFE006214843AF21C900471852482146E5
:108120004B4B0E31062238185C3B9847708F032169
:10813000C0B2890208437087B7870DE00198002319
:10814000027D19460698FFF7A7FE01980023827D5D
:1081500001210698FFF7A0FEA88E410701D48007F1
:1081600004D4308F800B800330870EE07721059890
:10817000C9004018318F8008890B8903014331877A
:108180000498018F4904490C0187308F4004400C4A
:108190003087A88E2B490207069870235843403930
:1081A00046180190002A0CDA02984914401801017F
:1081B00009090220F5F711FF2C4881880520296163
:1081C00000E004203082A078400701D5002000E0C4
:1081D000A07E01020198F184234BFF308D30C0183E
:1081E00021461B4B0E3106225C3B9847154A0199EC
:1081F000607B8F187882A88E000702D4F1200002DD
:1082000000E01B4830851F2070850098C07E8006E6
:10821000000E01017720C00008188008B0861549BB
:108220008888F083C888308413487084B18C5520C6
:10823000090A0902014321E0A89200200602000079
:108240008083002080810020CFAC011804920020A0
:10825000750F00003B7F0118037F011801600000CB
:108260002E070000B205000000800020D092002000
:10827000278000009892002055550000B18400200E
:1082800038817881A88EC006C00FC0003880009861
:10829000807F81000143F182217B0398C907C90FC8
:1082A0000002202210430843708201982146334B7C
:1082B000FF30143106225930C018314B984760788E
:1082C000F988E022914340010143F98002986860F7
:1082D0000020A8602846F5F738FA002808D106AB38
:1082E00007CBFFF76CFE0099002008776868A8624A
:1082F0000024204609B0F0BD10B503460C20EFF372
:10830000108472B69A001F49895800291ED0203166
:10831000087F002802D0012817D105E000220121A2
:108320001846FFF787FD10E0CA7E70235A43164BAC
:108330000120D218108005231B071868012252065D
:1083400090431043186002200877002084F31088BF
:1083500010BD70B5EFF3108472B68500094B5B5900
:108360003C25ED5C002D04D020315A5484F3108854
:1083700070BD0123FFF790FDF8E7000000800020AA
:10838000190F0000A89200208081002070B5FF4CDA
:10839000002520680068002828D0014620310A7E88
:1083A000002A02D0012A21D10FE00021F5F7C6FAF8
:1083B000F5F7D0FD2068006801F0BCFF206805607B
:1083C000017A49084900017210E0087D7023584382
:1083D000EF4B0122C018028005200007026801232C
:1083E0001B069A431A430260022008762068007A2E
:1083F00000280FD10223FF220021E64802F000F8F6
:108400002168497A4170057002F013F8206801F084
:1084100091FF256070BDF7B58100DC4882B005682A
:108420006C5826462036307D009002F095F903996D
:108430000746401A00010009401C216A4008814299
:1084400001D9091A12E0F5F785FDD3480068411CEF
:1084500001D0606007E0A18DE08D081A4000C119CD
:10846000CE48014061600020A060E18D2162084695
:10847000CB494843C8498988884200D308462061CF
:10848000C6496868491C88420BD86168081A00010F
:1084900001210009C906884203D2FFF777FF05B022
:1084A000F0BD0498002803D10521A17561686162BF
:1084B000BC49A182F17D012000038A0010430843DA
:1084C000009B70214B43B249403959180F46C8826E
:1084D000AF49208C59180880B07D0B2801D00A289C
:1084E00001D1B1480881B14A206A904200D31046B8
:1084F0000122D2030243FA850020C884287C800729
:1085000008D52946AA48FF330A31062259331818DC
:10851000A84B9847287CA97C82076B7CD20F002946
:1085200001D1800701D5012000E000201B020901D4
:108530000B43910000250B430343FB84B17D3A8A32
:10854000520952010A433A822046F5F7FEF8002804
:10855000A5D175776586A2E738B500280CD004460A
:108560002034227D0C210091A37E9349F5F714FA63
:10857000F5F7F0FC0120207638BD10B5040014D0CA
:108580003820005D002810D102F0E6F8616A411A37
:108590000A01A18D120949008A4203D3A17D491C19
:1085A000A17560622046F5F7D0F810BD70B5774927
:1085B0000C200968002920D00D68002D1CD038201F
:1085C000405D002818D102F0C7F869680446081B0E
:1085D000000101220009D206904203D9601A00016D
:1085E000000940423C2807DD00212846F5F7A6F99E
:1085F00028466C60F5F7A9F8002070BDF1B5634D11
:108600000C24286886B0002876D10021142001F0BF
:1086100037FE286000286FD0044602F09DF80490D1
:108620000020039006981C2148436449614F40187C
:1086300000901422002106695C372868B847B0789A
:10864000C00733D00021642001F01AFE206000280A
:108650002CD0642205460021B8475948E8615948A2
:10866000A8610320E8750520A87530894C49484366
:1086700049498988884200D308464A492861A98225
:10868000F088A885F288EA852846317920300023D1
:108690004175C3752A628376069A027501290BD04B
:1086A00000200390207A0121084320723078C0070F
:1086B000424803D0763002E00120F2E770300146F4
:1086C0000290062220463B4B0A30984730782074AF
:1086D00070786074069860720025A5740098808A8E
:1086E00000280AD038494843491101F02DFC04996B
:1086F00040180001000902E0F2E00020C043606081
:10870000069827688006000E00010590002F7DD096
:1087100001972037387D00213977092179762B4957
:108720001B4B8A8870214143403BCD188C46EA831D
:10873000264AD2882A84264A6A84AB8C55221B0A90
:108740001B021343AB84124B0022C9180091CA8448
:108750003178A27C8907637CC90F002A02D1227C70
:10876000920701D5012200E000221B0289000B4381
:108770001343EB8417492985009A00211181009A3F
:1087800051813178C907C90F000225E0B892002055
:108790008081002005020000D0920020FEFFFF0F24
:1087A000E204000001600000723E0000FF3F000094
:1087B00000800020190F0000B5B0011804920020BD
:1087C0007B85011859850118204E000098920020E1
:1087D000555500002780000020221043084368827E
:1087E00060465B4BFF3006225930C018594B029946
:1087F000984706206885787D01280AD00020A88641
:1088000000998882387F002812D000E039E00A20E1
:108810000FE077210598C90040188008A8860099C4
:108820008882387F002801D00B2002E0092000E078
:108830000820B875C0B20B2801D00A2802D10099CF
:1088400045480881B87D2882F87D0121090382000E
:1088500011430143E98201980099008C0880019836
:108860003E49006A884200D308460121C9030143FA
:10887000E985E88EC009C001E886A88D400840005F
:10888000A8850398002818D0354A05980321801838
:10889000428F120912010A43428700218187418FCA
:1088A0000322C9B2920211434187018F890B8903C8
:1088B0000187018F4904490C01872B4929484862E7
:1088C0002068002500280AD00499416004464162CE
:1088D000F4F73BFF002802D13D20055565860024B2
:1088E000204607B0F0BD10B50C20EFF3108472B62F
:1088F0001E490968002902D0FFF748FD002084F3D3
:10890000108810BDF8B5194905460C680C201646AC
:10891000002C1BD0002D0BD001F01EFF0746144881
:108920001449684301F010FB38180001000901E008
:108930000020C0436060002E05D006222046054B73
:1089400031460A309847FFF731FE0020F8BD00009D
:1089500000800020190F0000723E0000FF3F000061
:10896000808300200100010000010050B892002027
:10897000204E00007102000070B5FA4C00252068FE
:108980000068002827D0014620314A7B002A02D007
:10899000012A20D10FE00021F4F7D0FFF5F7DAFA31
:1089A0002068006801F0C6FC20680560C17C4908A9
:1089B0004900C1740FE0087E70235843EA4B01223E
:1089C000C018028005231B07186812069043104345
:1089D0001860022048732068C17C002912D14068C9
:1089E000002809D141200423FF22C00001F008FD26
:1089F0002168097D0170C57001F01BFD206801F040
:108A000099FC256070BDF7B50D46D6498000096810
:108A10000C5801F0A1FE0646401B00010009254646
:108A2000401C2035216A40082F7E814201D9091A55
:108A300009E0F5F78FFACD480068411C11D060605D
:108A40000020A060618D21620846C9494843C7499A
:108A50008988884200D3084620610298002808D0FF
:108A60000BE0218D608D081A4000C2498019084032
:108A7000E5E70A21A17561686162BF49A182012011
:108A8000687570204743B848218C38180180218CC4
:108A90000122D2030A43B44940397918CA85002615
:108AA000C6842046F4F751FE002800D1AE75FEBD05
:108AB000FEB504002DD0AB48254620350068297E40
:108AC00001916E7D02910189408900908F003946A5
:108AD000606801F039FA0098791A40000818B1006E
:108AE0000831814200D938180299702251439E4AB8
:108AF0008008801B403A8918C8870C200090EB7DC5
:108B00009E492046019AF4F747FFF5F723FA012022
:108B10006873FEBD10B5040014D02D20005D002840
:108B200010D101F019FE616A411A0A01218D120962
:108B300049008A4203D3A17D491CA1756062204689
:108B4000F4F703FE10BDF1B592B00320099069203F
:108B500000010F9001F000FE0E9001F0D3FD814C5A
:108B6000070220683F0A00287DD10021442001F03F
:108B700087FB2060002876D000210D9112991C22DD
:108B800051437F4A7F4B891844220D6904460021D6
:108B90009847129921756978A176A978E1762646D9
:108BA00029782036F175002131764020015568780A
:108BB000C007734801D0763000E07030014608905D
:108BC0002046704B062226305C3B984720466D4B72
:108BD0000622E91C2C305C3B9847BF2060759F2023
:108BE000A0750320E075CD2020761F2060762046FA
:108BF0001C3012990690FFF7E0F837802220390CDC
:108C000001550220F07038460C2101F09DF94F1DEE
:108C10005D4837710089F4F7B5FA7071594B042239
:108C200068465C3B06999847564B032231465C3BAD
:108C300001A89847F0786946C8710020088121464C
:108C4000504B052215315C3B04A898477079694662
:108C50004001384348752746687A0837C00748D02E
:108C600000213C2000E028E101F00AFB2060002800
:108C70003FD03C22434B069000210790984707982D
:108C80004249C16107984249816107980421C17531
:108C900007980A218175079800218160A889344AC4
:108CA0005043324A9288904200D31046079A10618E
:108CB0000798314A828206986A8902850698AA89AD
:108CC0004285069820300173069B1A62C1757F2287
:108CD000027501234375129A0276688B3880A88B3F
:108CE0007880688AB880A88AF8803972E07C184356
:108CF000E074388869464881B8888881F888214BB3
:108D0000C881162223485C3B98470120A0746878EC
:108D10000021B174129A80079206120E2168120186
:108D2000C00F0C9200297DD0069120311091097E50
:108D300070230B9159430C4B0622403BCF180A91EC
:108D40007A85094B2289C91807914A8077230C9AA2
:108D5000DB00D2189208BA868A82A17C00291BD037
:108D60000F211AE0BC92002080810020D0920020C8
:108D7000E2040000FCFFFF0F01600000F1B30118E6
:108D800004920020750F000098920020158B0118A6
:108D9000B18A0118908600200E2100233982504AA2
:108DA0009188F983D18839844E497984BA8C5521C8
:108DB000120A12020A43BA840799CB842978B27C3A
:108DC00009028000014350000143F984B07C00286F
:108DD00002D007990D988881287800280ED1B07CA0
:108DE00000280BD10A98404BFF30E91C06228D3039
:108DF000C0183E4B98470799A87848820126F60389
:108E00003B4900203985079908810799488169788D
:108E10000B98C907C90F000220221043084378822B
:108E2000062200E017E00A982F4BFF305930C01897
:108E30002E4B089998471098B110007B820011437F
:108E40000143F98206980799008C088006983146FC
:108E5000008C0143F985274A0C9805218018428F20
:108E6000120912010A4342870F998187418F11220B
:108E7000C9B2520211434187018F890B89030187CF
:108E8000A9781D4BCA07120E052100251A430A4373
:108E90004287018F4904490C0187656020680028DA
:108EA0000BD00E99416004464162F4F74EFC002855
:108EB00001D12034A57500200990099813B0F0BDA8
:108EC00010B50C20EFF3108472B60C490968002924
:108ED00002D0FFF751FD002084F3108810BD000080
:108EE000989200205555000000800020190F0000C6
:108EF000278000008083002020220000BC920020F8
:108F0000F8B5FC4980000C5826464036F08D00909C
:108F100000281DD0F848216E0289708E0F46101867
:108F20004143F648192278439202801A01F00CF866
:108F3000401E85B23946606E01F006F8401E85423B
:108F400000D22846009980B2884200D30846F085B6
:108F5000F8BDF8B50F46E74980000C580821F940E4
:108F6000E07D2346101A8033E54AC01E5043420874
:108F700094465A7B4820D04062460830101A5A88DE
:108F80001D7896381E46904200D310464822FA407B
:108F90000832801A4034E28F520601D58A00801AC6
:108FA00000F0D2FF854200D22846B071F8BDF8B576
:108FB000D04A8100555800902E468036B07B48221A
:108FC000C2407088B1880832884200D8084610181C
:108FD00095304000CA4900F0B7FFEA7D296E401C79
:108FE0008A1A101A801E2F4644084037F88FC0078F
:108FF00013D0C1487A8E008980184843192189010D
:1090000000F0A2FFBE49103000F09EFF241A388EF7
:10901000002802D0844200D30446009870214843BF
:10902000B84941180C80B74940394018C487708846
:10903000B18840184B214000C9004018A86528613C
:10904000F8BDFEB507468000AA4A019010580028D6
:109050004AD0064638020A46411CA948633801F046
:10906000F9F930462430009001F069F8344605469D
:1090700080341CE0207AA17A800040180006010D9F
:10908000A1480918488F8007800F012806D00228C0
:1090900004D0032802D1888F00F0EBFF207B04214D
:1090A000401E2073A07A401C00F04EFFA172207B6E
:1090B0000028DFD1308C002809D000F0DAFF06E06C
:1090C000A88800F0B5FF009801F039F80546002D9A
:1090D000F6D139460420F4F7A7FF304601F02AF90B
:1090E0008449019800220A50FEBDF8B50546814921
:1090F00080000C58824B264640362902B078643BEB
:10910000491C012804D002280DD0032824D10FE0E7
:109110000322184601F09EF92846FFF748FF226E09
:109120008034A17B15E00822184601F093F913E082
:109130000522184601F08EF9204620302746417C52
:1091400080377973007CB8732846FFF730FFB97B0E
:10915000226E2846FFF7FDFE0020B070F8BDF7B57F
:1091600088B008988C46810062483C27445800200B
:109170000590254600904035E88F666C810723D521
:10918000C00721D02146002080310874002A1BD05E
:10919000E88D002818D0EA8F530515D5530713D44E
:1091A000120711D4AA78002A04D0AA8E2B8812188C
:1091B0009A4209D2226E424392191601EA8E36096A
:1091C0001018E886012008740121C9066046801B3A
:1091D00000010009884207D2206E80190601E88E3E
:1091E0003609401CE886F1E7606D0190A8780128F7
:1091F00046D1204620300290C07F002840D1A88E62
:10920000E98E40182988401A81B24048814237D2FD
:109210000298807F002820D1208F80190601E88FD6
:109220003609C10704D0A18F490889190E013609F2
:10923000226B2266618FE985626B62660121029A68
:10924000C007917706D08820005DFFF759FEE88FB0
:10925000C00702D102990120C8770196A88EE98E35
:1092600040182988401A80B205E0226E0199891AB7
:109270000901090901910146401E80B20029F4D17B
:10928000E88F800701D5606E01E0206E80000390BA
:10929000C6E00296E88F0690C00764D000200490D4
:1092A0002A20285E0090E16C701A01011248090919
:1092B0000289688E101848431921890100F044FE84
:1092C000470006984037800705D401200490A88DF8
:1092D0000B494843C719A878012807D120462030F8
:1092E000817F002902D0C07F002811D00498002877
:1092F00013D018E0C09200209892002090D0030074
:10930000710200008081002080830020FF7F000028
:10931000A08FFD494843C71905E0FB49206E48432B
:109320004008B84270D979080491F749049800F0D0
:109330000BFE0299091A090109090291F2494843F1
:109340000499091A0098401A009008D50298EE492D
:10935000401E000100090290009840180090A06093
:10936000A06DC1192161029860602046F4F7EDF903
:10937000002860D0A07D401CA075206E80190601D9
:10938000E88E3609401C81B2E986A878012847D1C9
:10939000204620300290C07F002841D1A88E40187E
:1093A0002988401A81B2D948814239D20298807FF7
:1093B000002821D1208F80190601E88F3609C107C6
:1093C00004D0A18F490889190E013609226B226643
:1093D000618FE985626B6266C00703D08820005DFB
:1093E000FFF78EFD029901208877616E0391E98F66
:1093F000C90701D10299C8770196A88EE98E401855
:109400002988401A80B206E012E0226E0199891A7A
:109410000901090901910146401E80B20029F4D1D9
:109420000198301A010103980909814200D230E7FE
:10943000059800280CD00020892108556664E88F23
:10944000C00703D0009828853C37A7640BB0F0BD57
:10945000E88F800701D5082100E03E210898FFF73A
:10946000F0FDF3E7F0B5AA4980000D5887B0E86A2F
:10947000002808D1686AE862002804D0C088810505
:10948000890D7C2041532C464034E08FEE6AC006A3
:1094900009D5002E07D0A08F002802D130680028FF
:1094A00001D0012000E000200290298C014318D057
:1094B0002F468037387B042815D1F87A0421C01C48
:1094C00000F042FD387A800008180006010D91482E
:1094D0000818018FC90B04D1428F10218A430A4317
:1094E000428707B0F0BD04900428FAD2288C0028E7
:1094F00007D0698C039003200190009100202884FC
:109500002DE002980028ECD0A08F002808D1306808
:10951000002805D00646E862C0888005800DA08737
:10952000F088B1888205920D8A18A18F521A92B2E2
:1095300003928204920F012A00D002220192BA798A
:10954000914200D311460091032109038843012170
:1095500009034018F080A08F0099401AA087387A3C
:1095600082000292F87A1118C9B205910421C01C38
:1095700000F0EAFC029A8818C2B2E08FC10609D551
:10958000002E07D0A18F002902D13168002901D017
:10959000012100E000210291410603D50099091D37
:1095A00089B2009181040DD40299002908D1C00725
:1095B00008D00198032803D05748C07AC00701D0CB
:1095C000012000E00020059B00999C460902000153
:1095D000019B01431943634618014E4BC018418754
:1095E00003998187E18F890409D41101C9180A8F71
:1095F000D20B04D14B8F1022934313434B87018F1F
:109600004904490C0187F87A0421401C00F09CFCB5
:10961000F972387B401C38730498401CC0B262E772
:10962000FEB505007ED02E468036377A00202C46C7
:10963000403401970290A08EE18E4018A086019FD1
:1096400070214F433549791800910886E08FFF213A
:1096500001318843E087800516D5E08EF1794843D3
:10966000618F4018252100F06FFC08B2002801DA54
:10967000253000B2294AC1B2403ABB181A8D92096E
:1096800092010A431A8560870020E086E08FC007B8
:109690001BD0A86C2249401C400888420CD91A49AA
:1096A0004A1E801800F050FC0121C90301431B48E9
:1096B00040383818C18508E0C1030120C0030818EC
:1096C0001649000C40397918C885A178002941D085
:1096D000A08E2288801A0D4A80B290423AD2284643
:1096E000203002290CD1009A298E5180009A698E6F
:1096F00091800099027DCB885B095B011343CB808D
:10970000A17803291ED10EE071020000FF7F000046
:10971000C092002080830020989200208081002049
:10972000FF3F000029E0FF49427C7918CB8A0C27D3
:10973000BB4392001343CB82027CCB8A9B089B00E5
:109740001343CB82A178012902D1C07F002801D028
:10975000012002900020019B00901A46F249284601
:10976000F4F71AF9707A022801D001207072029879
:10977000002802D0307AFFF7B8FCFEBD10B5040017
:1097800015D000F0E9FF0146226E606C80180001E0
:109790000009606420464030C28E521CC286A07D03
:1097A0000022401CA0758034207AFFF7D8FC10BD41
:1097B000F1B500988100DD48445821468031487A4F
:1097C00000282AD125464035E88FC00725D0087CDF
:1097D000002822D0274600F0BFFF616C0646881B98
:1097E0000001216E0009884217D900213846F4F79C
:1097F000A5F8216E06E0401A000100096064E88EB9
:10980000401EE886606C821B120112098A42F2D85F
:10981000002231460098FFF7A2FCF8BDF3B587B0EF
:109820000798C24E8700F0590C250C4600287DD1C0
:109830000021942000F024FDF051002876D0074646
:109840000020029000F088FF059007989422049071
:10985000B74B002138469847B648F861B648B8611A
:109860000320F87500211020B960B8754002B88255
:109870003E46803607983D4630724035E88F4208B4
:1098800020785200002800D00120024301208002ED
:109890008243EA870020A886E88668872046203031
:1098A000039000798000A885608C8100F96520898B
:1098B000810039666089E885A0894101796603984D
:1098C0004079F071A07BF3F74FFC6886E88F102198
:1098D0000843E88700213173B172F1723984F9626B
:1098E000A9871B22FF21328049317180B180B2717A
:1098F00003998979717303998979B1730021F1739F
:10990000C00702D0307AFFF7FBFA217804980029CB
:109910007ED0032170225043824A03468018009073
:109920000190018203981121807900E0E6E00902AC
:109930008200114301430198C18204980102202052
:109940000143019841820198218AC1830198618A6B
:109950000184A17E607E090201430198418401983F
:10996000E17E828C120A12020A438284E07B002884
:1099700000D00120F1790122D2034003C90602433D
:10998000C80C024301980285664A002140329818AB
:1099900004900187E98F10158143E07B00286CD08B
:1099A000002040020143E987019906204885079875
:1099B000FFF7FDFA04997C20088104990020488172
:1099C0000146019A1E20D085049AA08A5080049AEC
:1099D000E08A9080049A207ED08001984187019887
:1099E000C28ED209D201C2860198828D52085200DD
:1099F000828500200190307A0199800004904018FF
:109A0000C0B20690481C042100F09EFA049800E0C1
:109A100031E0081801060A0D7721C90051188A089B
:109A20000121C90306981143020144481018018717
:109A30000021418781870198401C01900428DADBCE
:109A4000307A81017720C000081800998008888644
:109A5000EB8FD80713D00399E0698A79FF21593138
:109A6000D140228C083149005118354C89B28446C6
:109A7000624202910FE002214CE7012091E7E16987
:109A80000020F9646885E06913E00919401C89B277
:109A90000001000902919142F7D26146F9640299EE
:109AA0006985F96D001D0818A98D4908081800017D
:109AB0000009F96C396579657864D80700D0029897
:109AC000D90700B2288504D01D4AA98D52425143BE
:109AD00000E03C21B964D90700D10020B860002221
:109AE00005990798FFF73BFB00200090388A317AF0
:109AF00083B204203A6EF4F784FA0025284609B0B0
:109B0000F0BD70B505460C22EFF3108472B68300E9
:109B10000648C058002826D003468030427A002AE2
:109B200013D00FE040810020EBB70118C092002055
:109B3000750F00007D970118219601188083002081
:109B40008FFDFFFF012A0DD10AE0002908D0002176
:109B50001846F3F7F3FE16212846FFF772FA01E0E4
:109B600002214172002284F31088104670BD70B546
:109B700005460C20EFF3108472B6AE00ED4B9B59F6
:109B8000002B0DD01A8459844033D88F0821084304
:109B9000D8872846FFF766FC2846FFF709FE002015
:109BA00084F3108870BD70B505468400E2480C232C
:109BB000005900282FD040300278D24392072AD093
:109BC000CA88960522D0C678002E04D09E02B243E1
:109BD000CA800022C270EFF3108672B6D5480059D1
:109BE000002810D00446243000F08CFA2046403083
:109BF000C18F08221143C1872846FFF733FC28464E
:109C0000FFF7D6FD002386F3108804E09104890F46
:109C100001D10121C170184670BD70B506460C20F7
:109C2000EFF3108572B6B300C24AD258002A14D09E
:109C300014464032D08F102398430B011843D0872D
:109C4000002909D03046FFF70DFC8034207B002826
:109C500002D03046FFF7ACFD002085F3108870BDC0
:109C6000F0B504460C20EFF31086079F72B6A500EE
:109C7000B04C6459002C16D025464035A8780028F1
:109C80000DD10120A8702F808800A0879000208728
:109C90009800206305986087069840016063002063
:109CA0002034A077E07786F31088F0BD70B50C24DF
:109CB000EFF3108572B683009E48C05800280CD080
:109CC000034640339E78002E07D102249C701A80F0
:109CD00005229A4B30309847002485F3108820469F
:109CE00070BDF8B507460C20EFF3108672B6BD00C4
:109CF000904C6559002D0DD02C4680342280618017
:109D0000A3803846FFF753F9A17B38462A6EFFF748
:109D100020F9002086F31088F8BDF8B594460C278A
:109D2000EFF3108672B68400824A1459002C14D0C6
:109D300025464035AA78002A0FD10322AA702B802D
:109D4000224620321174634653748E22125D8A4279
:109D500002D9226EFFF7FDF8002786F310883846F7
:109D6000F8BD70B505460C20EFF3108472B6AB0059
:109D7000704AD358002B0AD004290BD08E20C05C27
:109D8000884203D91A6E2846FFF7E3F8002084F3CF
:109D9000108870BD1A6E8033997BF4E7014600206D
:109DA000EFF3108272B68B006249C958002901D0C6
:109DB0004031888E82F310887047F8B500259C46A4
:109DC0002E462C46EFF3108772B683005948C058D0
:109DD000002807D0034640339C8EDB8E466CE31888
:109DE000056E9CB287F310880123601ADB0398424A
:109DF00000DC081B910400B20C0C6843614680191A
:109E00004900401A00010009214600F09DF8601A3F
:109E1000A04200D100204A494843401C4010F8BDF0
:109E200010B5444A8300D258002A10D070235843FA
:109E3000444BC018438A0424A3438C002343438229
:109E40004032D08F4023984389010843D08710BD0A
:109E500010B5384A8300D258002A10D070235843D6
:109E6000384BC018438A0224A3434C002343438247
:109E70004032D08F2023984349010843D08710BD3A
:109E8000F0B52C4C8300E358002B2ED02D4F7023BF
:109E9000002458434037C3199C84DC841C855C85AE
:109EA0009C85DC85234615196E782D7836022E4365
:109EB0005D004519ED19AE83A41C5B1CDBB2E4B256
:109EC000042BF0D300220F23CC1825781D3C247FCF
:109ED0002D0225436CBA55004519ED19AC819B1E26
:109EE000521CD2B2DBB2082AEED3F0BD01460020EC
:109EF000EFF3108272B68B000E49C958002901D0C9
:109F00008F20085682F31088704710B50146002054
:109F1000EFF3108472B68A0006498958002906D0EA
:109F2000086D096E4008490800F00EF888B284F305
:109F3000108810BDC092002088920020190F0000E8
:109F4000710200004081002030B50B460146002020
:109F50002022012409E00D46D5409D4205D31D462F
:109F60009540491B2546954040191546521E002D27
:109F7000F1DC30BD70B500242546002801DA01244B
:109F80004042002901DA01254942FFF7DDFFAC42DA
:109F900000D04042002C00D0494270BD30B474461D
:109FA000641E2578641CAB4200D21D46635D5B00D5
:109FB000E31830BC1847000010B54B4C0021208836
:109FC00000280DD000F06FFB1F21081A2188C0B2B5
:109FD0000122824091432180DF21C001C900411844
:109FE000084610BDDF21C90010B5401AC109EFF3C2
:109FF000108072B63C4A138801248C40234313809E
:10A0000080F3108810BD10B5374C002061880029FE
:10A010000DD0084600F047FB1F21081A6188C0B226
:10A020000122824091436180C0000019183010BDA8
:10A030002E492D4A40185188C009012383401943F5
:10A040005180704710B5284C0021A08800280ED000
:10A0500000F029FB1F21081AA188C0B2012282400A
:10A060009143A180182148439721C900411808460F
:10A0700010BD972210B5D2001821801AFFF764FF97
:10A0800019498A88012383401A438A8010BD10B57C
:10A09000154C0021E08800280FD000F004FB1F21A0
:10A0A000081AE188C0B2012282409143E180820017
:10A0B000002112195181401CC1B2084610BD0A4945
:10A0C00080004018001D704759210901884202D3C1
:10A0D000401A800900E0401E034AD18801238340D2
:10A0E0001943D180704700000890002008F4FFFF5A
:10A0F00001460020096802E00968401C80B200297E
:10A10000FAD170470268002A05D0426811604160A8
:10A110000020086070470160F9E70368002B05D054
:10A120004368196042600020106070470160F9E7E1
:10A130000268002A00D141600A600160704702464F
:10A140000068002804D001681160002900D1516026
:10A15000704710B500242346026805E08A4201D109
:10A16000012405E013461268002AF7D1002C07D01D
:10A170000A68002B06D01A6042688A4200D1436008
:10A18000204610BD0260F7E7002906D013680B6077
:10A190004368934200D14160704703681B680360C5
:10A1A000F6E71368002905D00B604368934200D19D
:10A1B000416070470360F8E7F7B50F460646002593
:10A1C000046814E020460299B84700280DD02068A2
:10A1D000002D01D0286000E030602068002802D007
:10A1E0000020206005E0756003E025462468002C0F
:10A1F000E8D12046FEBD10B40C000ED0002301684B
:10A2000001E00B460968A14201D00029F9D1002BD9
:10A2100003D01A60116010BC704710BC114687E76C
:10A220000B000DD0016800E00968994202D00029B6
:10A23000FAD105E0002903D00B68002B02D002E020
:10A2400011465FE74260086810600A607047F7B522
:10A2500004680E4607460025002C08D0029A2146C5
:10A2600030469047002803D125462468F4E77E60F5
:10A270003460002D01D02E60FEBD3E60FEBD0000AA
:10A28000F3B5C01C00248508AD002D1D81B0264605
:10A2900027460C2D00D20C25EFF31080009072B6EB
:10A2A000029802213018FFF74FFE0806810D4F4833
:10A2B0002A46081880690C320EE04188A9420AD368
:10A2C000914202D28368002B05D0002C02D0638813
:10A2D0008B4200D9044640680028EED1002C03D000
:10A2E0006088904200D20546761CF6B2022E02D259
:10A2F000002CD5D001E0002C0BD06088A8420CD1F6
:10A30000A16860684860606800280AD0A168816020
:10A3100007E03748F2F79CFE07E0401B80B2608000
:10A320000419658033482080271D009880F3108829
:10A330003846FEBDF0B50023021F2F491180548816
:10A340001946EFF31085AC4672B69D00274E5F00AC
:10A35000AD19AD69BE19368CA84204D3AE19864238
:10A3600001D3294601E05B1CDBB2022B01D200299C
:10A37000EBD00020214B2DE04D886D18954211D176
:10A380004888001982B24A8048685318984228D1F8
:10A390004388D2184A8042684A604068002820D02A
:10A3A00081601EE08A4213D24260906010191380CF
:10A3B000884209D1486850604868002800D082600F
:10A3C0004888001950800CE051608A60548008E091
:10A3D000084649680029CFD142605160906054809E
:10A3E0001380604680F31088F0BD0000509000207C
:10A3F000F2F2F2F2388300000FF000005AA50000DC
:10A40000F8B504460F4618461D46164601210C3085
:10A41000FFF736FF0021C94301608480C7800681B1
:10A4200045810C30114B04462A46002198472046AE
:10A43000F8BD10B501460C39EFF3108472B60C4824
:10A44000FFF760FE0B48016808221143016084F3A6
:10A45000108810BD10B50023FFF7D2FFFFF7E9FF0A
:10A4600010BD03460C3BD9801A81E2E7750F00004E
:10A470005090002094900020F8B50C460746010A41
:10A48000C0B2082822D21A4A8000125800209047F1
:10A4900000281BD00178A14218D004701548164D31
:10A4A000082600903A4615490098FFF785FE0100FE
:10A4B0000CD0EFF3108472B60E480838FFF722FE76
:10A4C00028683043286084F31088EBE7F8BD10B5A6
:10A4D000010AC0B2FF24082807D2054A800012589A
:10A4E00000209047002800D00478204610BD0000CE
:10A4F000749000205890002094900020A9D000185B
:10A50000F0B50746414885B015460E46824201D94E
:10A51000054602E0002D00D10A253A043D483243A9
:10A520003B490490FFF748FE040006D101211020AA
:10A53000FFF7A6FE87800446C680EFF3108672B64A
:10A5400002A800F014F986F31088029800907D208C
:10A550000399000145436D1801912F492846FFF7E3
:10A56000F3FC2D492D4A4143691AE160009908180E
:10A5700000010009A06021460498FFF768FE254805
:10A5800010380069A04203D1C168806800F029F941
:10A59000E168A068F2F79CFD002802D0042000F0DA
:10A5A0003FF805B0F0BD70B51A4C0246103C256965
:10A5B000002D29D0AB88174893421AD1EB888B42E3
:10A5C00017D1FFF7BCFD2469002C0DD0E168A0680D
:10A5D00000F007F9E168A068F2F77AFD00280ED0D4
:10A5E000042000F01DF80AE00021481E00F0F9F8F0
:10A5F00005E012040A430649FFF7DEFD0546002D7B
:10A6000002D02846FFF796FE70BD0000FFFF7F02D4
:10A610003BD10018609000207102000013D1001897
:10A6200010B5EFF3108172B60A4B1A68012484400A
:10A6300022431A6081F3108810BD10B5EFF310812A
:10A6400072B6044B1A6801248440A2431A6081F355
:10A65000108810BD94900020410855221140401AE6
:10A660000246332180080A400840101801090818E2
:10A670000007000F70472021020401D0102110466E
:10A68000020201D010460839020101D01046091F0C
:10A69000820001D01046891E420001D01046491E9A
:10A6A000C00F081A70472021020C01D0102110465B
:10A6B000020A01D010460839020901D01046091FCC
:10A6C000820801D01046891E420801D0881E7047BA
:10A6D000081A70470021425C002A01D00020704710
:10A6E000491C0629F7DB0120704710B50022835C66
:10A6F0008C5CA34201D0002010BD521C062AF6DB60
:10A70000012010BD0549064A08685043054A8018D3
:10A71000086040087047014908607047D8920020DF
:10A720006D4EC64187D612000A49002804D04869F8
:10A730004004400E1830704708694004400E28302D
:10A740007047002902D080002C307047C000503084
:10A75000704700008000005001200D49C007886349
:10A76000886BC00FFCD1886B000100097047012184
:10A77000074AC9079163916BC90FFCD1916BD26BEA
:10A780000901090927231B019A1A06C07047000016
:10A79000C00000500521431C10220907002B06D0E1
:10A7A000694B58620A6288699043104301E08869E6
:10A7B00090438861704710B50522441C202312077E
:10A7C000002C0AD027242401611A5F4CA062E162A8
:10A7D000136290699843184301E09069984390612F
:10A7E00010BD30B5EFF3108472B6451C052240232E
:10A7F0001207002D0AD027252D01691A524D286312
:10A800006963136290699843184301E09069984323
:10A81000906184F3108830BDF0B50020844601209B
:10A82000494EC007B063B06BC00FFCD1B06B0501DF
:10A8300046482D090088002845D145480068002871
:10A8400041D10121C906002205200007836970203B
:10A85000034038D03F4FD80609D5706A401B040129
:10A860002409A01EB8422ED28C4200D2214698065E
:10A870000DD5B06A401B04012409A01EB84222D2A3
:10A880008C4204D2F06A214627221201121A58067D
:10A8900012D5306B401B00010009831EBB4212D24F
:10A8A000884209D8736B27242401E31A884201D314
:10A8B000934201D201461A46F06B80180A228009A1
:10A8C0005143401884466046F0BD7FB504461020D1
:10A8D000EFF3108272B61D4B1D8805431D8082F375
:10A8E00010881E4E1C481D4D5C36002902D01022D7
:10A8F000A84702E010220021B047002C04D010220B
:10A9000021466846A84703E0102200216846B04768
:10A910000D48009940384163019981630299C163F0
:10A92000094A039911604C21516004210522120744
:10A93000116293698B430B439361026B01218A433C
:10A940000A4302637FBD0000C00000500090002059
:10A9500094900020FFFFFF0730810020190F0000B6
:10A960001FB50220FFF769FE054B68461022034918
:10A97000984769460020F2F781FC1FBD4081002006
:10A98000190F000070B5EFF3108572B62048FFF77D
:10A99000D6FB040002D00020C043206085F310885D
:10A9A000002C26D020464038808F1A49884220D17A
:10A9B000E088194B010A0006A288800D1B5810463A
:10A9C0009847051E05D021460C312389E288A088CE
:10A9D000A847002804D001280BD0022809D103E0A1
:10A9E0002046FFF7A7FC04E0094821460830FFF79E
:10A9F00089FBEFF3108072B605490968002904D17C
:10AA000006490A6808239A430A6080F3108870BDDB
:10AA10005090002038830000749000209490002013
:10AA20007FB51C4D0420FFF708FE2C69002C30D0A8
:10AA3000EFF3108672B66846FFF799FE86F310882A
:10AA400001990098039102900146A0680122411AE1
:10AA5000C91E09010909D20691420CD2E168FFF72B
:10AA6000C0FEE168A068F2F733FB002811D0002196
:10AA7000481EFFF7B6FE07481030FFF760FB04469C
:10AA8000C1888088FF22FFF7E5FC2046FFF752FCD3
:10AA9000C8E77FBD50900020F8B50620FFF7CDFD38
:10AAA000104E3588002D1BD0002401270CE03846BD
:10AAB000A040284204D07088C1B22046F7F7A7F81A
:10AAC000641CE4B2032C02D270880028EFD13088D5
:10AAD000002805D07088002802D00620FFF7A0FDCE
:10AAE000F8BD0000F4910020F1B590B0109800245A
:10AAF00080000B90E2E0E8481C21807A4843E74957
:10AB00004518688A3D21084206D1A88A0107090F25
:10AB1000052902D0032971D0CEE0A88CE049222279
:10AB20004118E04E6846B0476846428BDE49104601
:10AB30000A388842F0D86846C18A0629ECD3192021
:10AB4000C0018142E8D86846008BFF23F433984265
:10AB5000E2D8401C484391008842DDD2A88A694669
:10AB60004006C00F0D90062209A83346984709A851
:10AB70000D99F9F75BFC0028CED12C23FF22002190
:10AB8000CA48FFF73DFC0746041D688B298B00046B
:10AB90000843A98B272289050C90890D1201E88AA8
:10ABA000561A800BFFF7C0FD4000301ABF4906B2AD
:10ABB0006B3106E0701806B20C98401E00010009C7
:10ABC0000C90002EF6DB1098387000207870012071
:10ABD000F8702070B6490B980858808EC00603D5CF
:10ABE000A88A8006C00F00D00120E0730B98085897
:10ABF000018F002903D02030807E01E042E0002058
:10AC0000B87004222046A74B103003A998470322AE
:10AC10002046A44B193004A998476846C17C2046B9
:10AC200020300E9001716846808A60846846C08A30
:10AC300020816846008B60816846408BA081052298
:10AC40002046984B143007A9984708A84078062258
:10AC5000C1060E98C90E417108A84078914B400971
:10AC6000A07309A9A01C98470D9860700C98E0612A
:10AC70002684E88A810B0E9881713846FFF7D9FB4C
:10AC8000012419E08A490B9808582030407F002899
:10AC900012D0A88C82490C224118824E6846B047D7
:10ACA000A88A69464006C50F062203A8B04703AA32
:10ACB00029461098F4F75DFCFDF756F81098FDF75B
:10ACC0006BF8002800D016E7204611B0F0BDFEB5A5
:10ACD000064677488B00C458002C41D00027002A34
:10ACE00016D0012A14D0022A3AD0042A38D1254697
:10ACF00008462035297F02297CD001212046F2F721
:10AD00001DFEA08E000776D5A07D401CA075B3E087
:10AD10000091019201212046F2F710FE25462035D0
:10AD2000A87E401CC0B2A876297F022904D0218FBA
:10AD300000290BD0884209D3218F002903D08842F3
:10AD400001D3432200E00022012106E0E87EFFF764
:10AD5000CBFE002805D0002211460098FDF76AF8C6
:10AD6000FEBDA08E400711D42A78002A05D0012309
:10AD700000210098FDF790F82F706A78002A05D01E
:10AD8000012319460098FDF787F86F70A08E494996
:10AD90000007019813D5002802D0A07D401C00E0D8
:10ADA0000A20A075A182606A6660E0602046F2F722
:10ADB000CCFC002801D12F77FEBD3C22C4E700283F
:10ADC0001AD0A06A301A0201E06A120940008242D9
:10ADD00002D3A07D401CA075A662E87F002802D0A7
:10ADE0006068B04202D0606A401C08D0A182616AEB
:10ADF000E16006E031E032E00522A275ECE72E4981
:10AE0000A182FFF77FFC1121FFF79EF84804E97F3C
:10AE1000000C002907D0002802D0202802D002E030
:10AE2000012000E01F20E16A49008919081801018A
:10AE3000090920466160F2F788FC0028BBD0E87F52
:10AE4000002803D00021C94361602F77606A411C4C
:10AE5000B2D0E1688142B0D0FEBD002219E0A06A04
:10AE6000301A0101E06A09094000814204D3A07D43
:10AE7000401CA0756168A1622046F2F766FC0028BC
:10AE800099D0E87F0028E7D1606A401CE4D0E87ED2
:10AE90003C22012162E700009892002000830020FC
:10AEA00000800020190F0000760C00000602000050
:10AEB000A892002001A0000001600000F0B5810010
:10AEC000B54889B0006841580591407A8006000E67
:10AED000203103910890D8E0B0481C21807A484383
:10AEE000AF494518A88C00900598AE4A408E904214
:10AEF0007ED8688A3D220290104001D0102877D178
:10AF00000020059C01903E3406900490FF27039892
:10AF1000012207944277A88A0607360F072E44D2EB
:10AF20000027042E0CD1A04900984018211DFFF7DE
:10AF3000DCFB002812D00398407E062811D01B2786
:10AF400024229A4B002120469847012E0BD0002E38
:10AF500011D0022E11D0062E11D011E0FF20A075C5
:10AF60008FE01A27ECE7A88A15270006C00F207685
:10AF7000062001900BE0132702E0102700E01227C3
:10AF800006200690A88A000A801FC0B20490002004
:10AF9000A075677560760421A176A0747F20E076A5
:10AFA000A88A4006C70FE77502E0A07DFF2868D099
:10AFB0000298C00607D5607D4007CFD57648006867
:10AFC000407C0128CAD9607D15281ED1019A0099BC
:10AFD000754B891889B2C9182046744B0A3006226D
:10AFE0005C3B9847688A4006C00F00D0012000E013
:10AFF00049E06070688A4006C00F06D1207E0028B4
:10B00000ACD0E07B80090328A8D0FF2F12D066497E
:10B010000098231D41181846644B06225C3B984754
:10B0200002980006C00F2070288C60800298C0062D
:10B03000C00FE0742423FF2200215D48FFF7E0F9F0
:10B040000746E88A2077594B242238465C3B07990B
:10B05000984704987877049800280BD00098388493
:10B060000698B8774D481C22807A002150434C4AFC
:10B070008018818448480068407A38753846FFF760
:10B08000D8F903984676FCF76FFE0398007DFCF72D
:10B0900083FE002800D01FE7089801014048803057
:10B0A0000818018FC90B03D0018F4904490C01878F
:10B0B00009B0F0BDF8B5044637480068002832D022
:10B0C0008B00C05800282ED00027002A13D0012A58
:10B0D00011D0022A46D0042A25D10446FFF73CFBB2
:10B0E000214605462031087E02283FD000200F76F9
:10B0F000002816D13CE01646024620300091017E21
:10B10000057D022904D000210776002904D10BE037
:10B110000121F9E7FCF728FE2846FCF73DFE002850
:10B12000F8D1FDF733F9F8BD01211046F2F706FC1E
:10B13000702045431F482818418D4905C90F04D088
:10B14000418D01229202914341850098FFF7B6FE9E
:10B15000002E01D0012200E0002221460098FDF7D8
:10B160005AF9F8BD0846FFF7A9FEF8BD0120BEE771
:10B1700001212046F2F7E2FB606A281A0101A08D46
:10B1800009094000814203D3A07D401CA07565627F
:10B190002046F2F7DAFAF8BDB89200209892002023
:10B1A000008300207206000000800020750F000060
:10B1B0000102000040810020F0B58100CB4887B03B
:10B1C0000568685802902030019060E0C8481C2152
:10B1D000807A4843C7494418608A3D21084253D1C8
:10B1E0002E462036307E00284ED1A08AA18C000742
:10B1F000000F05910121019A0028917501D00128C5
:10B2000042D1A08AE18A000A890B0091618B0A046D
:10B21000218B0A430492A18B27228905890D1201F3
:10B22000511A22300391C0B20099FFF78AFA0746FB
:10B230000098FFF779FA381A039940004018AE4990
:10B24000FF304A1E2D308018FEF77EFE049A8018CB
:10B2500000010009E863208CA886A08A8006C00F40
:10B2600000D00120402148550098B075A34B0599A6
:10B270000298C9180622A24B2E309847A08A400691
:10B28000C00FE87601203076FCF76EFD0198007E55
:10B29000FCF782FD002899D107B0F0BDF0B5810020
:10B2A000924889B0056868580690287D2F46800628
:10B2B000000E20370590387E00287DD005980101CA
:10B2C0008C4880300818008FC00B75D041202C238B
:10B2D000FF220021C000FFF793F80490041D069898
:10B2E000B97D0A2220305143007E4E197021484317
:10B2F00084494018808C80000790E86B0190708929
:10B3000041000198401A3189000189000009029129
:10B3100008360391FEF718FE08460399091A0198AA
:10B3200008180101090901980091081A01010798FC
:10B330000909814205D200990298401800010009CC
:10B34000009000202070E87E0622C007C00F6070C9
:10B350000699A01C6A4B2E319847294604221C31BD
:10B360002046674B10309847308820817088608471
:10B370002946052215312046614B14309847049820
:10B38000317A41702046B97D203001908171B088BA
:10B390006081F088A08103222046594B394619303C
:10B3A00098470198F9780171019839794171787954
:10B3B000A0730098E06100E00DE04020405DE07384
:10B3C00004980121C1700498297D01700498686077
:10B3D000FDF7D2FA01E000203876059801014548D2
:10B3E00080300818018F4904490C018709B0F0BD6D
:10B3F000FEB53E4B05461868002833D08C00005936
:10B4000000282FD00027002A13D0012A11D0022AA9
:10B4100052D0042A26D10446FFF79EF9214605465C
:10B420002031487B02284BD000204F73002817D1D1
:10B4300048E016460246203000950191417B057E8A
:10B44000022904D000214773002904D10BE0012117
:10B45000F9E7FCF789FC2846FCF79EFC0028F8D1A8
:10B46000FDF78AFAFEBD01211046F2F767FA702057
:10B470004543244840382818418D4905C90F04D058
:10B48000418D01229202914341850198FFF794FE7C
:10B490000198FFF703FF154800680028E2D0005923
:10B4A0000028DFD0002E01D0012200E00022009908
:10B4B0000198FDF7A8FAFEBD0846FFF77DFEFEBD28
:10B4C0000120B2E701212046F2F738FA606A281A13
:10B4D0000101208D09094000814203D3A07D401C59
:10B4E000A07565622046F2F730F9FEBDBC920020DF
:10B4F000989200200083002071020000008000204C
:10B50000190F000080810020F1B582B00298F14946
:10B51000800001900D582C468034207AA17A80005A
:10B5200040180299C0B20902009155E0708FB18FA6
:10B530008007800F012816D0022814D003283AD1A2
:10B540000846FEF796FDE4490198029B085800283A
:10B5500006D0006A4268002A02D0417A1846904715
:10B560000322009922E0708F000A042805D97E2268
:10B57000525B520601D5001F80B200281BD06F6AB3
:10B580000818FA88B9889205920D8918884212D352
:10B5900028462430FEF7D3FDE86AB84201D10020E6
:10B5A000E862B888FEF744FD0099022283208000FB
:10B5B000491CFEF74FFF708F102188437087207B56
:10B5C0000421401E2073A07A401CFEF7BDFCA1722E
:10B5D000207A80004018C0B2217B002905D00101EB
:10B5E000BE480E18308FC00BA0D14035E98F08201F
:10B5F0008143207B002800D00120C0000143E9875F
:10B60000FEBDF1B588B00898B24980000C580421FD
:10B6100025464035E88F8843E88708980002029065
:10B62000DBE0AF491C22887A5043AC4A803A80184C
:10B630000090478A828A01929207920F0392C28AEF
:10B640000026D2B20692226D0592FA070BD0A54AC7
:10B650001078401CC0B21070042803D3086800287A
:10B6600000D08047B4E09F4900220A70E98FCA07E2
:10B6700004D0428B008B16040643E664C80570D4E0
:10B68000FF2001300143E987C8070CD0A8780128C2
:10B6900009D120462030817F002904D00121C177C3
:10B6A0000898FDF722FDA88E2887E88FC00711D0E3
:10B6B0000098808B27218005800D0901081A0490CD
:10B6C0008D20005DFFF730F841000498401A00B269
:10B6D000854908E0606CE064206509E04018761E4A
:10B6E000360100B236090028F8DB688566642665F5
:10B6F000E88F810707D402210843C207E887D20FE9
:10B700000223029911E0C0071FD0206D410805985F
:10B710004008081A216E000100094908FEF714FCD0
:10B72000002912D002230299FF226F48491C623877
:10B73000FEF766FE0646206D216E40084908FEF7BA
:10B7400003FC31803046FEF774FEE88F410508D4D3
:10B75000810706D50199490703D5012189020843CC
:10B76000E887380734D4E06C66210F4260652FD13A
:10B77000F80607D5E88F80210843E8870220892151
:10B78000085525E00198060A22D0039800281FD00A
:10B79000042E04D9E88F800601D5361FB6B2009872
:10B7A000878C514802990823FF226638491CFEF70E
:10B7B00027FE0780468003990171A98EC180FEF79C
:10B7C00038FEE88F04210843E88700990020888428
:10B7D0008F2106980855FCF7C7FA0898FCF7DCFAA1
:10B7E000002800D01DE709B0F0BDF8B50F46394874
:10B7F00089004458002C3BD01300FEF7CFFB050412
:10B80000043C40473900154601212046F2F796F8DE
:10B810008920005D022823D0FEF79EFF01462046C6
:10B820004030C28F930724D5530722D4120720D467
:10B830008278012A1DD00E22266E636C9B191B0193
:10B840001B096364C38E26465B1CC386002D01D092
:10B85000A27D521CB275C08FC005C20F384633E0BE
:10B860004034E08F000632D53D213846FDF7E9FB34
:10B87000F8BD1022E0E73846FFF7C3FEF8BD3846B2
:10B88000FFF742FE3846FDF7EDFDF8BDFEF764FF19
:10B89000054601212046F2F751F820468030014646
:10B8A000407A022813D0626C206E1018020112092F
:10B8B000204640306264C28E521CC286A07D0022A7
:10B8C000401CA075087A2946FDF749FCF8BD1621F1
:10B8D000CBE70000C09200208892002080830020E7
:10B8E00098920020EB92002071020000F8B5052527
:10B8F0002D07EC69534EA00726D502202862A96BBC
:10B90000514C3E206268521853085F00D21B4143DD
:10B91000CF184E4938466260FEF716FB4C49064385
:10B920004E604A4A5043381A521E101A08600B20C3
:10B9300028630120A861801E286221880820014315
:10B94000042081432180F8BDE00737D00120286220
:10B950000020A8613F49E9603D4B80339E63996BAD
:10B96000C90FFCD1996B3C4E0A013749120949882D
:10B97000CF0607D55F6AD71B3F013F09B74201D207
:10B98000102738438F0607D59F6AD71B3F013F0911
:10B99000B74201D2202738434F0607D51B6BD21A76
:10B9A00012011209B24201D240221043264A8143B9
:10B9B000A961138808218B4313800443E00606D550
:10B9C00010202862A9698143A96100F01FF9A0062F
:10B9D00006D520202862A9698143A96100F040F8BA
:10B9E000200404D500F08EF80120C00328621B4912
:10B9F000600608D540202862AA698243AA610868C7
:10BA000010221043086060070CD504202862AA6940
:10BA10008243AA610C4A13881026B34313800A6834
:10BA200002430A60200706D508212962A8698843D5
:10BA3000A86100F057F82869C00384D501200004EC
:10BA40006861F8BD000000800090002071020000D5
:10BA5000400000501E0001000000000894900020EB
:10BA6000FEB5274D68462C68FEF781FE0126F606D6
:10BA70002F460C3716E0E17D6068401A0099401AA5
:10BA8000401C00010009B04224D200281ED0022828
:10BA90000AD81B48FEF753FBA8608169002900D033
:10BAA00088472C68002CE6D1386800280BD0082184
:10BAB00005200007016282698A430A4382610168A6
:10BAC000B14331430160F1F710FEFEBD0198A1685A
:10BAD0008842DED90A48FEF732FB01463846FEF7B7
:10BAE00011FBDEE710B5064C0C342046FEF727FBB1
:10BAF000002804D0C1690029F7D08847F5E710BDB8
:10BB0000BC900020F8B505200007416A0801040F29
:10BB10000E0F3B480A0701D5032202E0CA060BD5E7
:10BB20000222A5004359002B05D0011980312818A5
:10BB30000978006C9847F8BD314D4A07314B012711
:10BB40008035002A31DA298AB74039421BD03201C8
:10BB5000D11809888906490F062914D1B400035960
:10BB60000422002B05D08119803120180978006C3F
:10BB70009847A87CB04203D1401C0007000FA8746E
:10BB8000288AB8432882288A002808D0411E084203
:10BB9000D1D1A87C401C0007000FE874F8BD1A48FA
:10BBA0000188202291430180F8BD8907FCD522013C
:10BBB000D11809888906490F042911D00022A6004E
:10BBC0008359002B05D00119803130180978006C99
:10BBD0009847288A3946A14088432882E97C04E0B6
:10BBE0000122ECE7641C2407240F3A46A2401042CD
:10BBF00001D1A142F6D1AC740028D0D0F8BD00002C
:10BC0000D09000200080002000900020F8B501278F
:10BC100000250E4EFF06FEF79FFD3468002C12D063
:10BC20006168401A00010009B8420CD20748FEF7CB
:10BC300086FAA168002901D020468847002DEAD065
:10BC4000F2F702F9F8BD002CFAD1F8BD709100208E
:10BC50000246002000290FD1002A0ED035235B01B7
:10BC6000D11A9A4213D00ADC0C49511813D0122968
:10BC70000BD09E2900D10A4870470A487047062910
:10BC800007D05229FAD10848704708487047084839
:10BC9000704708487047084870470000FFF9FFFFE9
:10BCA000B1F20018DD920020F9FA0018E1EE001858
:10BCB0005DF10018A5F40018B1EC00180246002050
:10BCC00003290FD2002A0ED0104BD11A9A4219D054
:10BCD0000CDC0F49511813D00E4A89180ED00929CF
:10BCE00000D10D4870470D4840187047E0290BD02F
:10BCF000E12901D0E229F8D1094870470948704785
:10BD00000948704709487047094870471207000002
:10BD1000F9FBFFFF02FDFFFFBBE30018DE920020EE
:10BD20001D170118F1E10018CFE200189315011852
:10BD3000FFE2001802460020032910D2002A0FD08B
:10BD400051231B01D11A9A421BD00CDC0E49511809
:10BD500011D0FA2911D0FF39082900D10B487047BA
:10BD60000B4840187047012909D0302901D03129EA
:10BD7000F8D1084870470848704708487047084895
:10BD80007047084870470000F9FBFFFFA5E700185F
:10BD9000E192002001E900185DE90018FFE40018B5
:10BDA00005E80018BDE700180246002003290AD262
:10BDB000002A09D00849511809D0FF39FC3908D0A8
:10BDC000012900D1054870470548401870470548CB
:10BDD0007047054870470000F5FDFFFFD3EA0018E3
:10BDE000E492002033EA0018C9E9001801460D4B1F
:10BDF0000020CA1A994210D007DC03290FD0FF395E
:10BE0000FF39032900D108487047012A03D0032ACB
:10BE1000FAD10648704706487047064870470648FA
:10BE20007047000005020000954A01186B4E01188A
:10BE300037480118C54C01186D4A01180246002008
:10BE4000042912D2002A11D083239B00D11A9A42CE
:10BE500017D00EDCFF3A521E1BD0012A19D0062A39
:10BE600015D0FF3A0C2A00D10B4870470B484018F8
:10BE70007047012909D0022905D00329F8D10848C3
:10BE80007047084870470848704708487047084896
:10BE90007047084870470000ED530118E7920020F2
:10BEA000AF740118435401188B570118CD52011873
:10BEB0004B5201185D53011870B5064600F01AF98F
:10BEC000304600F07DF9304600F0A8F9304600F029
:10BED00047F8304600F088FA304600F0D7F90524DC
:10BEE0001A4D2407002E14D0304600F0AFF800F0B1
:10BEF000C5F8206840004008E10008432060206841
:10BF0000C00FFCD1134912480862002028806860E5
:10BF100070BD11490220F1F71DF91048A061012000
:10BF2000288070BD70B509480088C00701D0012481
:10BF300000E00224EFF3108572B600F05DF82046B1
:10BF4000FFF7BAFF85F3108870BD00000090002055
:10BF5000C8002C01C000005061A901180C8000002D
:10BF600010B51149002808D0104808803F204880AB
:10BF7000FF2088800F20C88010BD0D4B0020C2011B
:10BF8000C400D2186418401CA2830628F7D30020EE
:10BF900059231B0182018400D2186418401C22819D
:10BFA0000428F7D310BD000008900020FF03000014
:10BFB000F80B000070B5054624221F4C00211D48D7
:10BFC000A047202200211D48A047202200211C4814
:10BFD000A0471B481B4901611B4900244161A00087
:10BFE0002A586000401901892046F1F73FF8641C87
:10BFF000E4B2022CF3D370BD10B50E48FEF79FF8E3
:10C00000002802D0FEF796F9F7E70A4C08342046DC
:10C01000FEF795F8002802D0FEF78CF9F7E7054CFB
:10C0200010342046FEF78BF8002802D0FEF782F984
:10C03000F7E710BD50900020750F000074900020AD
:10C040009490002085A9011821AA011810B5094C67
:10C05000022808D12068002805D00648FEF76FF8AE
:10C06000FEF768F9F6E70020206003496060087079
:10C0700010BD0000B4900020DC92002070B51422A6
:10C08000144C00211248A047942200211248A047D6
:10C090000020124A05461A2103019B181980401CF2
:10C0A000C0B21028F8D30E482022056045600D4824
:10C0B0000021056045600C48A04700210A48C9439B
:10C0C00001600A4801600A498180857170BD0000E5
:10C0D000BC900020750F0000D09000200080002050
:10C0E000649100207091002078910020D09200206F
:10C0F000E457000070B505001BD0012D11D0022DB2
:10C1000016D100242046F2F728FD641CE4B2022C6C
:10C11000F8D300242046F3F7E2FD641CE4B2032CBC
:10C12000F8D3284600F030F800210620FEF7A4F9E5
:10C1300070BD0E490620F0F7BEFF00240C480E4BE0
:10C140000470282221460B4898470C490720F0F735
:10C15000B2FF00200A4A0B4B3F2111548500401CBE
:10C16000C0B25C510328F8D370BD000051BC011867
:10C17000DD92002098910020750F0000BDBC0118D1
:10C18000DE920020C091002010B502280BD01022B2
:10C190000A4B00210848984707480421183041718C
:10C1A000C171817110BD00242046F3F7BDF8641CF5
:10C1B000E4B2042CF8D3EFE7A0910020750F000043
:10C1C00070B5002400280ED001281CD0022809D107
:10C1D000F6F7D2FA00212046F5F7FCFB641CE4B226
:10C1E000032CF7D370BD09490520F0F764FF002048
:10C1F000074A084B102111548500401CC0B25C5105
:10C200000328F8D370BD0448046070BD35BD011823
:10C21000E1920020E8910020CC91002070B500252B
:10C22000002814D001280DD002280FD10620FEF7D7
:10C2300004FA002401212046F5F7B3FC641CE4B2A3
:10C24000032CF7D30C4805800621418070BD0B49B3
:10C250000620F0F77FFF0A490420F0F72CFF0020AA
:10C26000084A094B3F2111548400401CC0B21D51A3
:10C270000328F8D370BD0000F491002099AA01189A
:10C28000A9BD0118E4920020F891002070B51D4D61
:10C29000002829D0012817D0022824D11A4E0024C2
:10C2A00001212046F8F753FE1C20604380190069E5
:10C2B000002801D0FEF73EF8641CE4B2042CEFD352
:10C2C00000210420FEF76FF90324842200210E4888
:10C2D000A8470D481B2140308187FF214931C18784
:10C2E00040300470447070BD08490020F0F7E3FE50
:10C2F00007490120F0F7DFFE102200210548A8477A
:10C3000070BD0000750F000004920020EDBD011803
:10C310003DBE011888920020F8B5FF25052401359F
:10C320002407022814D12068A84320602068400018
:10C330004008E100084320602068C00FFCD1E060A5
:10C34000401E60613349086901221203904308616D
:10C35000314820603148E0602E4931484031086260
:10C360000026701C0621FDF7EFFD1C204143312003
:10C37000000108188003010C1C2032464243294862
:10C3800017183982FDF718FEB884761C062EE8DBF4
:10C39000C420A0620020E062234E1F231B027021F4
:10C3A000414389194A8A07029A433A434A82401C08
:10C3B0000428F4DB2068A84328432060F8BD10B5AA
:10C3C00010221B4B002119489847FF20174CF530CD
:10C3D00020811848A0801848E080FEF793F9207368
:10C3E00016490020087010BD10B5040010D0FFF7EA
:10C3F000E6FF2046FFF790FF204600F021F8204698
:10C4000000F038F8204600F049F8204600F062F8C5
:10C4100010BD0000C00000500F0610001E000100FB
:10C42000D902FFFF00830020408100209892002065
:10C43000750F0000D6BE0000898E0000EB92002030
:10C4400070B50B4D02280AD10324A00028580028FB
:10C4500001D0FDF76FFF641E64B2002CF5DA0020F6
:10C4600001468200401CC0B2A9500428F9D370BD17
:10C47000A892002010B5084C02280AD12068002894
:10C4800007D00068002801D0FDF754FF2068FDF7B1
:10C4900051FF0020206010BDB892002010B50C4C58
:10C4A000022811D1206800280ED04068002802D050
:10C4B0000C38FDF73FFF20680068002801D0FDF729
:10C4C00039FF2068FDF736FF0020206010BD000016
:10C4D000BC92002070B50E4E02280FD10024A5009A
:10C4E0007059002806D021460420F1F79DFD7059AF
:10C4F000FDF720FF641CE4B2042CF0D300200146B9
:10C500008200401CC0B2B1500428F9D370BD0000B5
:10C51000C09200200D0D0118C70D0118B50E0118AD
:10C520000D0F01184D0F0118890F0118CD0F0118BB
:10C530002710011857100118A3100118CF10011867
:10C540000D2D0118412D0118672E0118ED2F01182E
:10C5500035330118BF330118633401187F310118D6
:10C560008735011800000000FB350118EB36011873
:10C57000A74301189D3B0118D73B01189B3C0118AC
:10C58000573D0118DD400118DD400118C541011873
:10C59000DB3F01189142011800000000B54201186C
:10C5A000174301184D4301184D4301185B700118E2
:10C5B0002D76011857570118B760011861610118ED
:10C5C000C76101180B62011899550118A56401187B
:10C5D0003965011827600118756001186B59011839
:10C5E00059550118EF6401183B7101184F72011879
:10C5F0007955011800000000000000007368011860
:10C60000DF680118D37A01185F7B0118C17B01181C
:10C610000C010801020F17070D050105010D0201AC
:10C6200009010901010101030601020509011801BF
:10C6300018010305000000000901090103010301BD
:04C6400005010000F0
:0400000500000000F7
:00000001FF
